:020000040800F2
:1000000000000110551107086D2900082926020873
:10001000F5110708F5110708F511070800000000A1
:10002000000000000000000000000000E54400089F
:10003000E944000800000000ED44000851070108F1
:10004000F5110708F5110708F5110708F51107085C
:10005000F5110708F51107087DC0000881C00008E8
:10006000F511070885C0000889C000089131000813
:10007000A5310008B9310008CD310008E131000890
:10008000F531000809320008F5110708F5110708D5
:10009000F5110708F5110708F51107088DC00008CC
:1000A0003D300008653000088D3000082930000818
:1000B000B5300008C9300008DD300008F511070828
:1000C000F5110708F5110708F5110708F5110708DC
:1000D000F5110708D52A0008E12A0008ED2A0008D2
:1000E00091C00008F5110708F14400081931000813
:1000F0004131000869310008053100081D3200084F
:10010000F5110708F5110708F1300008F511070887
:10011000F92A0008052B0008F5110708F511070852
:1001200031320008453200085532000865320008B7
:1001300075320008F5110708F5110708F5110708D1
:10014000F5110708F5110708F511070845450008DE
:100150008532000899320008AD320008112B0008E2
:10016000F5110708F5110708F5110708F51107083B
:10017000F5110708F5110708F5110708F51107082B
:08018000F5110708F51107084D
:10019000D0E907239A422FBFD01AC0688018C01A2E
:1001A000704700BFD0E9092300699A4238BF12188E
:1001B000D31A0138C01A7047D0E90902101AB0FAF0
:1001C00080F04009704700BF0246036A4069D16869
:1001D000C05C01338B4228BF00231362704700BF0D
:1001E000436A8269D154436A0169426B01338B428D
:1001F00028BF00234362D36843F08003D360704775
:10020000436B188810F0100002D01A889B880120D8
:10021000704700BF436B99891A88890610B5044658
:100220000AD592B2900607D5E26A002A29D09888AA
:10023000216B80B29047636B99891A88090692B244
:100240000FD510060DD5D4E909128A4214D0A16940
:100250002069895C99800132B2FBF0F100FB112228
:10026000A262998A1A88C90592B204D5D20744BFFE
:100270004FF6F7721A8010BDDA6822F08002DA6059
:10028000EFE79B88E2696169DBB28B54E269E16860
:10029000636B0132B2FBF1F001FB1022E261CBE7AC
:1002A000036942681F2B10B40AD95468A3F1200CCB
:1002B000202101FA0CF1214207D15DF8044B70476F
:1002C0001468202199402142F7D081690024C86830
:1002D0000C7480684C68016821F00101016020689D
:1002E00094F805C00C4C818934F81C4089B221EA8D
:1002F00004011F2B818107D9A3F1200120238B400A
:100300005DF8044BD3607047202101FA03F35DF8D8
:10031000044B9360704700BF086A070882B0092247
:10032000274B8DF80720DA68D00319D4DA68D10694
:1003300040D4DA68D20541D4DA6812F0E00F3BD13C
:10034000DB6813F0020F14BF082309238DF8073070
:100350009DF80730012B0AD09DF8070002B07047C6
:1003600001238DF807309DF80730012BF4D1144A92
:1003700012E0D368DB0519D4D36813F0E00F17D16E
:10038000D36813F0020F14BF082309238DF8073038
:100390009DF80730012BDFD1D168C8034FF001036E
:1003A000F4D4D368D906E4D50623EFE70223EDE7BA
:1003B0000723EBE70623D4E70723D2E70223D0E79E
:1003C000003C0240704700BF704700BF01207047EB
:1003D000044BD3E90003984288BF03F50063181A61
:1003E000704700BF60200020054AD2E900318B42EF
:1003F000FDD0D1180133C3F30A03087A13607047A4
:1004000060200020064BD3F8080800B97047D3F8E5
:100410000808A0F10500B0FA80F04009704700BF5D
:1004200060200020012380F849307047064BD3F844
:100430000C08D3F81028431E90428CBF00200120E6
:100440009B1A03EBC02070476020002010B5D0F845
:10045000E83504461B699847032384F812310020CD
:1004600010BD00BF08B5042290F81211D0F8E8358D
:1004700080F8131180F81221DB689847002008BD2E
:1004800008B5D0F8E435DB6903B19847002008BD12
:1004900008B5D0F8E4351B6A9847002008BD00BFB6
:1004A00008B5D0F8E4355B6A9847002008BD00BF66
:1004B000037830B403B30446C0F1010C04EB0C0321
:1004C00014F8015FDBB2002DF8D101335B00DCB220
:1004D000138003230C704B7004785CB10223002559
:1004E0005A1CD2B2CC548D5410F8014F0233DBB2F7
:1004F000002CF5D130BC704702242346E8E700BF4A
:1005000010B5074C2068FF2808D00649D1F81428F8
:1005100001F6180100F080F8FF232360002010BDD1
:100520000000002060200020432301480B8070471A
:1005300004000020122301480B807047480000206F
:10054000042301480B8070475C00002008B5044B71
:1005500004480A461946FFF7ABFF084608BD00BF2E
:1005600080280020B0FD070808B5044B04480A465F
:100570001946FFF79DFF084608BD00BF80280020F0
:10058000C0FD070808B5044B04480A461946FFF7A2
:100590008FFF084608BD00BF80280020C8FD07085F
:1005A00008B5044B04480A461946FFF781FF084680
:1005B00008BD00BF80280020D4FD070808B5044B03
:1005C00004480A461946FFF773FF084608BD00BFF6
:1005D00080280020E0FD0708704700BF704700BF7B
:1005E000704700BF704700BF704700BF704700BF33
:1005F000044B00200522C3F80828C3F82009C3F8DB
:100600002409704760200020024B0020C3F808082E
:10061000704700BF60200020212838B50C4605D067
:1006200022282DD0202813D0002038BD0029FBD04F
:10063000072AF9D1194BD3F8280993F82C1993F804
:100640002D2993F82E39206021716271A371EBE797
:100650000029E9D0072AE7D1104DD5F8243913B184
:10066000096800209847206821796279A379C5F844
:10067000280985F82C1985F82D2985F82E39D3E716
:100680000029D1D0022ACFD1044BD3F82039002B36
:10069000CAD0098800209847C6E700BF6020002024
:1006A00010B4144CD4E900239A4286BF03F5006CC1
:1006B000ACEB02029A1A0A44B2F5006F13D8B1B13A
:1006C00001444A1E013810F801CFE118824203F1BB
:1006D000010381F808C0C3F30A03F4D1636000206A
:1006E0005DF8044B704702205DF8044B70470846E4
:1006F000F6E700BF602000201D49D1F884391A793F
:10070000022A00D0704710B41A4C93F9102002EB63
:10071000820204EB8202126E1089800708D51289CA
:10072000100605D49A6892070BD45DF8044B704705
:1007300000BFD1F884391A79022AE6D05DF8044B5B
:100740007047D1F888190C480C4A4FF4FA7404FB2E
:1007500001F1A2FB0121446889094268121B914200
:10076000FBD25B69002BE0D01A689B881383DCE71F
:100770006020002000000020001000E0D34D621037
:10078000034B93F85409003818BF0120704700BF8D
:1007900060200020034B93F85409032894BF0020E5
:1007A000012070476020002000487047B8290020D1
:1007B00030B4194B00209C7B14B11D688D4206D0CB
:1007C0000130082803F11003F5D130BC70479AB10D
:1007D000124B03EB40218A4219D0114B93F8B421FC
:1007E0008AB1104B01225A7000F5817003EB0010A2
:1007F0000123837130BC70470A4B00F5817003EB15
:1008000000108271E1E7012283F8B421E9E7022CAC
:10081000E3D1183BE8E700BFB85C0020B84C0020EB
:10082000A05C0020A04C002030B41D4C002384F8B4
:10083000A03004F1180004E00133082B00F110008F
:100840001ED005688D42F7D190F80EC0BCF1030FA1
:10085000F2D1BAB1134901EB4320824209D094F896
:10086000B42112B9012284F8B4210F4901224A703F
:1008700000E0183903F5817301EB031301229A712B
:1008800030BC70470849D4F89C2003F5817301EB14
:100890000313013204219971C4F89C20F0E700BFD2
:1008A000A05C0020B84C0020A04C0020A8B18368B8
:1008B0001BB10E4B07229A7070470C4A1178D36017
:1008C00003294FF004000CBF80214FF48071C2E96E
:1008D00001111361137590707047044A02F580513D
:1008E0000123537081F8B431704700BFA04C002041
:1008F00010B5812104466FF0FBF8204601216FF00E
:10090000F7F8204682216FF0F3F8FFF77DFE002014
:1009100010BD00BFC169026910B4002340F2011488
:10092000A0F844410B60D169846D21F002014FF0C1
:10093000010CD161A0F89CC32360D169044821F463
:10094000003180F88C395DF8044BD161184670474E
:1009500060200020202301480B807047B000002059
:10096000122301480B807047D00000200423014867
:100970000B807047E40000200A4608B5054920B9FD
:100980000548FFF795FD034808BD0448FFF790FDB3
:10099000004808BDF0290020F0FD070808FE070800
:1009A00008B5044B04480A461946FFF781FD08467E
:1009B00008BD00BFF029002020FE07082048D0F81D
:1009C000E837D0F8EC2730B59B184FF01A040C80AC
:1009D00001D11C4830BD1B4AD0F8EA174FF0000E79
:1009E00010467546B3F1204F4FEA137C0CF13004EA
:1009F0000EF1020E2ABF0CF1370C847080F802C091
:100A0000BEF1100FC5704FEA031300F10200E9D1E7
:100A100000200446B1F1204F4FEA117303F1300C6E
:100A200000F102002ABF373382F812C093740828FD
:100A3000D4744FEA011102F10202EBD1014830BD3A
:100A400000F0FF1FE800002008B5044B04480A46E8
:100A50001946FFF72DFD084608BD00BFF02900200C
:100A600034FE070808B5044B04480A461946FFF748
:100A70001FFD084608BD00BFF029002040FE070802
:100A800010B50F4C0F4BD4F8381BB4F83C0B08834F
:100A900003F58272C4F8DC2CD3F80431984702E0E5
:100AA0001B69984720B9D4F8DC3C002BF8D1FEE74D
:100AB000D4F8383BB4F83C2B5A83002010BD00BF5B
:100AC000602000200000002038B5084BD3F8DC3C43
:100AD00053B1DB6914460D4698474FF40073026822
:100AE0002A600020236038BD1B68FFDE60200020E4
:100AF00008B5074BD3F8DC3C33B11B69984780F04D
:100B00000100404240B208BD4FF0FF3008BD00BFB9
:100B100060200020002070472DE9F041164CD4F8E9
:100B20002C0B1646B4F8302B428303B30F4603EB6D
:100B3000060806E000234D681A4639463046A847A5
:100B400038B9D4F8DC1C0029F4D1FEE71B699847BA
:100B500020B9D4F8DC3C002BF8D1FEE70136B045D3
:100B600007F50077EDD1D4F82C0BB4F8302B0283C5
:100B70000020BDE8F08100BF602000202DE9F04199
:100B8000184CD4F82C0B1646B4F8302B42832BB3F8
:100B90000F4603EB060801E00B699847D4F8DC1C0C
:100BA00051B10023CD681A4639463046A847D4F8DB
:100BB000DC1C08B10029EFD131B10B69984720B98D
:100BC000D4F8DC1C0029F8D1FEE70136B04507F562
:100BD0000077E3D1D4F82C0BB4F8302B028300203B
:100BE000BDE8F081602000202DE9F041204E96F80C
:100BF000E03C002BFBD1B9B3014400F1FF384F1E9C
:100C0000D6F81018D6F80C3818F8010F4A1CC2F3A1
:100C10000A029A4234BF002401249B1A314403EB98
:100C2000C423012B81F8E40CC6F810281AD10FF068
:100C3000DBFD04460D460FF0D7FD031B61EB0501FC
:100C4000B3F57A7F71F10003F5D3D6F80C38D6F8F6
:100C5000102893428CBF002101219B1A03EBC12372
:100C6000012BE4D0B845CBD10020BDE8F08100BF16
:100C7000602000200A4B10B5D3F8084804B910BD15
:100C8000D3F80838052BFAD1064C002A0846D4F8C8
:100C9000EC331146F3DDFFF7A7FFD4F8EC3310BDBA
:100CA000602000205831002090F84820531C024456
:100CB000DBB280F8483082F8341090F849200AB14D
:100CC000132B03D9002280F8482003B970470A4A41
:100CD000D2F808180029F9D0D2F80828052AF5D149
:100CE00010B5064C19463430D4F8EC33FFF77CFFCE
:100CF000D4F8EC3310BD00BF602000205831002034
:100D000090F848100023A0F8483001B97047094B0B
:100D1000D3F80828002AF9D0D3F80838052BF5D1E4
:100D200010B5054C3430D4F8EC33FFF75DFFD4F840
:100D3000EC3310BD60200020583100202DE9F04731
:100D40005D4E1F4606EB80039C68002C00F0AD80D2
:100D500004F13E03A36104F59F73E3614FF48073D4
:100D6000C4E904332836236866600546E16094F8D8
:100D70003D00A363904606F06FF9814694F8440263
:100D800094F83CA0261D00284FD194F8450268BB7A
:100D9000D4F8403283BB390734D418F0020F60D145
:100DA00018F0010F44D194F9472294F84712D4F86F
:100DB0004832002A10DB41481B018418DBB284F85A
:100DC00000335209012301F01F0103FA01F140F839
:100DD00022103046BDE8F087394A01F00F010A447D
:100DE0001B01DBB213763046BDE8F0876CF0CAFE1B
:100DF000D4F84032002BCED0324A116B0B43390766
:100E00001363CAD50135EDB2B9F1000FCBD040F272
:100E10000673FA0689F80850A9F8063036D4BB06DE
:100E200094F8462245D4322133E06CF0ABFEACE7B7
:100E3000504606F011F90135EDB20028B3D040F26A
:100E400006620572C28094F8462202210BF022F954
:100E500094F9472294F84712D4F84832002AAADAC3
:100E6000BAE76B1CDBB2B9F1000F99D089F80830F2
:100E700040F20653A9F8063094F84622484602216B
:100E80000BF008F918F0010F8DD0D1E794F8462245
:100E9000022148460BF0FEF894F9472294F84712D5
:100EA000D4F84832002A86DA96E726463046BDE86E
:100EB000F0871221EDE700BF086A070800E100E0B3
:100EC000FCEC00E0003802402DE9F047038A8489F9
:100ED000A4B21C4082B045D0814688464FF0004500
:100EE00001F14C0701F13406B4FA84F325FA03F258
:100EF000D24391B2A9F8101014401B3BB8F1000F77
:100F00005DD0042B2CD8DFE803F050463B300300C3
:100F1000D8F80C30D9F82CA033B19B6823B11FFA54
:100F20008AF108F104009847D8F8243033B19B685F
:100F300023B11FFA8AF108F11C009847D8F83C3019
:100F40002BB19B681BB11FFA8AF130469847D8F83D
:100F500054302BB19B681BB11FFA8AF13846984771
:100F6000002CC1D102B0BDE8F087D8F80C30D9F818
:100F700034105B6808F104009847002CB4D1F1E705
:100F8000D8F82430D9F838105B6808F11C0098476D
:100F9000002CA9D1E6E7D8F83C30D9F83C105B68C2
:100FA00030469847002C9FD1DCE7D8F85430D9F868
:100FB00040105B6838469847002C95D1D2E7042B47
:100FC00007D8DFE803F00319140F0A00D9F84030FE
:100FD0000193019B002C87D1C4E7D9F82C300193F1
:100FE000019BF7E7D9F834300193019BF2E7D9F878
:100FF00038300193019BEDE7D9F83C300193019B18
:10100000E8E700BF38B5284C94F8E02C012A0346E5
:1010100003D0022A09D0002038BD2449D1F8F0239A
:10102000A2B984F8E02C002038BD002540F201125E
:10103000C0E95455C0E95655A0F8442100F5A27105
:101040006EF066FE84F8E05C002038BD402AD4F8DB
:101050000C0819D9403AC1F8F02340228118C4F88D
:101060000C1880B2124940F2011401440020C3E977
:101070005411C3E95620A3F84441184603F5A27160
:101080006EF046FE002038BD4FF00005C1F8F05369
:1010900002EB0001C4F80C1808BF022180B208BF9F
:1010A00084F8E01CDEE700BF6020002058310020FB
:1010B000442D002001EB810138B500EBC1010E4D3C
:1010C000B1F88C1304462846FFF7EAFAE378C4F82F
:1010D000A85340210022C4E9EC1201229342204689
:1010E000A4F89C2304F5677108BFC4F8AC536EF0F4
:1010F0000FFE002038BD00BF4C35002038B52A4B0C
:10110000D3F834240F2A04D0511CC3F8341400201F
:1011100038BD264A92F8E05C0021C3F83414002D53
:10112000F5D1D2F80C18D2F81048B1F5006F30D0D4
:10113000A14235D002F6E44594BF641AC1F50064BB
:1011400015FA81F5402C19D82144C2F80C184FF03B
:101150000001C3F8F0130CBF0223012382F8E03C26
:1011600040F201120023C0E95455C0E95643A0F8EB
:10117000442100F5A2716EF0CBFDC8E7403CC3F8F6
:10118000F04340310123C2F80C1882F8E03C4024BF
:10119000E6E7C2F80C581CB1294602F6E445D1E74F
:1011A000002382F8E03CB2E75831002060200020A4
:1011B00038B5224DD5F8403495F858C4044623B1CB
:1011C00095F844345CEA030331D00123E06984F8E4
:1011D000463140F20112A4F8442102681849002A5D
:1011E000A8BFC2F380739B0301EA124143F02003BE
:1011F0000B4363F31F42BCF1020F026000D038BD05
:10120000E278104BC4F8A8331F200021C4E9EC0198
:10121000012A4FF00101A4F89C1308BFC4F8AC33B5
:1012200004F567712046BDE838406EF071BD0121BC
:101230006EF024FC95F858C4C7E700BF5831002071
:10124000DFBFFFFF9035002070B590F8CF2590F8F4
:10125000D13590F8CE5590F8D0C590F8CC1590F8CF
:10126000CD6505EB02250CEB032C90F8D32590F807
:10127000D23503EB0223012284B080F8112101F062
:101280001F029BB2ADB21FFA8CFC012A04468DF8F6
:101290000810ADF80A50ADF80CC0ADF80E30C0F82B
:1012A00040318DF809600AD0022A57D0002A3CD07C
:1012B00001F080016EF0E2FB002004B070BD90F8F8
:1012C0001231032B2BD15FFA8CFCBCF1010F26D815
:1012D000D0F8E43502A99B689847BDF80E30002B82
:1012E000EAD1C4E94A33C4E94C3304214FF4807293
:1012F00084F81111A4F81C2104F58E7120466EF0BB
:1013000099FC636DC44A1A61E278012AD4D104F2CF
:10131000CC545C614FF0802219681A60CCE72046FB
:101320006BF0BCFE002004B070BD092EF7D801A2FE
:1013300052F826F0DF130008EF1400081F1300080E
:10134000291500081F13000857150008031400088A
:101350001F1300086D1400089D14000801F06001BF
:1013600020295FFA8CF334D0012E00F06181032E26
:1013700000F09581002E9FD190F81221022A00F0F2
:101380001B81032ACBD11CF0800F40F0A48103EB1A
:10139000830300EBC30393F87633002B00F0A681A0
:1013A0009E4B0122C3F868249D4A0223C4E94E33B0
:1013B0004FF48070002184F81131A4F81C01C4E9B5
:1013C0004C31C4E94A2204F58E7120466EF032FC9D
:1013D00072E7D0F8E43502A99B6898476CE790F86B
:1013E0001231023B012B9AD88C4BD0F818210021E6
:1013F000C3F8601412B10222C3F86024894A0223A0
:10140000D4E72E0A022EADF8063000F0CD81032E6F
:1014100000F09181012E82D1D0F8EC3580781B68E4
:101420000DF106019847BDF80630002B3FF444AF9C
:10143000BDF80E20002A3FF43FAF934228BF134669
:101440004FF480720221A4F81C210022C4E94A0052
:1014500084F81111C4E94E33C4E94C3204F58E719D
:101460002046ADF806306EF0E5FB25E7012B7FF452
:1014700056AF90F81221022A00F04981032A7FF426
:101480004EAF4FF4807100F588720220A4F81C1151
:10149000C4E94E3384F81101002190E7EDB25F4EAC
:1014A000012D86F859543FF63AAF90F81231022BCD
:1014B00000F02181032B7FF432AF002D00F07F81FB
:1014C00090F81011012910D0D0F8E4355B689847E6
:1014D00096F85914D4F8E43584F810111B682046A6
:1014E0009847D4F8E8359B6898470023F9E690F8C8
:1014F0001231023B012B3FF612AF012D7FF4DCAE1F
:10150000D0F8E43500259B68C0F8185102A9984727
:1015100004224FF48073C4E94A55C4E94C5584F859
:101520001121A4F81C31E7E6012D00F0CC80022D3A
:101530007FF4C2AE5FFA8CF3002B7FF4BDAE02697C
:101540004FEA1C23023B5268032B00F25681DFE86E
:1015500003F05B426B5F5CEA03037FF4E0AE90F85C
:101560001221032A3FF4DBAE016905F07F0680F803
:10157000146108681A4665F30A1202430A604FF4C0
:1015800080720421C4E94A33C4E94C3384F8111150
:10159000A4F81C2104F58E7120466EF04BFB636DA0
:1015A0001D4A1A61E278012A0DD0002E00F0128146
:1015B000022384F812317FE65A063FF47DAE1946C5
:1015C0006EF05CFA78E604F2CC525A614FF0802259
:1015D00019681A60E9E7032363F3061201210F4D2E
:1015E00084F816110421002384F811114FF480713E
:1015F000A4F81C11C4E94A33C4E94C3304F58E71D4
:101600002046C5F864247AE6022363F30612E5E770
:10161000052363F30612E1E7180008605831002043
:10162000C0350020B8350020042363F30612D5E747
:1016300090F81221022ABFD0032A7FF470AE002D49
:101640007FF43AAE13F07F023FF44FAF1CF0800FEF
:1016500040F0C48003EB830100EBC10181F87423E7
:1016600081F8765381F87553282101FB030300EBC1
:10167000820293F87713506D03688A1E012A6FF374
:101680005553D4F8E4258CBFC3F30071012161F3F5
:101690001C739268036002A92046904725E790F8E2
:1016A0001221022A88D0032A7FF439AE25B95906BF
:1016B00002D019466EF0E2F9D4F8E43502A99B682D
:1016C0002046984711E7D0F8E43502A99B68C0F896
:1016D0001851984709E703F07F0303EB830300EBFE
:1016E000C30393F81E31002B7FF45AAE454B002202
:1016F000C3F8682458E6002D3FF40AAF0121032205
:10170000D0F8E43580F8101180F81221E6E63E4961
:1017100084F811214FF480700022C4E94A11A4F822
:101720001C01C4E94E33C4E94C3204F58E712046E5
:101730006EF080FAC0E5EDB2052D3FF6F0ADDFE8C2
:1017400005F02B231B130B03D0F8EC3580789B6935
:101750000DF10601984766E6D0F8EC3580785B69B4
:101760000DF1060198475EE6D0F8EC3580781B69EC
:101770000DF10601984756E6D0F8EC358078DB6825
:101780000DF1060198474EE6D0F8EC3580789B685D
:101790000DF10601984746E6D0F8EC3580785B6895
:1017A0000DF1060198473EE6D0F8E43580789B6A53
:1017B0000DF1060198474670C4F8F00533E60222A1
:1017C000D0F8E43580F8122180F810515B68294682
:1017D00098479DE6012384F812316DE5282303FB29
:1017E000020181F81C2100EB820281F81E5181F870
:1017F0001D61906991F81F113EE7012363F3061202
:10180000ECE600BF58310020B435002010B5044686
:1018100029B990F81121032A0DD0002010BDD0F86D
:10182000E4359B69002BF8D090F81221032AF4D1FB
:101830009847002010BDD0F890230B46D0F87C13B9
:101840008A4213D9C078521A0128C4F8902336D09E
:101850008A4228BF0A4692B2C4E9E22304F55D71C8
:10186000A4F8743320466EF0E5F9D6E7D0F8E435F5
:101870001B691BB190F81221032A1ED000234FF4DC
:1018800080720421C4E94A33C4E94C3384F811114D
:10189000A4F81C2104F58E7120466EF0CBF9636D1F
:1018A000104A1A61E278012AB7D104F2CC545C6183
:1018B0004FF0802219681A60AFE79847DEE78A4246
:1018C000D4F88003A4F8743328BF0A46084492B2BF
:1018D000C4E9E22304F55D71C4F88003C4F884030D
:1018E000C0E700BF1800086038B5044649B990F851
:1018F0001131022B11D094F81631012B40D0002069
:1019000038BDD0F8E4355B69002BF8D090F812218F
:10191000032AF4D19847002038BDD0F83831D0F8E8
:101920002421934236D9C178012908BFD0F8281163
:10193000A3EB020318BFD0F82821C0F8383108BF44
:1019400052189BB24FF480710025C0E94C35A0F8C5
:101950001C11C0E94A2200F58E716EF06BF9E37834
:10196000C4F88053012BC4E9E255A4F8745308BFAE
:10197000C4F8845304F55D7120466EF05BF9BAE754
:101980002A4B2269D3F864145160002384F816317D
:10199000002038BDD0F83C31B3FBF2F502FB153521
:1019A000ADB99A4213D8D0F8402193420FD24FF4E8
:1019B0008073A0F81C31C0E94A55C0E94C5500F5C8
:1019C0008E716EF037F9E378C4F84051C8E7D4F867
:1019D000E435DB681BB194F81221032A23D0E278A6
:1019E0000023012A4FF0050108BFC4F88433C4E97D
:1019F000E23384F81111C4F88033A4F8743304F589
:101A00005D7120466EF016F9636D094A1A61E2783D
:101A1000012A7FF470AF04F2CC525A614FF0802259
:101A200019681A6067E720469847D8E758310020C0
:101A300018000860F8B50B7813F060060D460446F0
:101A400020D0202E25D1CE884EB31B0649D5384F45
:101A5000687832463946FEF7DFFDEB880222002621
:101A600084F811214FF48072C4E94E33C4E94A77F7
:101A7000C4E94C36A4F81C2104F58E7120466EF0A2
:101A8000D9F80AE04B780A2B17D00B2B0ED0062B77
:101A900003D120466BF002FB02263046F8BD02223D
:101AA00048781144FEF7B8FD3046F8BD8B78002B1E
:101AB0003AD1204BC3F86C64EFE7022280F8112181
:101AC0004FF48072A0F81C211B4A0123C0E94E3359
:101AD000C0E94A22C0E94C3600F58E716EF0AAF8D2
:101AE000DBE7164B164A4978116003F6180203210A
:101AF000C0E9E46680F81111C0F88863C0F880235B
:101B0000C078C3F8146801284FF00003C4F88C3380
:101B1000A4F8743304F55D7108BFC4F8842320462B
:101B20006EF088F80026B8E76BF0B8FAB5E700BFAA
:101B30007828002058310020C43500206020002083
:101B400000000020002310B51946044640226EF024
:101B500001F880212046002340226DF0FBFFD4F8DD
:101B6000E835A078012284F812215B6898470020AC
:101B700010BD00BF10B502230446402281216DF044
:101B8000E9FF20460223402201216DF0E3FF2046B9
:101B90000323082282216DF0DDFF0E4B0222A3F801
:101BA0004C20FEF725FDE2780B4BC4F8A83340200B
:101BB0000021C4E9EC01012A4FF00101A4F89C13B3
:101BC000204604F5677108BFC4F8AC336EF0A0F886
:101BD000002010BD000000204C35002070B5812190
:101BE00082B00446314E6DF083FF012120466DF036
:101BF0007FFF0025022340228121204686F88C5950
:101C00006DF0A8FF01210223402220466DF0A2FFC3
:101C1000274B86F88C59D3F8702483F858541268EF
:101C2000284690470095009BE16843F0100300931D
:101C3000009B0B610A691F4B009203E00A69009246
:101C4000013B02D0009AD006F8D400230193019BF7
:101C500043F020030193019A164B012060F38A128E
:101C60000192019A0A610A69019203E00A690192EC
:101C7000013B02D0019A9206F8D4E2780E4BC4F8E8
:101C8000A83300211F20C4E9EC01012A4FF0010113
:101C9000A4F89C1304F5677105D020466EF038F85F
:101CA000002002B070BDC4F8AC33F6E7602000201D
:101CB00058310020400D03009035002010B5144C21
:101CC000D4F8803943B119689A880B691A4203D154
:101CD000002384F8543910BD94F85439032B10D8DC
:101CE00094F848390133DBB2072B84F84839EFD830
:101CF000084A0123D2F8EC23C4F8442984F8543963
:101D000010BDD4F88409002107F048FEE8E700BFC1
:101D100060200020583100202DE9F047294FDFF8DE
:101D2000AC90294CDFF8A8A082B000F10108002691
:101D300006E09DF80700FF282FD1013646452CD03C
:101D4000D7F8845995F91030AA6803EB830309EB9F
:101D500083039207186E23D5012300220DF107019A
:101D60006EF088F8AB689B07E3D4D7F888296168E0
:101D70004FF4FA7303FB02F2AAFB02329209636882
:101D80005B1A9A42FBD26B69002BD2D09DF80700F8
:101D90001A689B881383FF28CFD002B0BDE8F08774
:101DA0006B6913B11A689B885383D7F888296168D7
:101DB000D200AAFB0232920963685B1A9A42FBD2F4
:101DC000CAE700BF60200020001000E000000020F3
:101DD000D34D621070B5044608200D46FFF79CFFF6
:101DE000FF2822D0FE2801D0022070BD254E2146BA
:101DF000D6F884092B4600226EF08CF8D6F8844978
:101E0000214A94F91030A16803EB830302EB8303AA
:101E10008A07186E0BD50022022311466EF02AF8AD
:101E2000A3689B0716D5002070BD012070BD6369B3
:101E300013B11A689B885383D6F888291349144B29
:101E40004D68D200A3FB023292094B685B1B9A4299
:101E5000FBD2E0E7D6F888290C490D4B4FF4FA7015
:101E600000FB02F2A3FB0232486892094B681B1A7E
:101E70009A42FBD260690028B7D0036882881A832F
:101E8000002070BD6020002000000020001000E055
:101E9000D34D621070B52F4C2F4AD4F8845995F960
:101EA000103003EB830302EB8303AA6882B00020A7
:101EB0004FF6FF519207C4F85009ADF80410186EA0
:101EC00034D5022301AA00216DF0D4FFAB689B0733
:101ED00015D50120FFF720FFFF280AD01F4BD3F8AC
:101EE000EC33C4F844390922002084F8542902B0A4
:101EF00070BD0423022084F8543902B070BDD4F8B8
:101F000088391749174E48684FF4FA7203FB02F2FA
:101F1000A6FB023292094B681B1A9A42FBD26B69EC
:101F2000002BD6D01A689B881383D2E76B6913B154
:101F30001A689B885383D4F888290949094B4E684D
:101F4000D200A3FB023292094B689B1B9A42FBD240
:101F5000B7E700BF602000200000002058310020BB
:101F6000001000E0D34D621070B582B004460B0E35
:101F7000080C0A0A44F040058DF8013095238DF8CD
:101F800000508DF802008DF803208DF804108DF8B4
:101F900005306BF021F808B9002C44D1234D244AB8
:101FA000D5F8844994F91030A16803EB830302EB60
:101FB00083038A07186E0CD506236A4600216DF04C
:101FC00059FFA3689B0717D50820FFF7A5FE02B0AD
:101FD00070BD636913B11A689B885383D5F888294B
:101FE0001449154B4E68D200A3FB023292094B688C
:101FF0009B1B9A42FBD2DFE7D5F888290D490E4B8F
:102000004FF4FA7000FB02F2A3FB02324868920917
:102010004B681B1A9A42FBD26369002BD4D01A6812
:102020009B881383D0E7FF2002B070BD60200020A2
:1020300000000020001000E0D34D62102DE9F041B7
:102040003A4C82B00546884617461E4694F8540915
:1020500004280DD0082807D1D4F84C39AB425FD002
:10206000FFF718FF0228F1D0012002B0BDE8F0818F
:10207000D4F884391A79022A36D094F84A398BBBBD
:1020800069021820FFF770FF002843D194F85439F3
:10209000082B4FF0FF038DF804300CBFFC23FE2308
:1020A000D4F884098DF8053001AA022300216DF0CF
:1020B00031FFD4F884094246802300216DF02AFFC5
:1020C000012206230020C4F83089C4F83459C4F82A
:1020D0003C79C4F8406984F8382984F8543902B04E
:1020E000BDE8F0812946CCE79A689207C5D55B69BF
:1020F00013B11A689B885383D4F888390C49DA00E5
:102100000C4B4868A3FB023292094B681B1A9A4297
:10211000FBD2B2E7FEF7F0FAFFF7D0FD0320A4E709
:10212000FF238DF80430FC23BAE700BF60200020B5
:10213000001000E0D34D621070B51F4C94F8543974
:10214000042B06460D4609D0082B25D1D4F84C396E
:1021500083422FD0FFF79EFE02281DD1D4F88409B8
:1021600007F068FC00213720FFF7FEFE2946172004
:10217000FFF7FAFEC0B994F84A397BB97102192009
:10218000FFF7F2FE80B9082384F85439C4F8505997
:10219000C4F84C69022070BD012070BD3146192081
:1021A000FFF7E2FE0028EED0FEF7A6FAFFF786FD65
:1021B000032070BD022070BD602000202DE9F04199
:1021C000294C94F854C9BCF1040F074688461646BA
:1021D0001D4609D0BCF1080F02D00020BDE8F081F7
:1021E000FFF758FE0228F8D1D4F884391A79022A68
:1021F00023D094F84A39BBB979021120FFF7B4FE15
:10220000C0B91A4BC4F83089D3F8EC33C4F8347928
:10221000052284F85429C4F83C69C4F84059C4F82C
:1022200044390120BDE8F08139461120FFF79CFEBA
:102230000028E6D0FEF760FACFE79A689207D8D573
:102240005B6913B11A689B885383D4F888390849AD
:10225000DA00084B4868A3FB023292094B681B1A4C
:102260009A42FBD2C5E700BF602000205831002011
:10227000001000E0D34D62102DE9F043844CD4F8F7
:10228000840987B0002836D094F85409814D824ED5
:10229000824F431E082B1CD8DFE813F09400BF00C8
:1022A00042011B000900590041001B003000D4F816
:1022B00030094FF40071FFF78DFD012800F0968181
:1022C000022800F09B81002800F0CC8194F854098A
:1022D000431EDBB2022B00F2D6806E4BD4F84429A9
:1022E000D3F8EC339B1AC82B00F29E81A0F10800B2
:1022F000B0FA80F0400907B0BDE8F0836AF06CFEE8
:10230000002840F06382D4F84439D5F8EC23FA333E
:102310009342DBD2FFF7D2FC94F85409B9E76AF094
:102320005BFE0028EFD0D4F850390022012B84F84E
:10233000482940F25382D4F84C29013B013208204D
:10234000C4F85039C4F84C2984F85409CEE7D4F8BD
:10235000303994F83829D4F8840903EBC2120021EB
:1023600080236DF0D7FD94F838390133DBB2042BAC
:1023700084F83839AAD1D4F88409022332460021DE
:102380006DF0C8FD0123D4F88409002202A96DF084
:10239000C1FD9DF8083003F01F03052B00F0FD81FF
:1023A000FFF78CFCD4F83C89B8F1000F00F03981BC
:1023B0000120D4F84039D4F834190022C04794F8E9
:1023C000540966E7D4F8840907F034FB0021084675
:1023D000FFF7CAFD8046FEF78FF9B8F1010F7FF4D1
:1023E00075AFD4F884094FF0000984F8499907F0D3
:1023F00021FB40F2AB110820FFF7B6FD052800F0E5
:102400001881012800F06181FEF776F994F84909F6
:10241000002899D0022384F85439D4F8840907F0AD
:1024200009FB94F84939022B0CBF4FF080484FF05C
:10243000000800213720FFF797FD41462920FFF7CC
:1024400093FD8046FEF758F9B8F1000F7FF43EAFD8
:1024500094F84939022B00F01B8184F84A89D4F89A
:1024600084391A79022A00F0E78000210920FFF759
:102470007BFDA8B1FEF740F994F85409431EDBB286
:10248000022B7FF62AAF04287FF430AF012032E719
:102490006020002058310020606A0708D34D621088
:1024A000D6481021FFF796FC0028E3D194F87F3935
:1024B000DB07DFD594F87019891100F01C81012920
:1024C000D8D194F87729DFF840E39200D2B21621F0
:1024D0004FF0020CCCF108038B4228BF0B46C3F12E
:1024E000080C42FA0CF29840C91A40EA02004FF078
:1024F000000C1EF8012FEDD1431C9B02C4F8583983
:10250000FEF7FAF8D4F8840907F094FA00210A20BB
:10251000FFF72AFD002840F0E780032384F85439B0
:10252000102102A8FFF756FC00287FF4CFAE9DF8DB
:10253000083084F85E39BDF809309DF816209DF802
:1025400010105BBAA4F85C399DF80B3084F85F3941
:102550009DF80C3084F860399DF80D3084F86139AD
:102560009DF80E3084F862399DF80F3084F8633995
:102570009DF815301B01DBB243EA121302F00F0283
:1025800003F5FA6384F86C29DDF81120A4F86A39A0
:102590000B0912BA84F8683901F00F0384F869391D
:1025A000C4F86429FEF7A8F894F84A397BB9D4F83E
:1025B000840907F03FFA4FF400711020FFF7D4FCB4
:1025C0008046FEF799F8B8F1000F7FF4A3AED4F877
:1025D0008409022107F0E2F9002204230120C4F853
:1025E000502984F8543907B0BDE8F083D4F8443951
:1025F000D5F8EC2364339342BFF468AEFEF77CF861
:10260000FFF75CFBD4F83C89B8F1000F09D0002239
:102610001046D4F84039D4F83419C04794F8540916
:1026200037E694F8540934E6FFF748FB94F8540968
:1026300029E784F84989E7E69A6892077FF515AF9C
:102640005B6913B11A689B885383D4F888396C4945
:10265000DA00A7FB0232486892094B681B1A9A42BB
:10266000FBD202E70190FEF747F8D4F83C590198F5
:1026700084F84809042384F85439002D3FF406AF48
:10268000D4F84039D4F83029D4F83419A8471DE6D5
:10269000D4F8840907F0CEF941463A20FFF764FCEC
:1026A000424681460423D4F8840902A96DF032FC25
:1026B000FEF722F8B9F1000F7FF42CAE029B1BBA93
:1026C000C3F3807384F84A39C9E60423D4F8840933
:1026D0004A4602A96DF01EFC9DF80B30AB2B04BFDF
:1026E000022384F849398FE6FEF706F8FFF7E6FA89
:1026F00094F85409CDE594F8753994F87909DFF820
:102700000C8103F00F0380014FF0010C0CFA03FC65
:102710005FFA80F903234FF0060ECEF108029A42C9
:1027200028BF1A46C2F1080049FA00F091409B1AEE
:1027300018F8019F41EA00014FF0000EEDD194F826
:102740007689DFF8CC904FEA881802315FFA88F872
:102750000C20062200E00022C2F10802824228BFBB
:102760000246C2F1080E48FA0EFE9340801A19F88C
:10277000018F4EEA0303EED1013303FA01F14FEA70
:10278000EC72A1FB0C3C01FB02C15B0A43EAC153A2
:10279000C4F85839FDF7B0FFB4E61A4BD4F83C59E9
:1027A000D3F8EC33C4F84439072084F85409002DD9
:1027B0003FF49CADD4F84039D4F83029D4F834191A
:1027C0000120A84794F85409431E82E50190FDF7C3
:1027D00093FF0423019884F854398CE508D004232E
:1027E00084F85439FDF788FF94F85409431E70E5C6
:1027F000FFF750FB02287FF469AD3BE6D0290020AB
:10280000001000E058310020D7290020D9290020ED
:10281000D6290020F8B500220C233221022009F02D
:1028200077FC374FC7F88409002866D0002107F0ED
:10283000B5F84FF47A760DF0D7FF04460D460DF04B
:10284000D3FF031B61EB0502B3F57A7F72F100033E
:10285000F5D3013EEFD1D7F884090379022B32D0AA
:1028600000220A2311466DF055FBD7F88409254C48
:1028700003792549022B0BD0244B0122D3F8EC130A
:10288000C7F84419002387F8542987F84839F8BD58
:1028900090F9103003EB830301EB83031B6E1A895D
:1028A000920702D51B891B06E6D5013CF0D107F043
:1028B00031F897F84839C7F88449013387F8544903
:1028C00087F84839F8BD83689907C9D5D7F888399A
:1028D0000F49104D4C684FF4FA7203FB02F2A5FB4E
:1028E000023292094B681B1B9A42FBD24369002BB0
:1028F000B6D01A689B881383B2E787F85409F8BDED
:1029000060200020A1860100000000205831002036
:10291000001000E0D34D62101049114BD1F888200F
:1029200042F4700210B4C1F888201A680D4C0020DF
:1029300042F001021A6098601A6822F0847222F450
:1029400080321A605C601A68074C22F480221A6098
:10295000D8608C605DF8044B704700BF00ED00E06C
:10296000003802401030002400000008704700BF0B
:102970002DE9F84346697EB9D0F80080C8F30D0907
:1029800004460F46B9F1000F26D03F68FDF7C6FC9C
:10299000092804D06FF001063046BDE8F8834A4D9F
:1029A0002B6923F440732B612B6943F400732B6173
:1029B0002B6943F001032B61C8F80070FDF7AEFCF2
:1029C0002B69092823F001032B61E3D12368043329
:1029D00023603046BDE8F8833C4B98452AD303F585
:1029E0008043984524D303F58043984554D3384B0E
:1029F000984554D903F58033984553D903F50033EE
:102A0000984552D903F50033984551D903F5003361
:102A100098453ED903F5003398454CD903F58023FA
:102A200098454BD9B8F1016F4BD305200DF038FF15
:102A30004FF00809FDF772FC092804D04FF0FF366B
:102A40003046BDE8F883204D2B6923F440732B6199
:102A50002B6943F400732B612B6923F0F8032B617E
:102A60002B6943EA090343F002032B612B6943F40A
:102A700080332B61FDF752FC2B6923F002032B619D
:102A80002B69092823F0F8032B61D7D1D4F80080F3
:102A90007BE74FF03809CDE74FF01009CAE74FF058
:102AA0001809C7E74FF02009C4E74FF02809C1E72C
:102AB0004FF03009BEE74FF04009BBE74FF048093F
:102AC000B8E74FF05809B5E7003C02400040000865
:102AD000FFFF00080148FDF79DBB00BF2801002053
:102AE0000148FDF797BB00BF740300200148FDF7C4
:102AF00091BB00BFC00500200148FDF78BBB00BFA4
:102B00000C0800200148FDF785BB00BF580A0020D3
:102B10000148FDF77FBB00BFA40C0020704700BF39
:102B2000F0B5254B0268254983B00646002401E034
:102B300051F834309A4209D001340E2CF8D10021DA
:102B40001F4A052006F038F8002113E01D4F07EB5F
:102B50008407D7F8745485B1717901EB410305EB13
:102B6000C30300221820C3E9032200FB01559E6025
:102B70001A75291D084603B0F0BD0721642006F030
:102B80000DF90146C7F8740470B12946642273F048
:102B90009EFE0A4BD7F8745403EBC404C5E9004504
:102BA000ED616D63ED64D7E70190074A052006F0FB
:102BB00003F80199DEE700BF00000140646A0708DE
:102BC00050FE07085831002078FE0708704700BF04
:102BD000B0B14B6810B4A3B18B6813B343681A68E3
:102BE000816058799189022383400B439BB2938182
:102BF00093899BB243F0010393815DF8044B7047C6
:102C0000704743681A685C7993894FF0020C0CFA9C
:102C100004FC9BB28C6823EA0C039381A4B181600D
:102C2000E6E744682268938923F001031B041B0C28
:102C300093818160607991895DF8044B0223834020
:102C40000B439BB293817047938923F001031B04CC
:102C50001B0C93818160D0E738B5D0E9004307EEC3
:102C6000902A1B68354A20680139934204688DB266
:102C700016D002F58062934212D002F57052934250
:102C80000ED002F5806293420AD002F58062934230
:102C900006D02B4BD3F8EC3E5B0807EE103A04E06D
:102CA000274B03F6EC6393ED007ADFED266AB8EE6E
:102CB000477AF8EE677A87EE270A30EE260A70F038
:102CC000D5FC1E4A23880138944280B29BB212D0B0
:102CD00002F5806294420ED0B4F1804F0BD0A2F581
:102CE0008032944207D002F58062944203D002F50C
:102CF0008062944202D123F070039BB2124A944244
:102D000012D002F5806294420ED023F4407302F593
:102D10006C429BB294422380E56220850AD1002355
:102D200023860123A38238BD2380E5622085012309
:102D3000A38238BD054B9C42F1D0F8E7000001406A
:102D4000000000200AD7233C00100040000401408E
:102D500070B54068837903F0020213F0040300F0B9
:102D6000C9804FF0000E134604247246754690F851
:102D700005C0BCF1030F30D8DFE80CF08E5F3002E5
:102D80000368188C20F480500004000C1884188C00
:102D90009C8820F4005000042A43000C40EA0232D0
:102DA000988B6C4D20F4E6400004000CAB42A4B2BA
:102DB00040F4C04000F0B08005F58065AB4200F003
:102DC000AB809C80988319641A849A8B22F40062E9
:102DD0001204120C42F400629A8370BD2A43056803
:102DE0005C4E288C20F480700004000C2884288C11
:102DF000B5F804C020F400700004000C40EA022280
:102E0000A88B20F073000004000CB5421FFA8CFC64
:102E100040F0600073D006F58066B5426FD0A5F82B
:102E200004C0A883E9632A84AB8B23F008031B0446
:102E30001B0C43F00803AB8370BD2A430568454E65
:102E4000288C20F010000004000C2884288CB5F891
:102E500004C020F020000004000C40EA0212288B7D
:102E600020F4E6400004000CB5421FFA8CFC40F44C
:102E7000C04061D006F58066B5425DD0A5F804C0BB
:102E80002883A9632A842B8B23F400631B041B0C67
:102E900043F400632B8370BD00682E4E2A43058CDB
:102EA00025F001052D042D0C0584058CB0F804C017
:102EB00025F002052D042D0C2A43058B25F0730502
:102EC0002D042D0CB0421FFA8CFC45F0600528D073
:102ED00006F58066B04224D0A0F804C005834163A3
:102EE0000284038B23F008031B041B0C43F008032C
:102EF000038370BD4FF4807E1C46012537E722F422
:102F0000006242EA032222F480622CF4405C42EA2E
:102F100004224CEA0E1C82E724F4804444EA8E1416
:102F20004FE74FF6F37616402CF4407C46EA030256
:102F30004EEA0C0C2243CFE722F0800242EA031251
:102F400022F040022CF4406C42EA04124CEA8E0C4F
:102F500094E700BF0000014070B4EFF3118210232A
:102F600083F31288C4684668A5682B6823F00103C0
:102F70002B603568114B767933F81660AB899BB2BC
:102F800023EA0603AB81236965681F2B11D9203B17
:102F9000202404FA03F3EB60D3B283F31188C368EF
:102FA0009B6859601A68012422431A60047470BC3B
:102FB0007047202404FA03F3AB60EDE7086A0708C2
:102FC00003681A7D012A04BF02221A7593F82C1097
:102FD0000CBF4FF400720022012904D1022183F8B2
:102FE0002C1042F4806293F84410012905D093F824
:102FF0005C1001290AD072B97047022183F844108D
:1030000093F85C10012942F4006204D1022183F894
:103010005C1042F480524168096800234B628B893E
:103020009BB21A438A817047024B0348D3F8741449
:10303000FDF74ABF583100200000014010B5064C92
:103040000648D4F87414FDF73FFFD4F894140448EC
:10305000BDE81040FDF738BF5831002000000140A6
:103060000040014010B5064C0648D4F87414FDF732
:103070002BFFD4F898140448BDE81040FDF724BF96
:1030800058310020000001400044014010B5064CBA
:103090000648D4F87414FDF717FFD4F89C140448BC
:1030A000BDE81040FDF710BF58310020000001407E
:1030B00000480140034B4FF08040D3F87814FDF7EF
:1030C00003BF00BF58310020024B0348D3F87C14E3
:1030D000FDF7FABE5831002000040040024B0348BF
:1030E000D3F88014FDF7F0BE5831002000080040EE
:1030F000024B0348D3F88414FDF7E6BE5831002094
:10310000000C0040024B0348D3F89014FDF7DCBEDE
:10311000583100200004014010B5064C0648D4F890
:103120009014FDF7D1FED4F8A0140448BDE8104077
:10313000FDF7CABE583100200004014000180040CD
:1031400010B5064C0648D4F89014FDF7BDFED4F82F
:10315000A4140448BDE81040FDF7B6BE5831002065
:1031600000040140001C004010B5064C0648D4F88D
:103170009014FDF7A9FED4F8A8140448BDE8104047
:10318000FDF7A2BE5831002000040140002000409D
:103190000348D0F8FC3E13B100F56F601847704744
:1031A000000000200348D0F81C3F13B100F5716007
:1031B00018477047000000200348D0F83C3F13B187
:1031C00000F5736018477047000000200348D0F8EE
:1031D0005C3F13B100F57560184770470000002090
:1031E0000348D0F87C3F13B100F57760184770476B
:1031F000000000200348D0F89C3F13B100F579602F
:1032000018477047000000200348D0F8BC3F13B1B6
:1032100000F57B6018477047000000200348D0F895
:10322000DC3F13B100F57D601847704700000020B7
:103230000348D0F8FC3F13B100F57F601847704792
:10324000000000200248C3690BB1103018477047D6
:10325000001000200248C36B0BB130301847704794
:10326000001000200248C36D0BB150301847704762
:10327000001000200248C36F0BB170301847704730
:10328000001000200348D0F89C300BB19030184754
:10329000704700BF001000200348D0F8BC300BB1CD
:1032A000B0301847704700BF001000200348D0F826
:1032B000DC300BB1D0301847704700BF0010002041
:1032C00002683649002310B422F00102212488420A
:1032D0000260036043608360C3600361446138D06F
:1032E0002F4B98422ED02F4B98423CD02E4B9842D9
:1032F00040D02E4B984232D02D4B984241D02D4B8E
:10330000984246D02C4B984217D02C4B98423CD038
:103310002B4B984216D02B4B984224D02A4B9842E4
:1033200028D02A4B98421AD0294B984229D0294BB1
:1033300098422ED0284B984208D14FF03D5243F886
:10334000AC2C03E04FF4746243F8202C5DF8044B7E
:103350007047224B5DF8044B3D229A607047204A2B
:1033600043F8642CF2E74FF474125DF8044B43F811
:10337000382C70474FF074625DF8044B43F8502CC2
:103380007047184A43F87C2CE0E73D2243F8082CAC
:10339000DCE7154A43F8942CD8E700BF10600240E0
:1033A0002860024040600240586002407060024065
:1033B00088600240A0600240B86002401064024091
:1033C0002864024040640240586402407064024035
:1033D00088640240A0640240B86402400060024079
:1033E0003D000020400F002000003D2000222DE97C
:1033F000F04713460D684FF0010E032604E0013339
:10340000102B02F1020239D00EFA03FC3CEA05044B
:10341000F5D1076806FA02F427EA040707600F7976
:10342000D0F800A007FA02F9013F49EA0A09012F82
:10343000A046C0F800906FEA040411D887683C40A9
:1034400084604C79876894403C438460446824EAF3
:103450000C0444608C7947689C40A4B23C434460AF
:10346000C46824EA0804C460CC79C7689440013376
:103470003C43102BC46002F10202C5D1BDE8F087C5
:103480002DE9F0412348244F244E254C82B03822A8
:10349000002173F01CFA002557F82510324600234E
:1034A00001E054F8332091422ED001330E2BF8D195
:1034B000002005356AF066FB4B2DEDD1DFF8588012
:1034C000184F08F596754FF0007698F8040003F051
:1034D000C3FD08F11408044688B1036803F13F43B3
:1034E00003F57E0307EB932393F8CC006AF04AFBC5
:1034F000A3880196206800936946FFF777FFA845E7
:10350000E3D102B0BDE8F081064A02EBC30393F8B1
:103510006000CEE7CC350020F01000200000014014
:10352000646A0708086A0708224A936803F00C03D4
:10353000042B10B421D0082B22D01F4B03601D4C4C
:103540001E4AA168C1F30311114491F82411CB4024
:103550004360A168C1F38221114491F8241123FA38
:1035600001F18160A1685DF8044BC1F342310A4466
:1035700092F82421D340C3607047114B0360DEE70B
:103580005368516813F4800F01F03F01536814BF72
:103590000B4A094AB2FBF1F1064A5268C2F30142F2
:1035A000C3F38813013201FB03F35200B3FBF2F3C0
:1035B0000360C4E7003802400024F400F810002043
:1035C00000127A0070B5446B8668A38923F4005317
:1035D0001B041B0CA38182790546407912F0040F6D
:1035E00014BF4FF4805C4FF0000C110310F0010F7A
:1035F0004FEA02220CBF0023042302F480628007FA
:1036000048BF43F0080342EA0C021343228A92B2F5
:1036100001F4005122F440520A432282A28922F48A
:10362000B05222F00C021204120C1A43A281A38A97
:1036300023F440731B041B0C84B0A3826846FFF77D
:1036400073FF244B9C4205D003F580639C4201D05C
:10365000029A00E0039AA3891F491B0402EB82022D
:103660004CBF7300B30002EB8202B2FBF3F3A1FB89
:103670000302A08952096426000406FB12334FEAB4
:1036800002121FD41B013233A1FB0313C3F34313F4
:1036900013439BB22381AB796A6B13F0080F938AB3
:1036A0000AD09BB243F00803938293899BB243F400
:1036B0000053938104B070BD23F008031B041B0C5E
:1036C0009382F2E7DB003233A1FB0313C3F342130F
:1036D0001343DEE7001001401F85EB512DE9F8434D
:1036E000394C9DF820509DF82490A0420F469046FA
:1036F0001E4649D0354B98424ED0354B984253D058
:10370000344B98422BD0344B984255D0334B98428F
:1037100021D14B462A4631460520FDF70FFB0446D2
:103720000023C4E90B78C4E90733C4E909336571A0
:10373000A66084F806902046FFF744FFEA07616B15
:103740001AD4AB0713D48B899BB243F400538B81FB
:103750002046BDE8F88300242046BDE8F8834B46A8
:103760002A4631460320FDF7E9FA0446D8E7CB683C
:1037700043F08003CB60E6E74FF6DF730B80CB6846
:1037800043F02003CB60DCE74B462A46314600205D
:10379000FDF7D4FA0446C3E74B462A4631460120DA
:1037A000FDF7CCFA0446BBE74B462A4631460220D9
:1037B000FDF7C4FA0446B3E74B462A4631460420D7
:1037C000FDF7BCFA0446ABE700100140004400409E
:1037D00000480040004C00400050004000140140F0
:1037E0008160EFE64171EDE62DE9F043DFF81482E8
:1037F00008EBC00985B00546C70099F8380103F009
:103800002BFC044699F8390103F026FC064699F88A
:103810003A016AF0B7F96B1CDBB2002C00F0AD8006
:1038200040F60B122372E280002E00F0C380337248
:1038300040F60B232046F38004223A2108F02AFCAC
:10384000042230463A2108F025FC08EB0703624ABF
:10385000D3F83441944200F09880604B9C4200F0D1
:103860009E805F4B9C4200F0AB80474497F83B2121
:10387000022A5CD0032A7ED05A4B5B4E012A18BF25
:103880001E46A7886846FFF74FFE27F03F07029BBA
:10389000564AB3FBF6F63F04A2FB03233F0C47EA6C
:1038A0009347A780228822F001021204120C228082
:1038B000B2B2C6F30B069B0C002E59D04FF4967192
:1038C00001FB03F34A49A1FB03139B0901339BB29C
:1038D00042F400422384A2832388464A9BB243F0E9
:1038E00001032380238823F4816323F002031B0454
:1038F0001B0C4FF4804143F4806323802181238893
:1039000023F080031B041B0C238023889BB202EB53
:10391000451243F0010323800121002382F8B054B3
:1039200082F8B11482F8B23405B0BDE8F083A688FD
:103930006846FFF7F9FD26F03F06029A2B4B360446
:10394000A3FB0213360C46EA9346A680218821F099
:1039500001010904090C21809B0C274901339209BC
:103960002384A1FB02329209042A38BF0422B2E761
:1039700042F00102A2E7214E83E7002E3FF465AF3B
:10398000337240F60B23F3805AE71D4B1A6A42F458
:1039900000121A621A6A22F400121A6265E703F52D
:1039A000F0331A6A42F480021A621A6A22F4800220
:1039B0001A625AE7042220463A2108F06BFB44E7DA
:1039C00003F5EE331A6A42F400021A621A6A22F40C
:1039D00000021A6249E700BF00540040005800404E
:1039E000005C0040804F1200009F240083DE1B43D8
:1039F000D34D621058310020632D3E05C0270900C9
:103A000000380240F81000202DE9F047954D90F95C
:103A100000108046807805EBC1060138CC0090B0DC
:103A2000D6F8341114282ED8DFE810F053012601FF
:103A3000150057006100A200AA00CB01BD017D0066
:103A4000870045020D02E001C500D50030003800B6
:103A5000AA019C015B01888A0C8B81B2824841EAF1
:103A6000044130EA010100F02681D8E90210521A1F
:103A700042F2107163EB00038A4273F1000302D338
:103A8000152388F8023010B0BDE8F08798F81300CD
:103A90000882C8E90223122088F80200888A0C8B69
:103AA00080B240EA0440714C34EA000000F0B68075
:103AB00000200E900F9001200F910E900E9900297A
:103AC00000F01E820F9914310F910F990968490572
:103AD000CBD5142388F80230D5E798F8110000F010
:103AE000FE000882C8E90223052088F80200888ABF
:103AF0000C8B80B240EA04405D4C34EA000000F0D8
:103B0000A480002000900190012001910090009974
:103B1000002900F00182019914310191019909688D
:103B20004F05D6D4A1E798F8110040F001000882B3
:103B3000C8E902230B2088F80200888A0C8B80B227
:103B400040EA04404B4C34EA00006FD0002004905F
:103B500005900120059104900499002900F0D68178
:103B6000059914310591059909684D05B1D47CE793
:103B700098F813000882C8E90223072088F8020099
:103B8000888A0C8B80B240EA0440384C34EA00004A
:103B90005FD00020029003900120039102900299CF
:103BA000002900F0C5810399143103910399096834
:103BB0004E058ED459E7088820F480600004000C7C
:103BC000088098F8110000F0FE000882C8E902237E
:103BD000102088F80200888A0C8B80B240EA0440EA
:103BE000234C34EA000012D000200C900D900120EC
:103BF0000D910C900C99002900F094810D991431CD
:103C00000D910D99096848053FF563AF2DE798F8C8
:103C10001330FF2B06D198F810301BB1132388F80E
:103C2000023030E7112388F802302CE7D8F814006E
:103C3000012800F09381022800F049820E20098BB0
:103C400088F80200C8E902231DE7062388F802303D
:103C500019E7D8F81400002800F07081082388F8CC
:103C6000023010E7F8100020010003008400070074
:103C70008200070002000300088820F400600004AE
:103C8000000C0880088880B240F4806008800888B2
:103C900080B240F480700880032088F80200888A8F
:103CA0000C8B81B2AB4841EA0441C8E9022330EAF7
:103CB00001037FF4E8AE98F81230002B40F0D38176
:103CC00098F81330FF2B00F04682042388F8023066
:103CD000D9E6098889053FF5C8AE002388F8023087
:103CE000D1E62C4494F8380103F0B6F9064694F86E
:103CF000390103F0B1F9984AB2F8103501339BB29B
:103D00008246A2F8103516B13368B2881A83BAF128
:103D1000000F04D0DAF80030BAF804201A83112119
:103D2000304603F06BFB1121504603F067FB4FF068
:103D3000090965272EB13368B28819690A4240F033
:103D40002881013F00F022810CF04EFD04460D4613
:103D50000CF04AFD001B61EB0501052871F1000321
:103D6000F6D3E7E7088880B240F4007008804FF689
:103D7000FF3088820121C8E9022388F8021082E618
:103D8000D8F81400002800F07281D8F8184014F810
:103D9000016B0E8201381225C8E90504C8E9022327
:103DA00088F802506FE6888A0C8B81B2694841EA34
:103DB000044130EA01017FF458AE0A2388F802304A
:103DC00061E6088880B240F480700880092088F895
:103DD0000200888A0C8B81B25E4841EA0441C8E93E
:103DE000022330EA01037FF44EAEE6E7002401250A
:103DF0000A940B940B910A950A98002800F04A81C6
:103E00000B9814300B900B98006846077FF52DAE89
:103E1000D8F81400032800F07281022800F24681CD
:103E2000088820F480600004000C0880088880B2B4
:103E300040F400700880098A88F81C40C8E9022311
:103E400088F802501FE6002001240890099009918B
:103E500008940898002800F01781099814300990F8
:103E60000998006847077FF500AEEFF31185102031
:103E700080F31288088880B240F400700880D8F877
:103E800018000E8A471CC8F81870EDB2067085F34A
:103E900011880D8AD8F818106FF001004E1CC8F870
:103EA00018600D70C8E90223C8F8140088F81C4097
:103EB00088F80240E7E5002006900790012007916E
:103EC0000690069C002C00F0EB80079C14340794AD
:103ED000079C246864067FF5C8AD0C8AD8F81810D2
:103EE0004D1CC8F818500C70D8F8141088F81C0035
:103EF0000139C8E90223C8F8141088F80200C2E5A5
:103F00000F9918310F910F990968AEE5059918318D
:103F1000059105990968A8E5019918310191019960
:103F20000968A2E50D9918310D910D9909689CE574
:103F30000399183103910399096896E5088880B2BE
:103F400040F4007008800121C8E9022388F80210BB
:103F500099E500BF0100030058310020088820F4D3
:103F600080600004000C0880EFF31184102080F3BF
:103F70001288088B088880B240F40070E4B2088090
:103F800084F311880C2188F802105BE616B13368BF
:103F9000B2885A830CF028FC04460D460CF024FC31
:103FA000031B61EB0501052B71F10003F6D316B17C
:103FB0003368B2881A830CF017FC04460D460CF0E7
:103FC00013FC031B61EB0501052B71F10003F6D314
:103FD000B9F101097FF4ADAE16B13368B2885A83E6
:103FE0000CF002FC04460D460CF0FEFB031B61EBDB
:103FF0000501052B71F10003F6D3BAF1000F04D0CF
:10400000DAF80030BAF804205A830CF0EDFB0446CD
:104010000D460CF0E9FB031B61EB0501052B71F16B
:104020000003F6D316B13368B2881A830CF0DCFBB8
:1040300004460D460CF0D8FB031B61EB0502052B73
:1040400072F10003F6D3BAF1000F04D0DAF80030B1
:10405000BAF804201A8398F90000441C3FF43DAEDE
:10406000FFF7C2FB39E60F2388F802300BE508881A
:1040700080B240F4007008800121C8E9022388F86A
:104080001C1088F80210FEE4099918310991099969
:104090000968EAE40B9918310B910B990968E4E47B
:1040A00007991831079107990968DEE4D8F81800D4
:1040B000098A441CC8F818400170D8F81410C8F8D0
:1040C00008200139C8F81410C8F80C30DBE408885F
:1040D00080B240F400600880EFF31184102080F378
:1040E0001288088B088820F480600004000CE4B279
:1040F000088084F311880D2188F80210A2E5088851
:1041000020F480600004000C0880EFF3118410207C
:1041100080F31288D8F818000D8A461CC8F8186079
:104120000570088880B240F40070E4B2088084F31F
:104130001188D8F81800098A441CC8F81840017082
:10414000D8F814100C200239C8E90223C8F814105A
:1041500088F8020097E498F81030002B3FF4B5ADD2
:104160002BE600BF38B5184D9DF814E005EB401460
:104170004FEA401C94F8B10400B938BD490084F8F6
:10418000C324C4F8C43484F8C1140023049984F807
:10419000C0E4022205F5966584F8C234C4F8C81458
:1041A00084F8CC3484F8B22465440CF01DFB02463C
:1041B0000B462846FFF728FC94F8B234002BF4D1C4
:1041C00094F8CC0438BD00BF5831002038B5184DE4
:1041D0009DF814E005EB40144FEA401C94F8B1043C
:1041E00000B938BD84F8C324C4F8C43401220023C4
:1041F000490005F5966584F8C22484F8CC34049A05
:1042000084F8C0E4022384F8C114C4F8C82484F8F4
:10421000B23465440CF0E8FA02460B462846FFF734
:10422000F3FB94F8B234002BF4D194F8CC0438BDED
:1042300058310020F0B587B00023834A00930193E2
:10424000136843F48033136003E0009BB3F5A04F81
:1042500009D0136803F400330193009B01330093EA
:10426000019B002BF1D0784B1B6813F4003318BF6F
:1042700001230193019B012B01D000BFFDE7724B8D
:1042800072491A6C724842F080521A640A6842F409
:1042900040420A609A689A609A6842F400429A60C2
:1042A0009A6842F4A0529A6058601A6842F080728C
:1042B0001A601A689201FCD5664A40F205711160D5
:1042C000996821F003019960996841F00201A2F513
:1042D00080629960936803F00C03082BFAD193680D
:1042E00003F00C03042B00F08D80082B00F08F806E
:1042F000594D5A4BC5F8EC3E534B59499868D5F87F
:10430000EC2E584CC0F303100144574891F84C115F
:10431000CA405649C5F8EC2EE160554A596FA26073
:10432000596B544A21F080015963596F41F08071F3
:104330005967196B0A431A635A6B5A639A6B9A63EB
:104340001A6C4D490A431A64596C4C4A0A435A6420
:1043500002A948F2FF73002602934FF6FF770396F7
:10436000FFF744F800F580600297FFF73FF800F58B
:1043700080600297FFF73AF800F58060FFF736F8A3
:1043800000F58060FFF732F800F58060FFF72EF847
:1043900000F58060FFF72AF800F58060FFF726F847
:1043A00000F58060FFF722F80846FFF7BDF8D4F863
:1043B000FC30029A3249334843F08073C4F8FC3031
:1043C000314BC3F8B01F5E60196841F001011960FC
:1043D000D5F8EC3E4FF47A71B3FBF1F3013BB3F146
:1043E000807F2A49B2FBF1F2C0F8882908D24FF049
:1043F000E022F0215361072384F8231096611361B2
:1044000007B0F0BD144D224BC5F8EC3E74E753687D
:104410005168114D13F4800F01F03F01536814BF30
:104420001B4A0E4AB2FBF1F1074A5268C2F301423D
:10443000C3F38813013201FB03F35200B3FBF2F321
:10444000C5F8EC3E58E700BF00380240007000405D
:1044500008544007003C0240000000200024F40003
:10446000F810002000ED00E0000002400003FA0513
:1044700000000008FF916700FFC9FE1033570700D6
:1044800055CEACC560200020001000E040420F0077
:1044900000127A0082B0064B002201920193019B28
:1044A00003EB80000190019B196002B0704700BFD0
:1044B0005028004010B51C2002F0CEFD112104460A
:1044C00002F09CFF4CB12368A2885A83C8200CF0EC
:1044D000B9F92368A2881A8310BDBDE81040C8202E
:1044E0000CF0B0B9704700BF704700BF704700BF05
:1044F00010B5124C94F81E3523B9114B4FF480229D
:104500005A6110BD4FF0E022D2F8103D23F00603AF
:10451000C2F8103DFEF700FA94F81E35002BECD0DF
:10452000D4F824359B68DB07E7D5D4F82026136838
:1045300023F0030161F307031360DEE75831002025
:10454000003C01402DE9F04FB34CD4F820355A69B6
:10455000D2078BB002D50BB0BDE8F08F5A699B69CA
:1045600012EA0309F7D0C9F3074319F4002F0093A7
:1045700040F0E180009B590743D419F0020F5FFA25
:1045800089F603D0D4F8203502225A61B9F1000F20
:10459000C0F2EE8119F4006FC9F3072540F04A819B
:1045A000330708D59D4B9E48D3F868319847D4F817
:1045B000203508225A61F70600F1C481EE0600F1A9
:1045C0006F81A90600F1E880009BDA0609D5934BBC
:1045D0009348D3F878319847D4F820354FF48012B7
:1045E0005A61009B9B06B6D58C4B8D48D3F87C3125
:1045F0009847D4F820354FF400125A610BB0BDE84B
:10460000F08FD4F824259369D26913401FFA83FAF6
:10461000BAF1000FB1D0DFF81882CDF80C90A8F1F4
:10462000180500271AF0010F78D0FEB2D4F824251F
:1046300004EB86031069D3F82C15536B8968F3409B
:10464000DB01DBB203430B4013F00109D9B240F0A8
:10465000AB810A0740F1C881D8F800200823936095
:10466000994619F0800F59D0D5E94CC0D5F82431BE
:10467000D8F800E0ACEB00018B42DEF8182028BF30
:104680000B4692B20333B2EB930F47D9D4F82425EB
:1046900094F81795323604EB8603CDE90178674626
:1046A00098469446874237D9D5F82431391A994229
:1046B00028BF194601F1030BD5F828314FEA9B0BAF
:1046C000B9F1000F10D18AB203329210D8F81C65EC
:1046D0000AD04846013053F8047B37608242F9D152
:1046E000D5E94C70D5F8283108440B44B842C5F8D8
:1046F0002831C5F83401DEF818300AD195F81C11BC
:10470000012202FA01F1DCF8342022EA0102CCF89D
:1047100034209BB29B45C5D3DDE901785FEA5A0A94
:1047200007F1010708F1040805F128057FF47AAFC5
:10473000DDF80C9021E7D4F824359D69DB691D4034
:104740002D0C3FF417AF04F21458DFF8D0B004F585
:10475000AD660027C24608E06D0807F1010706F1C3
:10476000040608F128083FF405AFEB07F4D5F9B2C9
:1047700004EB8103D4F82425D3F868359B6852698B
:104780001340D807DAB200F13F81930740F1678107
:10479000336802229A60DFE7D4F82435D4F82C1568
:1047A0009A680868C2F34102022A06BF032262F334
:1047B0000A006FF30A0008605A6842F480725A6077
:1047C00006A8FEF7B1FED4F82025D4F82415D36846
:1047D000079D6FF38D23D36088681249C0F34100B1
:1047E000014491F8D410032900F05F810E490F486D
:1047F0000126294484F8166581424FF04006A4F84A
:10480000186500F2AC810E2161F38D234FF4005145
:10481000D3605161D8E600BF58310020F810002065
:104820006C360020086A0708401E1BFF3F420F003D
:104830008436002000238DF8133094F826368DF846
:104840001330B64BB648D3F870319847D4F82435B6
:10485000D4F82025986894F81E354FF40061516112
:10486000002B3FF49DAEC2077FF59AAE94F829362F
:10487000012B7FF495AE9DF81330032B7FF490AE9F
:10488000D4F82036A7491A6842F001021A601A6863
:1048900042F003021A600B6943F006030B617FE6E6
:1048A000D4F82465D4F820157368002723F0010399
:1048B00073600597059B43F020030593059B67F301
:1048C0008A130593059B0B610B690593BC46964BB8
:1048D00003E00A690592013B02D0059A9006F8D4DC
:1048E00094F8152552B1914B03EB820EFF2253F839
:1048F000040F8260D86B73458260F8D10B2363F399
:10490000070763F3070C4FF0FF33B3614FF0011358
:10491000F3617761C6F810C0336885486FF30A13F6
:10492000336094F81725D4F86835012A186100F02F
:10493000B5804FF480534B61784B7948D3F86C3194
:1049400098473EE6D4F820359A6922F010029A6121
:104950001A6AC2F34340022802F00F0100F0B0804F
:10496000062800F087809A6942F010029A6125E6D5
:1049700094F81E353BB1D4F82026136823F00301C8
:1049800061F307031360D4F82425644B6448D3F81B
:104990007411536823F0010353608847D4F820351D
:1049A0004FF000425A61F5E5516BD8F800005B4BBF
:1049B0004FF0010C0CFA07FC21EA0C0151630122B3
:1049C000D3F86031826031465548984794F81735DE
:1049D000012B00F0B18019F0020F3FF442AED8F87D
:1049E000003002229A6099E6CB0604D5D8F8003050
:1049F00010229A6092E6480658BF8946EBD5D8F84F
:104A0000003040229A6089E694F817253368012027
:104A10008242986007D11A69D8F87C33C2F3120237
:104A20009B1AC8F88C33DBF85C315046984794F8F1
:104A30001735012B7FF490AE002F7FF48DAE94F8E4
:104A40002536052B7FF488AED4F86835384A1A61CC
:104A5000384A5A611A684FF080221A607CE61007C3
:104A60007FF57AAEDBF86431504698473368082208
:104A70009A6071E601EB810104EBC101D4F8E465B1
:104A8000D1F8A008C2F30A1202443068C4F8E00A60
:104A90003068C4F8E40AC1F8A02864E7254A5A61DE
:104AA0001A684FF080221A6043E7002184F8161537
:104AB0004FF40071A4F81815092161F38D23A5E6C0
:104AC00047F6F07010423FF44EAFC2F30A1201EB0A
:104AD000810004EBC00002F1030C5FEAAC0CD0F8DB
:104AE0009468D4F8E4E54FEA810818BF002006D0A6
:104AF0000130DEF8007046F8047B8445F8D141446B
:104B000004EBC101D1F894081044C1F89408D1F81D
:104B1000A0080244C1F8A02825E700BFF810002033
:104B20006C36002000ED00E0400D030080360020D0
:104B300018000860383C0020002F7FF44CAF94F838
:104B40002536042B7FF447AFD4F868352B4A1A6119
:104B50002B4A5A611A684FF080221A603BE72948B5
:104B6000A5F57401A1F51051814203D80D2161F31F
:104B70008D234BE6244925482944814203D20C2148
:104B800061F38D2342E62248A5F18C71A1F54341E2
:104B9000814203D80B2161F38D2337E61D491E485E
:104BA0002944814203D20A2161F38D232EE61B4959
:104BB0001B482944814203D2092161F38D2325E654
:104BC0001848A5F1B771A1F55851814203D20821C7
:104BD00061F38D231AE6144914482944814203D213
:104BE000072161F38D2311E61149124829448142BE
:104BF00034BF0621052161F38D2307E61800086004
:104C0000383C0020DFC810002013FBFE20D6130024
:104C1000FF69180000D3CEFE40771B00C05BB3FED7
:104C2000C091210040AC2700C01D6AFE40E1330066
:104C3000803C36FEE09C41000378022B12D00E49E6
:104C400043680269D1F8180210B41840D1F8104234
:104C5000D1F80C12931E400A04FB030008445DF8CF
:104C6000044B7047044B4268D3E9800100EB4100DC
:104C700000EB5220704700BFA05C00202DE9F84FE8
:104C800012F0020E01D000283CD08A4DD5F80872EF
:104C9000002F43D14FF0FF3C874CE146E046E2460F
:104CA00000262768B84200F0D98094F80EB0BBF116
:104CB000000F4ED0BBF1010F16D1804F06F5817B5E
:104CC00007EB0B1B9BF807B01BF0010F0CD11BF07F
:104CD0007E0F09D15FEADB1740F0B480D4F808B04A
:104CE000D34501D2DA46B1460136082E04F110044C
:104CF000D7D1BCF1FF3F38D1B8F1FF3F30D06F4C76
:104D0000C44633E06B4D95F8B431A5F58054E3B15A
:104D10000123637002263046BDE8F88FD5E983464B
:104D200006FB0744A042B5D395F8B43113B901236B
:104D300085F8B431614B012200265A703046BDE837
:104D4000F88F95F8B431002BE2D1012385F8B43106
:104D5000DEE7B4460136082E04F11004A1D1C8E7FD
:104D6000B9F1FF3F18BFCC4674D0544CD5F89860C9
:104D700004EB0C1841F21809013648F8090041F219
:104D80001C090CF5817748F809604FEA0718C5F847
:104D9000986044F8086004EB07164FF00008C6F866
:104DA000048004EB0716B679042ECAD8DFE806F0B3
:104DB000031952192F0012F0010868D104EB0710F3
:104DC000D61090F80790032B66F3C71980F8079068
:104DD0005BD94FF6FF70834228BF034604EB0710F0
:104DE0008380BEF1000F12D0D5F89830D5F89C0022
:104DF00001330130C5F89830C5F89C0004EB0C1065
:104E000041F21C05435104EB07130420987150072D
:104E100005D504EB0710C37943F00103C371D30632
:104E200008D504EB0714E379C3F34502013262F3BA
:104E30004603E371224B012603EB4C230B60304603
:104E4000BDE8F88FB0460136082E04F110047FF457
:104E500028AF4EE700263046BDE8F88F174C06F520
:104E6000817704EB071C4FEA07189CF806C0BCF1D9
:104E7000000F01D1B44679E7B446D5F89860013601
:104E800044F80860C5F898608BE74346A6E70D4BE9
:104E9000D3F8DC3C002BDDD009495D680A4A01EB00
:104EA0004C210023A8470028D4D004EB0714022388
:104EB000A37130E7A05C0020B85C0020A04C00206B
:104EC000B84C002060200020B107000870B5104EDB
:104ED0003378022B0F4B0BBF020AC0F3D412C4B2BB
:104EE00000F07F04D3F8000282B010440D46002386
:104EF000032201A9FFF7C2FE012807D13378022B54
:104F0000019B0CBF23F8145043F8245002B070BD2D
:104F1000A04C0020A05C00202DE9F04FDFF82C8190
:104F200098F80060032E85B00C46154643D0012842
:104F30008CBF00220122022E0B68019269D14FEA38
:104F40001329DFB24FF4807A0138012820D84FF0BE
:104F5000010B9D4217D93C4ED6F878211AB1D6F8EC
:104F60009411994258D0D6F80002002348440922EF
:104F700003A9FFF783FE01282CD0022817D020B107
:104F800023689D42E8D82560032005B0BDE8F08F76
:104F9000F7B12D4B93F8B42112B9012283F8B42153
:104FA0000123022088F8013005B0BDE8F08F02200F
:104FB00005B0BDE8F08F01288CBF002301230193C9
:104FC0000B684FF0800AC3F3D41903F07F07BBE7E7
:104FD000D346BEE798F800200399DDF804C0022A02
:104FE00014D0032AE3D151F8273023F07043B3FAE9
:104FF00083F35B0963455F44236821D05B445745D5
:105000002360ECD309F101090027BAE731F8173022
:10501000EDE74FF4807AD6E7D6F81012013A02EBAA
:1050200041224902B2FBF1F21344B3FBFBF20BFB4A
:1050300012320AB15B449B1A9D4223608CD8A2E7CE
:10504000AB42A2D39FE700BFA05C0020A04C002091
:105050002DE9F04FDFF86CB19BF800C0BCF1020FF6
:10506000894683B009688246174640F08C800BF56C
:105070008053CEB2D3F80052A6EB010805EB112500
:1050800090444FF480739844B94208F1FF38B8FB5C
:10509000F3F84CD2A844BCF1030F07EB06040CBF95
:1050A00080224FF48072641A9442A8EB050328BF53
:1050B000144666B994422CBF0A220B2201A9284645
:1050C000FFF7DCFD012809D003B0BDE8F08F0B220B
:1050D00001A92846FFF7D2FD0128F5D19BF800C0B1
:1050E000D9F80010BCF1020F01F1010323D0B44242
:1050F00010D9019906F18042013A01EB820204398C
:1051000001EB840142F8043F914203F10103F9D11C
:10511000D9F80010A61B3144BAF1010FC9F80010EC
:1051200021D08F4205F101054FF00006B3D80120D0
:1051300003B0BDE8F08FB442ECD9019806F100420B
:10514000013A00EB4202023800EB440022F8023F31
:10515000904203F10103F9D1A61B3144BAF1010FCA
:10516000C9F80010DDD1B942DBD1BCF1020F1DD06E
:1051700004F18044019B013C4FF0FF3243F82420AE
:10518000D9F80010CDE70BF5805301F07F06D3F876
:105190000032BCF1030FC1F3D415A6EB01081D4486
:1051A000904414BF4FF4807380236CE704F10044F3
:1051B000019B013C4FF6FF72504623F8142003B0C8
:1051C000BDE8F08FA04C002030B50446C06983B024
:1051D00010B9012003B030BD0D460023032201A900
:1051E000FFF74CFD0128F5D1B4F92030002B0ADA85
:1051F000144B93F8B4210AB983F8B401124B01227D
:105200005A700220E6E7019A012D4FEA431102EBA2
:10521000431303D0022D11D1E5255554A268DA615C
:105220002278032A04D100221A775A779A77DA77FC
:10523000626A5A83120C9A8203B030BDE268DA6166
:10524000EEE700BFA05C0020A04C00202DE9F0415B
:1052500090F83C30002982B0044614BF022100219E
:10526000042B7BD8DFE803F0030C3D486900FFF70F
:10527000ABFF012870D1626B002A75D184F83C0025
:10528000404EDFF808814FF6F77706F5805516E0B7
:10529000BA424FD867F076FE01284FF000011DD1C9
:1052A000206BFFF713FE012818D1019AD5F81412CC
:1052B0002263531E8B4228BF0B46C5F81432327846
:1052C000236B032A01A918469AB2E1D1434531D88C
:1052D00067F058FE01284FF00001E1D002B0BDE8B0
:1052E000F081426B04F130010020FFF7B1FE01288C
:1052F00032D1032384F83C302348E16AD0F894315A
:10530000D0F81022C0F894115B1A02FB03F3D0F816
:10531000782102EB4322C0F87821D0F87C2102EBFF
:105320004323C0F87C31002100F5B870FFF74CFF33
:10533000012811D1042384F83C3094F82830042B40
:1053400004BF002384F82830A36B8BB12046984714
:10535000012002B0BDE8F0810228BFD194F82830C6
:10536000042B09D00220B9E7022384F83C30B9E7C6
:10537000012002B0BDE8F081002384F8283002202B
:10538000ACE700BFA04C0020A05C0020F7FFFF0F9F
:1053900038B590F834300446052B43D8DFE803F0E5
:1053A0001E033C0F185E006B4FF0FF31FFF78EFDC0
:1053B000012837D1E06AB8BB032384F834300021D8
:1053C0002046FFF701FF01282CD1042384F8343054
:1053D00094F82830082B2BD0012038BD204DD5F86B
:1053E000082200F1300102320120FFF795FD01286B
:1053F00023D00238C0B2012814D8052384F83430F1
:1054000094F82830082B04BF002384F828300123A7
:1054100085F8B531022038BDC06A216BFFF756FD13
:105420000128C9D0002038BD022384F83430F4E7C5
:10543000002384F82830012038BDE368D5F8101225
:10544000D4E90B2003EB4123C5F81402C4E903306F
:1054500002B96062012384F83430A5E7004DCFE73C
:10546000A05C002010B590F838300446032B4DD8CE
:10547000DFE803F0022F38432B4AC068117802F5A9
:1054800080530329D3F81012D3F894210CBF4FF0A6
:10549000800C4FF4807C01FB0CF100EB4120C4E94F
:1054A0000302D3F87801A0EB4120C3F87801D3F8C8
:1054B0007C01A0EB4121E06AC3F87C1102EB0C01F6
:1054C000C3F89411C4E90C2148BB6262012384F83B
:1054D000383016480021FFF777FE012811D102234A
:1054E00084F83830626B04F130010120FFF7B0FD21
:1054F000012806D1032384F8383000212046FFF725
:1055000063FE431EDBB2012B01D910BD022094F8CB
:105510002830062B04BF002384F8283010BDA2EBEE
:105520000C022263D2E700BFA04C0020105E0020D6
:105530002DE9F0434368C3F308020A44B2F5007F43
:1055400083B004460D4605D22B446360012003B0AE
:10555000BDE8F08390F91A20501C0AD0444902F5A6
:10556000817201EB0212D1796FF30001D171FF2238
:10557000A27694F91B20511C16D03D4802F581718A
:1055800000EB011200EB0111D279C879C2F3450298
:10559000012A86BF02F1FF3202F03F020022FF26FD
:1055A00062F34600C871E67694F800C0BCF1020FC1
:1055B000CAD0DFF8C480D8F81022B5EB422F4FEAEA
:1055C000422915DCD8F818721F407A42AA420FDC33
:1055D000EA194A4510D220690028B7D0244A127827
:1055E000032A40D080B24FF6F7729042ACD9ADE7B3
:1055F000002003B0BDE8F083227E206912F0080687
:1056000026D0D8F89421411C8A4213D300D100211E
:105610004B44A5EB0905DB1BBCF1020F60613D4467
:10562000216163600846D7D1D8F82022B3EB422F1E
:105630008AD38BE798F8B42122B9012388F8B431D2
:10564000636820690A4A0126567094F800C0DFE7B3
:1056500001A967F097FC0128CAD10199636894F801
:1056600000C02069D4E7034A90427FF66DAF6DE732
:10567000A04C0020F7FFFF0FA05C00202DE9F047B1
:1056800090F8384082B00546032C00F2AD80DFE888
:1056900004F00219730BFFF77BFE012810D00228DB
:1056A0000AD1032385F838302B6C002085F82800B8
:1056B000002B71D098470224204602B0BDE8F08745
:1056C00085F838002B78022B62D0484A6B68D2F8F4
:1056D000182203EA0208C8F34F282846FFF7ACFA5D
:1056E000424F0646A8EB0008A7F5805901A90222FF
:1056F00000233046FFF7C2FA08EB060401281FFA20
:1057000084FA4FF400724FF000010446D4D101989E
:1057100071F0DDF8EB694FF40071284613B16B6846
:10572000002B3DD0D7F810325A1E924506F10106E3
:105730000DD2FFF7FDFE0028D8D197F8B43113B988
:10574000012387F8B431012389F80130CEE7C3EB98
:10575000C353590201F500712846FFF7E9FE40B92D
:1057600097F8B43113B9012387F8B431204B0122E3
:105770005A70022385F838302B6C002285F82820D7
:1057800063B1284698470124204602B0BDE8F0875F
:105790006B68C3F34F28A0E702248DE701248BE751
:1057A000019B4FF020324FF02E0E4FF0100C1A607C
:1057B0005A6083F800E0C3F807206C6A1A625A62E4
:1057C00083F80BC0C3F8272083F820E083F821E09A
:1057D000EA6B5C835A8724FA0CF422FA0CF29C825E
:1057E00083F82BC09A869DE7002465E7A05C002023
:1057F000A04C00202DE9F041B1F904300F2B82B00C
:105800000E460446174635D02046FFF715FA94F9A0
:105810001B80B8F1FF3F3ED0554B41F2180203EB1D
:1058200008118A58904211D1183303EB4825B388E8
:1058300001331BB205EB4315B38020463D60FFF7F3
:10584000FBF93060012002B0BDE8F08103F5805221
:1058500092F8B41100296AD001225A702278022AE3
:1058600069D02369002B50D1002301203B6002B096
:10587000BDE8F0814FF40071FFF75AFE002852D0C6
:105880004FF6FF73B3802046FFF7D6F994F91B80DB
:10589000B8F1FF3FC0D12278022A54D02369002BEF
:1058A000DDD03349097803290EBF32499BB24FF648
:1058B000F7718B4294BF00230123002BCFD138B95D
:1058C0002D4A92F8B431002B4ED0294B01225A7048
:1058D0000023112201A9FFF7D1F9012842D1019D2E
:1058E000264BEB1A48BF03F2FF13B3F5805F4FEA74
:1058F000632230D3204A92F8B43113B9012382F8DD
:10590000B4311B4B01225A7027E0194A1278032A3E
:105910000EBF184A9BB24FF6F772934294BF002312
:105920000123002BA0D1002002B0BDE8F0810121AD
:1059300082F8B41190E7104A6368D2F82022B3EBE2
:10594000422F91D2EFE70C4A6368D2F82012B3EBF2
:10595000412FB4D3F1E74FFA82F884F81B80002D71
:105960007FF465AF22787AE7012382F8B431ACE79F
:10597000A04C0020F7FFFF0FA05C0020B84C0020D7
:105980002DE9F04790F8303086B00446042B54D807
:10599000DFE813F005000E005600E6004F00C24895
:1059A00068F06CFA4FF6FF720123228484F83030DD
:1059B000DFF8F48204F11C0501AE04F1310932462E
:1059C00029464046FFF716FF012800F0F080022824
:1059D00033D1B64901F5805595F9D221531C0AD02F
:1059E00002F5817201EB0212D3796FF30003D371D8
:1059F000FF2385F8D23195F9D3315F1C16D003F51A
:105A0000817301EB031201EB0313D279D979C2F34D
:105A10004502012A86BF02F1FF3202F03F02002256
:105A200062F34601FF22D97185F8D321042384F85B
:105A300030300020E36A2070984706B0BDE8F08758
:105A40009B4D95F8E031002BF7D1974F04F11C09DD
:105A500001AE4FF00908324649463846FFF7CAFE04
:105A6000012840F00F810198002800F0EB800378B6
:105A7000E52B01D0002BEED18E4A821A48BF02F2EC
:105A8000FF12B2F5805F4FEA622380F06781874999
:105A90001B01894A13449A7B042A0CD0D5F898201C
:105AA0000132C5F898205A6004229A73D5F89C30C8
:105AB0000133C5F89C3095F9D2315E1C0AD003F54C
:105AC000817301EB0313FF2285F8D221DA796FF39A
:105AD0000002DA7195F9D3315A1C18D003F581739D
:105AE00001EB031201EB0313D279C2F34502012A41
:105AF0004FF0FF0188BF02F1FF3285F8D311D97949
:105B00008CBF02F03F02002262F34601D9712022CD
:105B1000002170F0DCFE019BD4F83120D4F8351060
:105B200059601A60B4F8392094F83B1099721A81C0
:105B3000019B627EDA7203A803F068FB002840F044
:105B4000D480019B6FF07E01472219745A749873B8
:105B5000D87344F2817503221D83D88284F83020E3
:105B6000237E980608D5E0690023112202A9FFF7D9
:105B700085F801287FF461AF204668F07FF923693A
:105B8000002B00F08380237E03F0F70213F0040360
:105B9000227640F09380122A00F0CE800022E36A41
:105BA00084F828202046984706B0BDE8F087019F7A
:105BB000002F00F0DF803B78002B00F0DB8097F8AF
:105BC0000BA01AF0080F7FF4FAAE0B2249463846B4
:105BD00070F0CCFE00287FF4F2AE637E8AEA030305
:105BE000D90640F10881314901F5805595F9D23146
:105BF0005A1C0AD003F5817301EB0313FF2285F8C9
:105C0000D221DA7960F30002DA7195F9D321571CB9
:105C10003FF40CAF02F5817201EB021301EB0211AC
:105C2000DB79CA79C3F34503012B86BF03F1FF3348
:105C300003F03F03002363F34602FF23CA7185F894
:105C4000D331F3E695F8B831022B3FF4EFAE95F877
:105C5000E031002B7FF4EAAEC5E97D3385F8F03101
:105C600085F8EC31D5F8CC31C5F8E431D5F81432EB
:105C700085F8E081C5F8E8313846FFF7FFFC0128D8
:105C80003FF4E9AE02283FF4D1AED6E6237E1907F1
:105C900084D5074B93F89821002A7FF4CEAE0722D3
:105CA00083F898217AE700BF585E0020A04C0020BE
:105CB000A05C0020B84C0020B85C0020A568E66A13
:105CC000002384F8283029462046FFF731FC0028BD
:105CD00040F08B8094F82830002B7FF4AEAE022386
:105CE000C4E90B6584F82830A7E6654B03A9B3F82F
:105CF000083BADF80830084602AA67F08DF89DF819
:105D00000E509DF80F10BDF80C00019B9DF810205F
:105D100041EA4511A0F2BC7041EA40218DB21982DE
:105D20009DF81110D20242EA41129DF8121042EA87
:105D3000510290B2DA810EE7626AE16AA16304203F
:105D400084F82800C4E90B22C4E9023384F83C300B
:105D500063636362204668F091F86EE695F8B431AB
:105D600013B9012385F8B431464901234B706FF014
:105D70000F038EE6434901F5805595F9D2315F1C3A
:105D80000AD003F5817301EB0313DA796FF3000294
:105D9000DA71FF2385F8D23195F9D3315E1C16D024
:105DA00003F5817301EB031201EB0313D279D97967
:105DB000C2F34502012A86BF02F1FF3202F03F0220
:105DC000002262F34601FF22D97185F8D321237E98
:105DD000D8067FF52BAE2C4868F050F84FF6FF72CE
:105DE0000223228484F830302BE6002E3FF425AEC7
:105DF0002046B04721E6BA8A7B8B244D43EA024312
:105E00006362D5F81022FB69A3605202B3FBF2F182
:105E100002FB113109B113445B1AE36084F819A045
:105E200095F9D23117495E1C0AD003F5817301EB55
:105E30000313DA796FF30002DA71FF2385F8D231A8
:105E400095F9D321501C16D002F5817201EB021393
:105E500001EB0211DB79CA79C3F34503012B86BF3D
:105E600003F1FF3303F03F03002363F34602FF23F4
:105E7000CA7185F8D331032384F8303070E600BF4F
:105E800058310020A04C0020585E0020A05C00206B
:105E900010B5037890F818C0023B012B044602D9D4
:105EA0001CF0060F6AD11CF0200F44D194F91A306F
:105EB000591C0AD0384A03F5817302EB0313FF2102
:105EC000DA796FF30002DA71A17694F91B305A1C6B
:105ED00016D0314903F5817301EB031201EB031373
:105EE000D279D979C2F34502012A86BF02F1FF3285
:105EF00002F03F02002262F34601FF22D971E276EE
:105F00001CF0080F0ED0254B93F89821072A06D0D5
:105F100093F8B421002A3BD01F4A0121517000227E
:105F200083F89821E26A0023237084F8283022B392
:105F3000BDE81040104700231949E0691A018A584A
:105F4000904206D00133082BB0D01A018A589042F3
:105F5000F8D1114903F5817301EB0312D279C2F331
:105F60004502012A12D9013A02F03F0201EB031364
:105F7000D97962F34601D97198E710BD0121FFF785
:105F800023F90128F9D194F818C08CE70022EDE735
:105F9000012283F8B421BFE7A04C0020A05C0020C0
:105FA000B85C00204FF0FF302DE9F041344A354D08
:105FB0000446002304E00133082B02F1100216D03E
:105FC00011780429F7D103F5817105EB0111C97925
:105FD000CF07F0D4661C52F80A1C01D08142EAD2E5
:105FE0001C460133082B084602F11002E8D1631C5D
:105FF00002D10120BDE8F081224DDFF8988004F540
:10600000817705EB07139988F9B91F4ED8F8DC3C66
:1060100006EB442123B3D3F80C801C4A41F2180349
:1060200005EB0414E0580023C047C8B1022824D16E
:1060300006F6E87605EB0715D6F89C300122013B01
:10604000C6F89C30AA710020D4E7D8F8DC3C3BB1FC
:106050009A6841F2180005EB041318589047D4E7EA
:106060000B4BD3F89C2005EB07150320013A0121C7
:10607000C3F89C20A87183F8A0100020BDE8F0812F
:10608000C65C0020A04C0020B84C00202908000865
:10609000A05C0020602000202DE9F04F90F828300F
:1060A000013B83B00446082B0BD8DFE803F0383CF3
:1060B0001E2305290A2E33000121FFF7C7F8012806
:1060C00002D003B0BDE8F08F2378002284F82820A6
:1060D000002BF6D0D4E901138B4238BF0B46226C5B
:1060E000A360032184F82810E262204603B0BDE8D3
:1060F000F04FCDE6002103B0BDE8F04FFFF7A6B8A2
:1061000003B0BDE8F04FFFF7ADB903B0BDE8F04F05
:10611000FFF73EB903B0BDE8F04FFFF7AFBA03B0E9
:10612000BDE8F04F2CE4534F4368D7F81852016B89
:10613000D7F810221D406818B0EB422F4FEA4226D4
:106140009C46C0F0938094F800E0DFF82C91A7F50E
:10615000805A4FF6F778BEF1020F14D0206900285C
:1061600057D1D4F804C0A368E26A634538BF6346D8
:106170000021A36084F82810002AA2D0204603B092
:10618000BDE8F04F1047D4F804C0D7F82022BCEB8C
:10619000422FE8D22069227E12072CD5D7F894210D
:1061A00000F1010C624522D297F8B42122B90123F3
:1061B00087F8B4316368216B01228AF8012094F8D2
:1061C00000E0891B294433445B1B8E42C4E904C0B0
:1061D000636021639C464FF00005BCD9BEF1020FFD
:1061E0003ED020690028BED0DFF890B01FE0E8D193
:1061F0004FF0000CE5E701A966F0C4FE01287FF42A
:1062000060AF2069DDF804C094F800E06368216B9A
:10621000D7E79AF80020032AD3461AD082B2424523
:1062200094BF00220122002AB5D0D4F804C09BF804
:106230000030032B0EBF104B80B24FF6F77398421D
:1062400094BF0020012000288DD18C44C4F804C0E4
:1062500089E7484594BF00220122002A9BD0E4E749
:10626000D7F82022B3EB422FEFD37CE794F800E07D
:10627000B4E700BFA05C0020F7FFFF0FA04C002098
:1062800010B5184C18484422002170F020FB2378E8
:1062900004F580544FF6FF70D4F81C22A4F8D20104
:1062A000022B4FF0030118BF03234FF0100C84F8AA
:1062B000D01104F5DC700021C4F8C82184F8B8318D
:1062C000C4F8DC2184F8D1C1FFF732F938B994F869
:1062D000E03123B9C4E97933022284F8E0210120B6
:1062E00010BD00BFA04C0020585E002070B51A4DB4
:1062F0001A4BC5F80C3B1A4B85F8181B002683F87F
:106300008C6905F60C33C0E954330D230446C0F8FC
:10631000583140F20113C0F85C6100F5A271A0F899
:10632000443169F0F5FCE378C4F8B4631F22C4F883
:10633000B023012205F587659342C4F8A853A4F859
:106340009C2308BFC4F8AC5304F567712046BDE830
:10635000704069F0DDBC00BF5831002055534253F6
:1063600060200020F0B50B7813F0600683B00C4677
:10637000054633D0202E2DD14A78FE2A6BD0FF2A35
:1063800063D14A88002A40F08B80CA88002A40F0F6
:106390008780190600F184806148624B80F88C295F
:1063A000C5F8B423EA78012183F85814A5F89C13A2
:1063B00003F587631F21012AC5F8B013C5F8A83378
:1063C00005F5677108BFC5F8AC33284669F0A0FC35
:1063D000002600E00026304603B0F0BD4B780A2BC3
:1063E0006AD00B2B63D0012BF5D18B88D9B21B0659
:1063F00076D40196019BC06843F010030193019B82
:10640000036103690193484B03E002690192013B78
:1064100002D0019AD206F8D42846424F69F068FBB0
:10642000022321794022284669F094FB97F85834DA
:10643000022B6DD094F90420002ACCDA012BCAD0AB
:1064400001212846FFF752FFC5E766F027FE022626
:10645000304603B0F0BD4E8816BBCC88012C1FD14E
:1064600018061DD52F4FD7F870349B699847C0B2D6
:1064700087F81C0BA0B1022307F61C3785F81131F1
:106480004FF48073C5E94E44C5E94A77C5E94C46E7
:10649000A5F81C3105F58E71284669F0CBFB9AE70B
:1064A000284666F0FBFD0226304603B0F0BD1D4BCA
:1064B0004A8883F81D2B8EE7022280F811214FF4C1
:1064C0008072A0F81C21194A0123C0E94E33C0E9AB
:1064D0004A22C0E94C3600F58E7169F0ABFB7AE7D1
:1064E0000096009BC06843F020030093009B61F37B
:1064F0008A130093009B0361036900930A4B03E036
:1065000002690092013B87D0009A9706F8D483E78E
:106510008121284669F0B2FA002387F858345AE7F7
:106520006020002058310020400D0300753C002001
:1065300010B50D4B93F88C39022B07D0033B012B80
:1065400002D80021FFF7D2FE002010BD074B93F8C0
:106550004514044666F04CF90028F5DA012120467E
:10656000FFF7C4FEF0E700BF602000205831002094
:10657000F8B5404E96F88C59074655B1012D06D115
:106580003D4B93F8451466F033F9002832DB0020C8
:10659000F8BD394CB0F8B433D4F83C24C4F8102B0F
:1065A0001F2BD4F84024C4F8142B08D1334BD4F853
:1065B00038249A4203D194F8451401291FD994F83C
:1065C0001E3B04EBC3020133DBB2042B4FF0050189
:1065D00008BF002382F8201B4FF4005184F81E3BB3
:1065E00038460223C2F8241B84F85834FAF7E0FD39
:1065F0000020F8BD29463846FFF778FEC7E794F833
:106600004634013B0F2BDAD866F0F2F8002827DB7E
:1066100096F88C39013B022BB9D9B4F8403B1BB337
:10662000042286F88C29164AC7F85C51C7E954221F
:10663000D4F8402484F8185B934228BF1346D4F85A
:10664000142BC7F8583140F20111A7F84411D31A9E
:1066500007F5A2713846C4F8143B69F059FB96E778
:106660003846FAF7A5FD92E719463846FFF73EFE91
:106670008DE700BF60200020583100205553424371
:10668000A03C0020002070472DE9F04F604D85B000
:10669000EB892868B5F80C8001911B0229896E8965
:1066A0002C8AC01A67EB07074FEA014EA8FB001CB3
:1066B000EB8808FB07CCC90941EA4C6111EB0E01DC
:1066C00093464FEAC332A6FB003E06FB07EE4FEAB5
:1066D000132343EA0E634FEAEC1C4CF1000C9B18A9
:1066E000A4FB002604FB07644FEAD25242EA44228C
:1066F0004FEA2E2E4FEAE4544EF1000E12F5FA69DD
:1067000044F10006B9F5FA6F029476F1000403969D
:1067100031DA029CA2FB02A602FB04F806EB480455
:106720004FEA84084FEA8A0616EB0A0648EA9A7886
:1067300044EB08084FEA560A4AEAC87AB608354CCC
:10674000B1EB0A0146EA88766CEB680C9B1B039E52
:106750006EEBA80EA1454FF0FF3476EB040426DB68
:1067600000FB07F7A0FB000202EB4707C00F40EA5F
:106770004700B9EB0009019C84B16869A0FB0332B2
:1067800000FB0E2E5B0D43EACE235B1A4FEA6E5ED2
:106790006EEB0C0CDB0B43EA4C432360BBF1000FA8
:1067A00001D0CBF80090012005B0BDE8F08F40F695
:1067B000AC56029C921944F1000402FB04F4A2FBC3
:1067C000028202EB4404E6004FEAC802B8EB020280
:1067D00046EA587664EB060651184CEB060C18EBAB
:1067E000080644EB040A16EB080644EB0A0A4FEAD3
:1067F0008A0A4AEA967AB600B6EB08026AEB040403
:10680000520842EAC4729B1A6EEB640EA8E700BFFE
:10681000C85E002024FAFFFF31B10A4BD3ED0C7A99
:10682000FDEEE77AC1ED007A52B1064B9FED067A94
:10683000D3ED0D7A67EE877AFDEEE77AC2ED007A46
:1068400001207047C85E00200000C84200797047F0
:106850000079C0F34010704700794009704700BFCD
:10686000704700BF704700BFD0ED007AD0ED036ADB
:1068700030EE677AE6EE877AB0EE670AC0ED007A0E
:10688000704700BFD0ED017AF5EE407AF1EE10FAD4
:1068900005D19FED0C7AC7EE207AC0ED017A31EE7A
:1068A000277AD0ED007A80ED021AC1EE076A30EE49
:1068B000677AC0ED036AE6EE877AB0EE670AC0ED4C
:1068C000007A704783F9223E9FED047AC7EE007A82
:1068D00077EEA07A80EEA70A704700BF72C7D13D5D
:1068E00000230360436080ED020A704790ED017A57
:1068F000D0ED036AD0ED027A30EE470AA6EE807A38
:1069000090ED000A80ED017A37EE676AE6EE867A4E
:1069100037EEC07AC0ED027AA6EE870A80ED000A53
:10692000704700BFD0ED056AD0ED017A90ED007A96
:1069300090ED066AD0ED025A90ED035A80ED050AFB
:1069400066EEA77AC0ED066AE7EE007A90ED077A68
:10695000E5EE867A90ED086AD0ED045A80ED087A6B
:10696000E5EE477AE5EEC67AB0EE670AC0ED077A43
:10697000704700BFD0ED057A90ED006A90ED067A81
:10698000D0ED035AE6EE007A90ED016AF0EE406A2F
:10699000A6EE267AB0EE670AD0ED047A90ED026A90
:1069A00067EEC07AA5EEC07AE6EE267A80ED057A2B
:1069B000C0ED067A704700BF03685A1C0260197068
:1069C000704700BF03690133012B03611CD0D0ED78
:1069D000005AD0ED026A07EE903A30EE656AF8EEA2
:1069E000E77A86EE277A77EE257AB0EE667A30EE91
:1069F000670AC0ED017AA6EE007AC0ED007A80ED5C
:106A0000037A80ED027A7047002380ED010A80ED61
:106A1000000A8360704700BF03685A1C0260197047
:106A2000704700BF024B986B03681B68184700BF94
:106A3000C85E002090F83020034602F0FF0012B13B
:106A4000002283F8302070474FF4805383817047D1
:106A50004FF4006383817047012070470120704725
:106A60002DE9F84F6E4DD5F83CC0B5F84000B5F9AA
:106A70004A90B5F846E0C0EB2C1303FB03F4B5F9DC
:106A80004430241303FB04F44000B5F94230C0EB5A
:106A9000EC0003FB00F0A41304EBE024B5F948304C
:106AA000AC650F46A4F5FA31164683FB013281FB33
:106AB000018C12034FEAE97B42EA13524FEA033A90
:106AC00009FB0CF308FB0B3BA9FB0839D9441B0A53
:106AD00043EA096313EB0A0342EB292202F5004261
:106AE000A3FB0E390EFB029E4FEAEE734FEA6E02D5
:106AF00053EA6E0E4FF0000000F08580B5F950901B
:106B000009FB0CFEB5F94EC08CFB011C4FEAE97A7B
:106B10004FEA4C4C08FB0AEE4CEAD13CA9FB089822
:106B2000490411EB0901F04448EB0C0C4018E96DE5
:106B3000C1F58019B5F94C1009F0004E4FEAC9783B
:106B4000B8EB00080CEBC1014EEA590E6EEB010EDA
:106B500018EB080C4EEB0E011CEB080C4EEB010180
:106B60004FEA81194FEA8C1049EA9C691CEB000C32
:106B700041EB0901890041EA9C714FEA8C0C1CEB46
:106B8000080C4EEB01014FEA8C00890010EB080065
:106B900041EA9C714EEB01016AF0F6F8B5F9562016
:106BA000B5F954E0B5F952504FEA6138430B43EA66
:106BB000C14302FB08FC4FEAE27903FB09C9A2FBCF
:106BC000032CCC4402FB08F803FB0C88A2FB032C2B
:106BD000C444520E42EACC12121841EB6C6C4FEADC
:106BE000EE730EFB01F103FB0011AEFB003001441C
:106BF000DB0C43EA4133D0184CEBE141000A40EA98
:106C0000016000EB05100FB1000A386026B104EBFB
:106C100084048034241234600120BDE8F88F00BF62
:106C2000C85E0020012070470C4B0D481B6810B453
:106C3000046E1B1BFA2B09D809B1436E0B604AB1D5
:106C4000836E5DF8044B13600120704700205DF8EF
:106C5000044B704701205DF8044B70474435002019
:106C6000C85E0020034B0022C3E91B22C3E91D229A
:106C700001207047C85E0020094B0A4A1B68916FCB
:106C80005B1AFA2B0AD810B4D2E91B41536FC486A1
:106C9000018743875DF8044B01207047002070474F
:106CA00044350020C85E00202DE9F04F984D0026A5
:106CB00005F17C0C95F8C010A5B00A243346E646D1
:106CC00037469BE002EBC70205EB4200C2F3072701
:106CD000B0F8C40010F0040F5FFA82FEC6B24FEAAB
:106CE000102900F0C480480614D403F10208B8F15A
:106CF0008C0F41F0400100F2FC800DF1900A581C0D
:106D000053444FF0040A03F88CAC24AB034403F85B
:106D10008C1C434603F10208B8F18C0F47F0020BBC
:106D200000F2E78024A8184400F88BBC4FF0050B54
:106D300000F88CBC03F1040BBBF18C0F00F2D9807E
:106D40000DF1900AD044B6004FF0060A08F88CAC5A
:106D50005FFA86F89E1D8C2E00F889EC00F2C9803F
:106D60000DF1900AD3444FF0070A0BF88CAC00F8F1
:106D7000878C03F10808B8F18C0F00F2BA800DF18E
:106D8000900B5E444FF0050B06F88CBC03F10A062D
:106D90008C2E00F8857C00F2AC8024AFB8444FF014
:106DA000060A08F88CAC00F883EC03F10C008C2880
:106DB00000F29F800B333B443E444FF0070A06F835
:106DC0008CAC03F88C9C0346570902F01F00012687
:106DD00086405CF82700013C20EA06004CF82700BA
:106DE00000F08A80561CB6F5F07F80F0858072092D
:106DF0000CEB820E9700474A96457DD206F01F02A3
:106E00004FF0FF30DEF8006000FA02F2324092FAF2
:106E1000A2F2B2FA82F2D2B2202A7FF453AF3D4AF4
:106E20000EF1040090421AD23B4AA2EB0E0727F063
:106E300003070EF1080E774401E0B8420FD0064672
:106E40000430326892FAA2F2B2FA82F2D2B2202A66
:106E5000F3D0A6EB0C0612EBC6027FF535AF85F832
:106E6000C0101846002B49D125B0BDE8F08F11F0B5
:106E7000400F03D101F03808B04513D021F078015C
:106E80009E1C01438C2EC9B233D80DF19008581CBA
:106E900043444FF0040803F88C8C24AB034403F8FC
:106EA0008C1C3346981C8C2823D824AE06EB030890
:106EB0004FF0050608F88C6C1E1D8C2E08F88B7C94
:106EC00017D824AF38444FF0060700F88C7C981D83
:106ED0008C2808F889EC0CD824AF3E444FF0070703
:106EE00006F88C7C053324AE334403F88C9C0346AF
:106EF0006AE76FF0004367E785F8C010D5F8B8007F
:106F000001AA002169F006F8012025B0BDE8F08F44
:106F1000C85E0020805F00207B5F00202DE9F041EB
:106F20000C4E356873691D4011D0DFF82C800127A5
:106F3000B5FA85F4C4F11F0408EB840307FA04F4DE
:106F4000D3F8840403689847A5437461F0D1BDE881
:106F5000F08100BF003C0140C85E002038B51446F7
:106F600000294CD0394B9FED3A6AD3F8C42407EE80
:106F7000902AB8EEE77AD3F8E024C7EE066A0D4609
:106F800007EE902AB3F9DC2404EE902AB3F9D82452
:106F900005EE902AB3F9DA24F8EEE77A05EE102A26
:106FA000D3F8D02487EE864AF8EEE44A07EE902A1A
:106FB000F8EEE55AB3F9D624E6EEA45A06EE102A06
:106FC000B8EEE77A03F2CC42B8EEC55AB3F9D4343E
:106FD00092ED000AB8EEC66AA6EEA57AA6EE856A1C
:106FE00007EE903AB8EEC00AF8EEE77AA6EE870A06
:106FF000E6EE867AA4EE270A6CF038FB28601CB314
:10700000124BDFED135AB3F9CA249FED120A07EEB3
:10701000902AD3F8E024B3F9C83407EE102AB8EE6A
:10702000C76A06EE903A86EE257AF8EEE77AF8EE31
:10703000E66A67EE277AB6EE006AE6EE867A27EE13
:10704000800A6CF013FB2060012038BDC85E002070
:107050000000F04A0000C84238B50409013C032C86
:1070600018D80E4D35F8141000F00F0341FA03F252
:1070700012F0010210D001209840013808402C4441
:1070800069F0EAFE237A064A184400EB400002EB5E
:10709000800038BD002038BD104638BD1C6B070885
:1070A000F02A00202DE9F04F3C2204460021B84888
:1070B00093B06FF00CFCB74A611EE01C144611F847
:1070C000013F5D1E032D88BF0023814244F8043B2D
:1070D000F5D102F11003114651F8040B012800F01C
:1070E0004C818B42F8D10020114651F8044B022C00
:1070F00000F039818B42F8D1114651F8044B032C32
:1071000000F027819942F8D152F8041B042900F0BD
:1071100016819342F8D1DFF878B2DFF898829E4F5B
:107120005C460F250026002839D0FFF795FF94F91B
:107130000D908246C0B1052383710023037203685A
:10714000964AC57103F13F4303F57E039B0AD05C69
:1071500066F018FDBAF804300393914B0493DAF803
:10716000000003A9FCF742F9217B0023302201E053
:1071700018F8332091422BD00133102BF8D1002284
:1071800009EB490907EBC90322615A6922750132EB
:107190005A6107210122A17562751A7416440135DE
:1071A000EDB2132D04F10C0401D0207BBBE766B1D6
:1071B000794CDFF804920025237C73B90135032D47
:1071C00004F1180409F1C809F6D113B0BDE8F08F35
:1071D000744A02EBC3031A69D2E7607966F0D2FC05
:1071E000207966F0CFFCA068FCF76AF82368A068F5
:1071F000CDF814904C3304936369142202FB03F31B
:1072000007930023CDE90E33CDE91033069308939D
:10721000E36803934FF480624FF40063CDE90923E0
:107220004FF400514FF48073CDE90B134FF400334A
:1072300003A90D9366F07AFCA2685B49136843F0DA
:1072400001031360594A536823F4733323F44773DB
:1072500023F0030343F440335360226863695068AA
:107260000194012B20F0407020F48070D4BF0026E0
:10727000012640EA062050609068014041F002017A
:107280009160D16A013B21F47001DBB241EA035302
:10729000D3620BF130075B4601214FFA85FC4FF0BA
:1072A000070A587D18B193F90D00604514D00C33CE
:1072B000BB42F6D19368019C43F4007393609368DA
:1072C00043F480739360936843F001039360936881
:1072D00043F08043936071E7187C4E1C09285FFAE5
:1072E00086F89E7D1CD8146900EB400E06FA0EF657
:1072F0000AFA0EFE24EA0E0E46EA0E06166106296A
:107300005CD8013901EB8101D2F834E01F2404FA82
:1073100001F688402EEA0606304341465063C6E730
:10732000A0F10A0ED4680EEB4E0E06FA0EF60AFA1B
:107330000EFE24EA0E0E46EA0E06D660DFE71C4B70
:1073400093F888273021013283F8141583F88827B1
:10735000E1E61749202481F8084591F8884701346F
:1073600081F88847D0E61249352481F8FC4491F829
:107370008847013481F88847BEE60D4991F888476F
:107380003420013481F8F00481F88847ACE600BF6E
:10739000AC630020E863002080120020D46A070854
:1073A000030001001C6B0708FDF7FFC0002301402C
:1073B000C85E0020286B0708F86300200C290ED84F
:1073C000073901EB8101D2F830E01F2404FA01F6FD
:1073D00088402EEA060630434146106367E70D39C0
:1073E00001EB8101D2F82CE01F2404FA01F6884059
:1073F0002EEA060630434146D06258E728B30368B8
:10740000124A30B503F13F4303F57E039B0A05465C
:1074100083B00C46D05C66F0B5FBA988009104F0FF
:107420000303C4F381028DF8043028688DF8052029
:10743000C4F300136946C4F341148DF806308DF887
:107440000740FBF7D3FF03B030BD7047D46A07088D
:1074500082B08DED010A019802B07047C31783EA2C
:10746000400070479FED087AC0ED020AC7EE007A2F
:107470000023036030EEA77AC0ED017AC0EE877A70
:10748000C0ED037A704700BF83F9223E80ED010A08
:10749000704700BF90ED017AD0ED007AC0ED020A8E
:1074A00030EE877AC0EE876A30EE677AE6EE877A4A
:1074B000B0EE670AC0ED007A704700BF80ED000AA9
:1074C000704700BF9FED047AC7EE007A77EEA07A8E
:1074D00080EEA70A704700BF4E2DA63D0023036033
:1074E0004360836080ED030A704700BF80ED030AAC
:1074F000704700BFF5EEC00AF1EE10FA06DCF0EEC0
:10750000407A80ED000AB0EE670A704760EE810AAB
:1075100090ED007A77EE607AF4EEC07AF1EE10FA30
:107520000ADC77EE200AF4EEC00AF1EE10FA8CBF06
:10753000F0EE407AF0EE607AC0ED007AB0EE670AC5
:10754000704700BFB4EEE00AF1EE10FA07D4B4EED3
:10755000C10AF1EE10FA88BFB0EE410A7047B0EEF2
:10756000600A7047894BB3FBF2F399420DD30023B5
:107570004FF07E52026043608360C360036100236A
:10758000836143610362C361704707EE902ADFEDB8
:10759000806AB8EE677A07EE901A27EE267AF8EE40
:1075A000677A27EE277AFDEEC77A17EE903A2033F6
:1075B000402B00F2DA80DFED777AB4EEE77AF1EE75
:1075C00010FAF0EE477A0CDDDFED735A9FED736A27
:1075D000F0EE676AF4EEC66AF1EE10FA77EEE57A3D
:1075E000F6DCDFED6F6AF4EEE67AF1EE10FA0CD518
:1075F000DFED695A9FED6B6AF0EE676AF4EEC66ADA
:10760000F1EE10FA77EEA57AF6D4DFED676AF4EEC4
:10761000E67AF1EE10FA00F39C80DFED646AF4EE96
:10762000E67AF1EE10FA44BFDFED5D6A76EEE77AB6
:1076300027EEA76ADFED5E5ADFED5E6A9FED5E5AC8
:10764000DFED5E4AE6EE256ADFED5D5AA6EE265ACC
:1076500027EE864AE6EE055AF7EE006AE4EE257A52
:10766000F0EE665AE7EEA45AE7EEE46A86EEA54A23
:10767000DFED4D6A77EE267ABDEEE76A16EE103A38
:107680002033402B6AD8B4EEE67AF1EE10FA0CDD26
:107690009FED416ADFED416AB0EE677AB4EEE67ABB
:1076A000F1EE10FA77EEC67AF6DC9FED3D7AF4EE55
:1076B000C77AF1EE10FA0CD59FED376ADFED396A23
:1076C000B0EE677AB4EEE67AF1EE10FA77EE867AEB
:1076D000F6D49FED357AF4EEC77AF1EE10FA49DD73
:1076E0009FED2C7A77EE677A67EEA76A9FED306A96
:1076F0009FED307ADFED304A9FED315AA6EE867A63
:1077000027EEA63AE6EE874AB7EE006AA6EEA45A3E
:10771000B6EE007AE3EE057AF8EE003A36EE676AE6
:1077200067EEA37A26EE077AB7EE005AC5EE256A11
:1077300080ED044A26EE877A26EE866A66EEA77A00
:1077400080ED007A80ED016A80ED027AC0ED037A67
:1077500015E7DFED106A76EEE77A69E7DFED197A73
:10776000B6EE007AB7EE006ADEE7B7EE004AF0EE5A
:10777000445A7DE79FED0D7AF4EEC77AF1EE10FAE8
:1077800044BF9FED077A77EE677AADE720A1070047
:1077900027D4D236DB0F4940DB0FC940E4CB16417A
:1077A000DB0F49C0E4CB16C1DB0FC93FDB0FC9BFFC
:1077B0009A7C2E36FAAF4FB93587083CF304353F33
:1077C000A4AA2ABE00000000FDEEC07A17EE903A8F
:1077D0002033402B53D8DFED2B7AB4EEE70AF1EEDD
:1077E00010FA0CDDDFED286A9FED287AF0EE407A82
:1077F000F4EEC77AF1EE10FA30EE660AF6DCDFED51
:10780000247AB4EEE70AF1EE10FA0CD5DFED1E6A29
:107810009FED207AF0EE407AF4EEC77AF1EE10FA9E
:1078200030EE260AF6D4DFED1C7AB4EEE70AF1EE6C
:1078300010FA1FDCDFED197AB4EEE70AF1EE10FA68
:1078400044BFDFED137A37EEC00A60EE007A9FED99
:10785000147A9FED146ADFED146AA7EE876A9FED34
:10786000137AE7EE866A60EE275AA7EEA67AA5EEAF
:10787000870A7047DFED037A37EEC00AE5E79FED30
:107880000C0A7047DB0F4940DB0FC940E4CB1641BF
:10789000DB0F49C0E4CB16C1DB0FC93FDB0FC9BF0B
:1078A0009A7C2E36FAAF4FB93587083CA4AA2ABE77
:1078B000000000009FED307A70EE077AFDEEE76A77
:1078C00016EE903A2033402B53D8B4EEC70AF1EEAF
:1078D00010FA0CDD9FED296ADFED296AB0EE677AB8
:1078E000B4EEE67AF1EE10FA77EEC67AF6DC9FEDAA
:1078F000257AF4EEC77AF1EE10FA0CD59FED1F6AE7
:10790000DFED216AB0EE677AB4EEE67AF1EE10FAB6
:1079100077EE867AF6D49FED187AF4EEC77AF1EE18
:1079200010FA21DC9FED197AF4EEC77AF1EE10FA25
:1079300044BF9FED147A77EE677A27EEA77ADFEDE2
:10794000146ADFED145A9FED146AE7EE265ADFED54
:10795000136AA7EE256A27EE875AE7EE066AE5EE78
:10796000267AB0EE670A70479FED0D7A77EE677A58
:10797000E3E79FED0C0A7047DB0FC93FDB0FC940FF
:10798000E4CB1641DB0F49C0E4CB16C1DB0FC9BF06
:107990009A7C2E36FAAF4FB93587083CA4AA2ABE86
:1079A000DB0F494000000000B5EE400AF1EE10FA8E
:1079B00025D007EE902AF8EE670ADFED117A08B5B8
:1079C000034660EEA70A0846F0EE406A13B9FFF7D7
:1079D00049FD0CE0022B06D0032B08D1FFF772FD06
:1079E000BDE808407AE5FEF76FFFFEF779FFFCEE91
:1079F000E66A16EE903A99B2BDE80840B2E57047E3
:107A0000BD378635B5EE400AF1EE10FA01D1044BD0
:107A100003E003280CBF034B034B0B60704700BF10
:107A200061680008ED6800087569000890ED0E7A3D
:107A3000B5EEC07AF1EE10FA00F3988030EE607A7D
:107A4000D0ED015A037867EE255A002B5BD101F087
:107A50000103D0ED117A002B61D077EE677AF0EE5A
:107A6000470A87EE816AD0ED0F6AC0ED110AF5EE84
:107A7000C06AF1EE10FA57DCD0ED037A26EE276AE1
:107A8000D0ED056A90ED105A60EE266A76EE857AA2
:107A900077EEA57A77EE867AF4EEE71AF1EE10FA31
:107AA00000F38480B4EEE72AF1EE10FA8CBFB0EE5A
:107AB000670AB0EE420A70EE677A90ED044AD0EDA4
:107AC000024AC0ED135A67EE847A4A07E7EE247A39
:107AD000B0EE457AA1EE277A80ED125A80ED146A55
:107AE000C0ED156A80ED160A08D5F0EEC77AF0EE03
:107AF000C56AF4EEE67AF1EE10FA6BD580ED107AF5
:107B00000B0756D4704711F001034FF000020CBF71
:107B1000F0EE607AF0EE477A0270002B9DD177EE9E
:107B2000E07A87EE816A9EE7D0ED0B7AD0ED034ACA
:107B3000F5EE407AF1EE10FA05D19FED285AC5EE28
:107B4000267AC0ED0B7A71EE276AD0ED0A7A80EDC5
:107B50000C1A81EE265A36EE676A80ED0D5AE5EE74
:107B6000067A24EEA76AC0ED0A7A89E7D0ED077A93
:107B7000F5EE407AF1EE10FA70EE606A05D19FEDF5
:107B8000176AC6EE077AC0ED077A71EE277A90ED94
:107B9000067A80ED081A81EE276A76EEC77A80EDC4
:107BA000096AA6EE277A80ED067A49E7B0EE610A07
:107BB00081E7F4EEC71AF1EE10FA08DCB4EEC72A3A
:107BC000F1EE10FA8CBFF0EE471AF0EE421AC0ED5B
:107BD000101A7047B0EE457A92E700BF83F9223E53
:107BE000002301220270C364836403650364436459
:107BF0004365836283657047DFED1B7A80ED010A80
:107C0000F4EEE70AF1EE10FAC0ED020A80ED031A75
:107C1000C0ED051A12DC00238360036100230122FA
:107C200080ED0F2AC0ED0E2A0270C36483640365E1
:107C3000036443644365836283657047B4EEE70A77
:107C4000F1EE10FA0CDD81EE007AC0EE207AF0EE53
:107C5000006A77EE877A86EEA77A80ED047ADDE710
:107C600000230361DAE700BFBD378635F0EEC07A46
:107C7000B0EEE07AB4EEE77AF1EE10FAB4BFB0EE0F
:107C8000676AB0EE476AB5EE406AF1EE10FA46D088
:107C9000B4EEE77AF1EE10FA8CBFF0EE675AF0EE30
:107CA000475AC5EE866ADFED1F2ADFED1F3ADFED8A
:107CB0001F4A9FED1F5A9FED1F3A9FED1F4ADFEDB0
:107CC0001F5AE6EEE23AA6EE834AE6EEA34AB7EE84
:107CD000006AA6EEA45AA6EE846AE6EE855AC5EEC0
:107CE000866AB4EEE77AF1EE10FA48BFDFED147A57
:107CF000F5EEC00A48BF77EEE66AF1EE10FA48BF2B
:107D0000DFED107AB5EEC00A48BF77EEE66AF1EE15
:107D100010FA48BFF1EE666AB0EE660A7047DFED12
:107D2000076ADEE739094E3DE3B59E3E88FA163E06
:107D300045FE7F3F99FB243F69A2163EA7DFA8348A
:107D4000DB0FC93FDB0F4940B7EE007AF0EEC07A97
:107D5000F4EEC77AF1EE10FA77EE676A1DD8B1EE4D
:107D6000E67ADFED0F5ADFED0F6A9FED0F6AE7EE5F
:107D7000A65ADFED0E6AA7EEA56AE7EE866A67EE01
:107D8000266AB5EEC00AF1EE10FA44BF9FED087AFC
:107D900077EE666AB0EE660A7047DFED066AF0E7D6
:107DA0002716983D306E99BC843459BEA40DC93F46
:107DB000DB0F494000000000B0FBF1F301FB1303AF
:107DC00008463BB11946B0FBF1F301FB130308462B
:107DD000002BF7D1704700BF44F25063984203DD97
:107DE000A0F50C40A0387047034B9842BCBF00F58B
:107DF0000C40A030704700BFB0B9FFFF48F69F436A
:107E0000984203DDA0F50C40A03870470028BCBFA5
:107E100000F50C40A030704780EAE073A3EBE073FC
:107E20008B4203DB002803DD401A704700207047B7
:107E3000FDD00844704700BF884203DB9042A8BFD2
:107E4000104670470846704700230361704700BF23
:107E5000036970B50446A3B1214DD4ED067A77EEDF
:107E6000807A013304F11C062361C4ED067A3046A2
:107E7000FEF7A8FD62682B689B1AA268934207D898
:107E800070BD4268164D002AE7D12A684260E4E7D7
:107E9000E06A94ED0A0A67F009FCD4ED057AB4EEC5
:107EA000E70AF1EE10FA04DD237B7BB10323237094
:107EB00070BDD4ED047AD4ED066AF8EE677A022339
:107EC00086EEA77A237084ED067A70BD296861601A
:107ED00000222361A2613046BDE87040B4E700BFD4
:107EE000443500202DE9F04100F11C0604463246DD
:107EF000054600F1640752ED017AB1EC010A77EE14
:107F0000807A104642ED017A1832FEF75BFD974207
:107F1000F1D12369264F6268013323613B689B1AC4
:107F2000A268934229D904F14808E86A95ED0A0A43
:107F300067F0BCFBD4ED057AB4EEE70AF1EE10FA77
:107F400005F118051BDCA845EFD1D4ED047AD4ED7A
:107F5000066A94ED0C7AD4ED125AF8EE677A022391
:107F600086EEA76A2370C7EE276A85EEA77A84EDAE
:107F7000066AC4ED0C6A84ED127ABDE8F081237BB9
:107F80001BB103232370BDE8F0813968236100220F
:107F900030466160A261FFF757FF04F134002263AD
:107FA000FFF752FFA26404F14C00BDE8F0414BE73B
:107FB0004435002010B4019C401AA4EB030C00FBD4
:107FC0000CFC511A5DF8044B9CFBF1FC0CEB03001C
:107FD000704700BF30EE600A32EE612A71EE600A2F
:107FE00022EE002A82EE200A30EE210A704700BFFE
:107FF000D1ED007ADFEDE36A37EEA67ABDEEC76A0F
:1080000016EE103A2033402B00F25D82F4EEE67A51
:10801000F1EE10FA0CDDDFEDDC5A9FEDDC6AF0EEDC
:10802000476AF4EEC66AF1EE10FA37EE657AF6DCCE
:10803000DFEDE26AB4EEE67AF1EE10FA0CD5DFED90
:10804000D25A9FEDD56AF0EE476AF4EEC66AF1EEB9
:1080500010FA37EE257AF6D4DFEDCA6AB4EEE67A86
:10806000F1EE10FA00F30D82DFEDD36AB4EEE67A9A
:10807000F1EE10FA44BFDFEDD16A36EEC77A67EE53
:10808000076A9FEDC76A9FEDC75ADFEDC75AA6EE94
:10809000865A9FEDC66AE6EE855A27EE264AA6EE78
:1080A000A56AA4EE067AF0EE474ABDEEE77A17EE2F
:1080B000103A2033402B00F203829FEDBD7AF4EE9C
:1080C000C77AF1EE10FA0CDD9FEDAF6A9FEDAF7A43
:1080D000F0EE676AF4EEC76AF1EE10FA77EEC67A50
:1080E000F6DC9FEDB67AF4EEC77AF1EE10FA0CD515
:1080F0009FEDA56A9FEDA87AF0EE676AF4EEC76A75
:10810000F1EE10FA77EE867AF6D49FED9E7AF4EED1
:10811000C77AF1EE10FA40F309829FEDA57A77EE67
:10812000677A27EEA77ADFED9E6ADFED9E5A9FED14
:108130009E6AE7EE265ADFED9D6AA7EE256A27EED6
:10814000874AE7EE066AE4EE267AB0EE675A91EDCA
:10815000017ADFED8C7A77EE276ABDEEE66A16EEDD
:10816000103A2033402B00F2A481B4EEE77AF1EE0E
:1081700010FA0CDDDFED845ADFED847AB0EE666A2A
:10818000B4EEE76AF1EE10FA76EEE56AF6DCDFEDC2
:108190008B7AF4EEE76AF1EE10FA0CD5DFED7A5A3D
:1081A000DFED7D7AB0EE666AB4EEE76AF1EE10FAC2
:1081B00076EEA56AF6D4DFED737AF4EEE76AF1EEB7
:1081C00010FA40F3A781DFED7A7A77EEE66A66EE81
:1081D000A67ADFED735A9FED734A9FED736AA7EE9F
:1081E000A54ADFED725AA7EE846A66EEA73AE7EE7B
:1081F000865AE3EEA56A66EEC52A24EEA63AB0EEEC
:10820000666AFDEEC77A17EE903A2033402B00F2F3
:108210004D81DFED677AB4EEE77AF1EE10FA0CDD0E
:10822000DFED595ADFED597AF0EE476AF4EEE76A6E
:10823000F1EE10FA37EE657AF6DCDFED607AB4EE37
:10824000E77AF1EE10FA0CD5DFED4F5ADFED527AF6
:10825000F0EE476AF4EEE76AF1EE10FA37EE257AAF
:10826000F6D4DFED487AB4EEE77AF1EE10FA40F397
:108270004581DFED4F7A37EEC77A67EE077ADFED9B
:10828000485A9FED484ADFED486AA7EEA54ADFED60
:10829000475AE7EE846A67EE273AE7EEA65AA3EE5E
:1082A000A57AF0EE476AD1ED027ADFED365A37EE65
:1082B000A57ABDEEC74A14EE103A2033402B00F2E7
:1082C000EA80F4EEE57AF1EE10FA0CDDDFED2E3AFD
:1082D0009FED2E4AF0EE475AF4EEC45AF1EE10FA32
:1082E00037EE637AF6DCDFED355AB4EEE57AF1EE7F
:1082F00010FA0CD5DFED243A9FED274AF0EE475AED
:10830000F4EEC45AF1EE10FA37EE237AF6D4DFED2C
:108310001D5AB4EEE57AF1EE10FA40F3E380DFED9A
:10832000245A35EEC77A67EE075A9FED1D4A9FED36
:108330001D2ADFED1D3AA5EE842A9FED1C4AE5EECD
:10834000823A67EE251AA5EEA34AA1EE847A25EEBD
:10835000072A64EE871A26EE821A26EE077A26EEA0
:10836000A10AFDEEE75A15EE903A2033402B00F2B9
:108370008D80DFED0F5AF4EEE57AF1EE10FA2CDD88
:108380001EE000BFDB0FC93FDB0FC940E4CB164145
:10839000E4CB1641DB0FC940E4CB16C1DB0FC93F6C
:1083A0009A7C2E36FAAF4FB93587083CA4AA2ABE6C
:1083B000DB0F494000000000DB0FC9BFDB0F49C0E5
:1083C0005FED0C3A1FED0E4AF0EE675AF4EEC45A18
:1083D000F1EE10FA77EEE37AF6DC5FED085AF4EE90
:1083E000E57AF1EE10FA0CD55FED163A1FED164A5C
:1083F000F0EE675AF4EEC45AF1EE10FA77EEA37A73
:10840000F6D45FED1A5AF4EEE57AF1EE10FA5DDD7E
:108410005FED195A75EEE77A27EEA74A5FED205A0D
:108420005FED203A5FED200AE4EE253A67EE845ACC
:10843000E4EE230A5FED233AE4EE203AE5EEA37A78
:1084400064EEA74A65EE275AA6EEA42AE6EEE51AE0
:1084500067EEC67A31EE241A75EEC05A80ED007AC6
:10846000C0ED017AC0ED026A80ED031AC0ED041A76
:10847000C0ED052AC0ED065A80ED072A80ED083AC6
:1084800070475FED356A36EEC77AF8E55FED375A2B
:10849000F0EE657AE0E71FED392AF0EE421AB0EE11
:1084A000420AB0EE421AB0EE427A5AE75FED3F6AF6
:1084B000F9E61FED403AF0EE432AB0EE436AA0E63B
:1084C0001FED445A43E65FED454AEEE55FED465A3F
:1084D000F4EEE57AF1EE10FA44BF5FED485A75EE1E
:1084E000E77A99E75FED4C5AB4EEE57AF1EE10FACF
:1084F00044BF5FED4E5A35EEC77A14E75FED527A0E
:10850000B4EEE77AF1EE10FA44BF5FED547A37EE3D
:10851000C77AB2E65FED587AF4EEE76AF1EE10FA48
:1085200044BF5FED5A7A77EEE66A50E61FED5E7A59
:10853000F4EEC77AF1EE10FA44BF1FED607A77EEE1
:10854000677AEEE50023036143618361C3610360E1
:10855000036243628362C362436003634363836372
:10856000C3638360036443648364C364C36070470C
:10857000D1ED017A91ED007AD0ED044A90ED065AE2
:10858000D0ED075A90ED050AD0ED080AD0ED0A1A91
:10859000D0ED0C2A90ED0D3AD0ED0E3A90ED091A7F
:1085A00090ED0B2AF8EEE76AD1ED027AB8EEC77AC1
:1085B000F8EEE77A26EEA64AA7EE275AE7EE074A34
:1085C000B0EE446A75EE875AA7EE076AE7EE272AEF
:1085D000E7EEA73AA7EE260AE7EE260AE6EEA71A86
:1085E000A6EEA73A31EE041AC0ED044A90ED0F4A08
:1085F000D0ED104A80ED065AC0ED075A90ED115AA1
:10860000D0ED125AC0ED0E3AA7EEA76A34EE274A13
:1086100074EE874A75EEA75A35EE265A32EE262AB0
:1086200080ED0F4AC0ED104A80ED115A80ED050A29
:10863000C0ED080A80ED091AC0ED0A1A80ED0B2A78
:10864000C0ED0C2A80ED0D3AC0ED125A90ED004AB3
:1086500090ED025AD0ED014AD0ED133AD0ED035A15
:10866000A7EE064AB0EE457AA7EE867AE6EE864A8F
:10867000F7EE007A73EEA77A35EE866AC0ED137ACC
:1086800080ED004AC0ED014A80ED027A80ED036A78
:10869000704700BF10B50024034684468646002C70
:1086A00000F00E81DEED006A9CED007AD3ED007AD9
:1086B000E6EEC77A012CC3ED007A00F01081DEED02
:1086C000016A9CED047AE6EEC77A032CC3ED007ACA
:1086D0006CD1DEED026A9CED087AE6EEC77AC3ED56
:1086E000007AD2ED007A90ED085AD0ED0C5AD0ED18
:1086F000044A92ED017AD2ED026A92ED036AA7EE86
:10870000E47AE7EEC56AA7EEE56A90ED095AD0ED86
:108710000D5AE7EE456AA5EEC76AD0ED0E5AA5EEF2
:10872000E66A81ED036A90ED0F5AC1ED026AC6EE6A
:10873000055AC1ED035A90ED0B6AE5EEC66AC1ED2C
:10874000026A90ED0A5A81ED017A86EE856A81ED22
:10875000026AD0ED066AA6EE667A81ED017AD0ED66
:10876000076AA5EEE67A81ED017A90ED055AC1ED32
:10877000007AC7EE056AC1ED016A90ED017AE7EE75
:10878000667AC1ED007A90ED027AE7EE467AC1EDA5
:10879000007A90ED037AE7EE657AC1ED007AD0EDCC
:1087A000006A87EEA67A81ED007A10BD9EED007A10
:1087B000DCED016AD3ED017AE7EE667A022CB1EEC8
:1087C000476AC3ED017ADEED016A9CED057AE6EEBB
:1087D000C77AC3ED017A40F0B580DEED046A9CED06
:1087E000007AD3ED047AE6EEC77A012CC3ED047A61
:1087F00040F28880DEED056A9CED047AE6EEC77AE9
:10880000032CC3ED047A40F08480DCED086A9EED11
:10881000066A93ED007AE6EE667AC7EE876AC3EDE4
:10882000046A9EED086ADCED006AD3ED087AE6EE94
:10883000667A012CC3ED087A74D99EED096ADCEDE5
:10884000046AE6EE667A032CC3ED087A07D19EED42
:108850000A6ADCED086AE6EE667AC3ED087A93ED03
:10886000086AD3ED0C7AC6EE076A032CC3ED086ADA
:108870009CED006ADEED0C6AE6EE667AC3ED0C7ADA
:108880009CED046ADEED0D6AE6EE667AC3ED0C7AC5
:1088900007D19EED0E6ADCED086AE6EE667AC3ED5E
:1088A0000C7AD3ED0C6AC6EE877AC3ED0C7A0134EC
:1088B00014330EF1100E0CF1040C002C7FF4F2AE08
:1088C000D3ED047A93ED007A93ED086AC7EE876AD8
:1088D000C6EE077AC3ED046AC3ED087AE1E7DEED80
:1088E000006A9CED016A93ED017AD3ED027AA6EE5F
:1088F000C67A83ED017A9CED027AE7EE667AC3EDE3
:10890000027A6AE793ED007AC7EE876AC3ED046ADC
:1089100087E793ED007AC7EE876A022CC3ED046AFD
:10892000C5D07EE7C7EE876AC3ED086ABFD09CED6D
:10893000006ADEED0C6AD3ED0C7AE6EE667AC3EDE2
:108940000C7AAEE79CED027AD3ED027AE6EE077A76
:10895000032CC3ED027ADCED066A9EED017AE6EEA9
:10896000C77AC3ED027A7FF438AFDEED026A9CED80
:108970000A7AE6EEC77AC3ED027AB2E610B584B0A1
:108980000C46024669461030FFF784FEDDED006AB2
:108990009DED017ADDED027AB6EE006A66EE866A3A
:1089A00027EE067A67EE867A0120C4ED006A84ED30
:1089B000017AC4ED027A04B010BD00BF20EE000AB7
:1089C000FEEE007A60EE277A60EEA00A9FED020AC2
:1089D000C7EEA00A6AF0CCBF54F82D4008B568F085
:1089E00075F807EE900AF5EEC07AF1EE10FAACBF1A
:1089F000B1EEE70A9FED010A08BD00BF00000000CC
:108A000060EEA00AE0EE000AB1EEE00A704700BF97
:108A100021EE011AA0EEA01AA0EE001AB1EEC10AD2
:108A2000704700BF2DE9F04F83B005469DF83040F8
:108A30000D9E0192002C14BF4FF030094FF0200919
:108A40001C1E88464ADB16F8010B014600286CD034
:108A5000002C65D04FF0000A324601E0002C34D0E3
:108A600012F8013B2746013C002BF7D1BAF1000F69
:108A70003CD1023F002C65D0BA4645450AF1FF3A89
:108A80004946284601D2019B9847BAF1FF3FF4D1ED
:108A90000D9A107823463C1B01469B4688B14FF047
:108AA000000A01339F1B454506EB070B284601D200
:108AB000019B984716F8011B0029F4D1BAF1000F69
:108AC00018D1584603B0BDE8F08FBAF1000F31D08D
:108AD000014683460028F4D02346E2E716F8010B4E
:108AE000634258B31C464FF0010AB5E7014683467E
:108AF0000028D6D1002C04F1FF36E2DD344645458E
:108B000006F1FF364946284601D2019B9847731C5F
:108B1000F5D10BF1010BA344584603B0BDE8F08F2B
:108B20002346A2464FF0FF34BBE7671EA346002C46
:108B3000A2D1C6E723464FF0FF34ADE7E6438346B4
:108B40003446DCE723463C46A6E700BF0FB430B509
:108B500083B006AB0B4C53F8042BD4F89017D4F821
:108B60008C07019364F0A0FE0546A06B03685B6967
:108B700098470028F9D0284603B0BDE8304004B03B
:108B8000704700BFC85E00200EB410B583B005ABBF
:108B9000044653F8042B0749009301A8019464F09C
:108BA00083FE019B00221A7003B0BDE8104003B0A1
:108BB000704700BF196A00080CB4F0B53C4CD4F8FB
:108BC0009437ADF5277D002B4CD094F89C37994213
:108BD00040D8384B384A1B68A2FB031292094FF465
:108BE0007A7101FB123306A83449FFF7CDFF06ABBB
:108BF00003443349AC9A01930646ADAB01A80093F8
:108C000064F052FE019BD4F894570A210246581C86
:108C100001901970019B591C01910021197035B305
:108C20002B681B6A1BB128469847D4F894579DF8C7
:108C3000181049B10DF119042B6828461B68984794
:108C400014F8011B0029F7D10DF5277DBDE8F04090
:108C500002B07047D4F8A027012303FA00F01042B5
:108C6000B7D1F1E7D4F89837002BAED1ECE7D4F8C0
:108C70009877002FE8D0901926AB841CFD20CDE911
:108C8000045506A92246ADF8100018466DF0E6FB23
:108C900002220346044402A93846CDE9023432F0E8
:108CA00065FC0DF5277DBDE8F04002B0704700BFC0
:108CB000C85E002044350020D34D621094FE0708A2
:108CC000B969000830B54FF4004087B02DF020FBA3
:108CD00058B14FF4004104462DF0D0FE022806D1D1
:108CE000226848F201039A4224D007B030BD002325
:108CF0004FF46121022294F904008DE80E001A4617
:108D00004FF4004130F0FAFD1C4BC3F894070028E3
:108D1000EBD01B4A1B4B1C4C1C481D490091CDE954
:108D20000332CDE901041B4B1B4A02210020FFF74F
:108D300043FFDAE7114C00254FF4004084F8385A1D
:108D400062F03EFD0028D0D0D4F8A43783420AD088
:108D5000D4F8803883420BD0D4F85C3998420AD0DA
:108D6000C4F89857C1E704F2A473C4F89837D0E761
:108D700004F50863F9E704F65C13F6E7C85E002023
:108D8000B8FE0708C4FE0708D0FE0708DCFE070887
:108D9000E4FE0708C0FD0708A0FE070838B5184C18
:108DA000D4F83C5A033005EB9003B3F5007F19D893
:108DB00020F003021348C4F83C3A00EB8101C3F5EC
:108DC0000073D1F8480104F524641044C1F8480147
:108DD0000D4A04EB85049B0004210020FFF7ECFE04
:108DE000204638BD00210846084AFFF7E5FE084A3C
:108DF0001368002443F000731360204638BD00BFA1
:108E0000C85E0020C06F0020F4FE070818FF0708A6
:108E10000000001038B50568EB69044653B1987836
:108E200000B938BD9A88E281DA8822821B89638280
:108E3000012038BD09211420FFF7B0FF0346E86187
:108E4000EDE700BF2DE9F041944603EB43031CF826
:108E5000068B86B0144602EB430315464FFA88F69C
:108E60009CF80070A0EB070E821BBEF1000FB8BF8C
:108E7000CEF1000E002AB8BF52429645B8BF6546F3
:108E80000CF1060CB8BF7EB26345E9D1B0456F88DE
:108E9000A3F1060206D0BE46A24216D014F8068FF1
:108EA000B045F8D1B4F80280CB1BA1EB080C002B25
:108EB000B8BF5B42BCF1000FB8BFCCF1000C6345FA
:108EC000BE46E9DD47462546E5E76B7904932B79F5
:108ED00003932B78064A0091CDE9013E0321034616
:108EE0000120FFF769FE284606B0BDE8F08100BF0B
:108EF00028FF070803681A46591C016012F8021B74
:108F00000260587841EA0020704700BF02681146AD
:108F1000531C036011F802CB0160D31C517803602D
:108F200093781B0443EA0123111D0160D07843EAC2
:108F30000C0343EA0060704712B370B504468646DE
:108F400004E0981B17D114EB0C0C15D01EF8013B54
:108F5000A3F14100192811F8010BA0F1410598BFB8
:108F60002033192DA2EB0E0C00F12006E9D91B1AB3
:108F700004D10028E7D170BD604670BD184670BDB1
:108F80001046704710B40288C378184CA2F5FA62F4
:108F900002F0030140F2B55C9208013B0CFB023386
:108FA000827801EB4101013A02EB810204EB4201BC
:108FB0000279B1F88C404179234403EB430302EB7F
:108FC000C30384790A4A0089C3EB031301EB8303CB
:108FD000C3EB0313224402EB830200214FF47A73A4
:108FE000C2FB03015DF8044B704700BF1C6B070810
:108FF00080436D382DE9F04117461E4605464FF473
:109000007A7200233846314667F0BEFE4449454A2D
:10901000014482FB0143C8170B44C0EB631382FB7E
:1090200003021A44D817404CC0EB621284FB0204BE
:109030004FEAE27C3D48CCEBA40C80FB0C404FEAAD
:10904000EC74C4EBE010C3EB0314A1EB8401A97131
:10905000C2EB0211A3EB81036B710CEB4C03A2EB8F
:10906000C30240F2B55303FB10CCBCF5896F2A71E3
:109070004FEA800045DA40F2DA239C4548DCBCF533
:10908000B77FB4BF00220122294B02EB420103EB60
:10909000C1034FEA4208B3F8A23091B2254C08EB65
:1090A000020E04EBCE0416344FF00B0E01E034F840
:1090B000023D634520DDBEF1010EF8D11C4B424458
:1090C00003EBC2024FF0010EB2F88C3085F802E0DB
:1090D00000F5FA600CF1010C0844ACEB030C28809D
:1090E00085F803C04FF47A7200233846314667F0A2
:1090F0004BFE2A81BDE8F0810EF1010E5FFA8EFE73
:10910000E4E7032140F296530A464FF00608C5E70C
:10911000022140F229430A464FF00408BEE700BF8F
:1091200080BC92C789888888ABAAAA2A73B06D16BA
:109130001C6B0708A86B070830B52E4D84468E4679
:109140000FCD8DB06C460FC40FCD0FC495E80F0046
:109150001CF0030F84E80F000DD1274B274A03FBB7
:109160000CF3B2EBB30F43D3254AB2EB331F2CBF42
:109170001D241C2400E01C240CF1FF33002B40F2C2
:109180006D12194602FB0CF2B8BF0CF1020102EBA2
:10919000A1021C491C4D019481FB0301DB17A3EBC9
:1091A00061100244C3EBE1131A44253285FB0230FF
:1091B0001044D317C3EBA000C0EBC000ADF1040313
:1091C000101A0DF1040C03EB8E0E01E05CF8044F55
:1091D000031985FB0320C218D817C0EBA200C0EB0F
:1091E000C000E645A3EB0000F0D1201A0DB030BD61
:1091F0001D24C1E7086C0708295C8FC2285C8F0218
:109200000AD7A3001F85EB519324499208B50C4B54
:10921000D3E9742352EA030C09D1002340F201126E
:1092200042808380837103800381184608BD05490D
:1092300009688A1843F10003FFF7DCFE012008BD2E
:10924000C06F0020443500208842F0B54FF0010483
:1092500061D301FB04F4B0FBF4FC8C45F9D284B378
:10926000002A45D0002511E0BCF1090F2646CCBFED
:10927000372230229444B14283F800C0744603F18F
:10928000010305F101051CD8B0FBFEFCB4FBF1FEA7
:1092900004FB1C00002DE7D1BCF1000FE4DCA1426F
:1092A0000BD8B0FBFEFCBCF1000F74460EFB1C009B
:1092B000BEFBF1FED8DCA142F3D90CF1300C03F86F
:1092C00001CB00221A70F0BDBCF1090F2646CCBFBD
:1092D0004FF0570E4FF0300EF444B14283F800C007
:1092E0002C4603F1010302F10102EAD8B0FBF5FCC0
:1092F000B4FBF1F504FB1C00002AE5D1BCF1000F22
:10930000E2DCA142D9D8B0FBF5FC2C4605FB1C00E1
:10931000B5FBF1F5F2E78446002AA3D1E8E700BFE8
:10932000002870B503DA2D2301F8013B40420928DB
:1093300004464FF0010307DD03EB83035B00B0FB42
:10934000F3F2092AF8D83BB3164D4FF0000C0AE0AF
:10935000092A8CBF572130210A44092B0EF8012B12
:1093600016D971460346A5FB0320B4FBF3F25CEA71
:1093700002068E464FEAD00003FB12440CF1010CAA
:10938000E6D1092B01D9B446EBE730320EF8012BB8
:1093900000238EF8003070BD8E4600238EF800301A
:1093A00070BD00BFCDCCCCCC90422DE9F0410B4636
:1093B000044615460AD2B0FBF5F6134A05FB1644DF
:1093C0001846135D00F8013BBDE8F081B0FBF2F6F2
:1093D0009642B6FBF2F706D20B4A05FB1767D15D42
:1093E00003F8011BEAE7BA42B7FBF2F807D9064ACD
:1093F00005FB187812F8081003F8011BEDE740464A
:10940000FFF7D2FF0346F2E764FF0708B5EEC00A94
:10941000DFED347AF1EE10FACCBF30EE270A30EEF1
:10942000670ADFED317A20EE270A70B5FDEEC07ACB
:1094300086B017EE904A054684EAE470002303A93B
:10944000A0EBE470CDE90033029364F0BFFB002C85
:10945000ACBF20232D2303A88DF8003066F0A2FEB8
:1094600001286E4628D0022832D003281CD003A938
:1094700030466DF034FA304666F094FE0338C4B2DC
:109480002246314628466CF0E9FF00232B5528463A
:1094900066F088FE2E232B540130311928446DF0DC
:1094A0003AFA284606B070BD302303A930468DF83D
:1094B00001306DF014FADEE743F23002302303A9E5
:1094C0003046ADF801208DF803306DF008FAD2E790
:1094D00043F2300303A93046ADF801306DF0FFF9D7
:1094E000C9E700BF6F12033A00007A440378202BCB
:1094F000024600F10100F9D0092BF7D02D2B28D01E
:109500002B2B03BF5378B7EE000A0246B7EE000AD2
:10951000A3F13001C8B209289FED567A10D8F2EEB7
:10952000046A07EE901AF8EEE77A12F8013FE7EEC8
:10953000267AA3F13001C8B20928B0EE677AF0D9D3
:109540002E2B5ED003F0DF03452B07D020EE070A59
:1095500070475378BFEE000A0246D9E710B451783D
:109560002D2978D02B296AD0A1F13003092B02F1E3
:1095700001026BD80024002303EB830301EB4303B8
:1095800012F8011FA1F130000928A3F13003F3D92B
:10959000B3F59A7F1A4628BF4FF49A72072B66D903
:1095A000DFED356A1346F7EE007A083B072B67EECE
:1095B000A67AFAD802F00702DAB1F2EE046A012ABA
:1095C00067EEA67A15D0022A67EEA67A11D0032A92
:1095D00067EEA67A0DD0042A67EEA67A09D0053A7E
:1095E00067EEA67A05D067EEA67A012A18BF67EE65
:1095F000A67A6CB387EE277A5DF8044B20EE070A53
:1096000070475378A3F13001C8B2092802F1010272
:1096100098D8F2EE046AF0EE665A07EE901AF8EE69
:10962000E77A12F8013F87EEA66AA3F13001C8B2CB
:10963000092866EEA56A37EE067AEED982E79178B8
:10964000A1F13003092B02F1020293D9F7EE007A5F
:1096500027EE277AD0E79178A1F13003092B02F1A8
:10966000020288BFF7EE007AC4D8012483E7F7EE40
:10967000007AA1E70000000020BCBE4C0378202B3C
:10968000024600F10100F9D0092BF7D0303BDBB2E4
:10969000092B4FF000000AD812F8011F00EB8000E0
:1096A000303903EB4000CBB2092BF5D97047704736
:1096B0000378202B024600F10100F9D0092BF7D0E6
:1096C0002D2B0CBF0246012092F800C0ACF13001F6
:1096D000CBB208BF4FF0FF30092B4FF000030CD87E
:1096E00012F801CF03EB830301EB4303ACF130012C
:1096F0005FFA81FCBCF1090FF2D903FB00F070475F
:10970000F0B5384D2B78082141F221008B4002E062
:10971000013993B209D013F4004F4FEA4302F7D056
:1097200080EA430301399BB2F5D1B5F80120002A44
:1097300055D0DFF8C0C02C4EB4452DD2ACF1060C8C
:109740000CEB0204B44227D2052A41F2210022D9AF
:10975000A44514D00CF1FF3C04F1FF3E1CF8011F9E
:10976000082283EA012313F4004F80EA43010ABF71
:109770005B008BB29BB2013AF5D1E645EED122886F
:1097800062B1A11DB14206D2A118B142A44602D2D3
:10979000052A0C46DCD800210846F0BDA71C264649
:1097A00041F2210016F8011B082283EA012313F479
:1097B000004F80EA43010ABF5B008BB29BB2013AC3
:1097C000F5D1B742EED16188084AC91AB1FA81F1E0
:1097D000231D49095B1BA2F8D8310846F0BD044F90
:1097E000BC1EDCE700000E0800001008C06F00205F
:1097F00003000E0807000E082DE9F0410446D0E9E9
:109800000030134483421DD88E188E4217D00D4667
:1098100004F10C08002701E0AE4210D023695A1C65
:109820002261234415F8010B1873042AF4D1414630
:109830002046F9F79DF8AE42C4E90470EED16069A4
:10984000BDE8F0814FF0FF30FAE700BF70B5458802
:109850000B460446C5F30B052A46002118466DF059
:1098600036F82169084A9142034602D3074A9142D9
:1098700005D319B1BDE870401846084770BD2A46A7
:10988000BDE870406CF0EABD7C6A0808226F0808E9
:1098900010B50446C06900B110BD09211420FFF7BE
:1098A0007DFAE06110BD00BF10B5184C04EB8000DC
:1098B000D0F8200530B300EB400004EB800393F9AF
:1098C000E5C4BCF1FF3F1ED093F8ED04D0B104EB2A
:1098D0000C0293F8EC0492F888E76423142103FB4C
:1098E0000CFC00220CEB000304EB43030139B3F83A
:1098F0003035704412FA83F2F4D10548A0FB0230EF
:10990000C0F30F1010BD002010BD00BFC85E0020C6
:10991000CDCCCCCC10B503681A79022A044603D00A
:1099200000232371236010BD987AFDF795FB002872
:10993000F6D040F619610022C18002722021FDF7A5
:109940005DFD00232371236010BD00BF70B5114B76
:10995000114CA34203D319E00C33A34216D293F85F
:1099600005C08C45F8D193F804C0844501D0002887
:10997000F2D193F807E09645EED11D6895F804E022
:10998000E645E9D12E689E42E6D100E00025284652
:1099900070BD00BF246F0808987008080379022B77
:1099A00000D0704710B590F9102082B002A8014491
:1099B00003241E488DF802304FF0000C02EB8202A7
:1099C0004FF0010E8DF800C08DF801E08DF80340D6
:1099D00050F8222011F8084C15498A4222D0A1F5EE
:1099E00078418A4220D001F580618A4218D11188DD
:1099F00021F04001090403EB8303090C118000EB03
:109A000083001388C16823F0380331F824101B0445
:109A10001B0C0B43138013889BB243F0400313804D
:109A200002B010BD6346E2E77346E0E76000002045
:109A3000003001400379022B00D0704783689B07F8
:109A4000FBD5436913B11A689B885383064B0749BA
:109A50001A68074B4868D200A3FB023292094B6890
:109A60001B1A9A42FBD27047E8290020001000E040
:109A7000D34D621070B50446234894F9103003EBBF
:109A80008303154650F82300A3689A0782B00CD5CB
:109A9000019066F087FA0198294666F083FAA36878
:109AA0009B0717D5012002B070BD636913B11A6816
:109AB0009B885383154B164A1B6856684FEAC30CA4
:109AC000144BA3FB0C3C4FEA9C1C53689B1B9C450E
:109AD000FBD2DDE70D4B0E491A680E4B4FF4FA70BE
:109AE00000FB02F2A3FB0232486892094B681B1A82
:109AF0009A42FBD26369002BD4D01A689B881383E7
:109B0000012002B070BD00BF60000020E8290020E5
:109B1000001000E0D34D621010B50379012B84B022
:109B20008E460DD0022B08D18368DB0758BF01F0A9
:109B30007F0104B0BDE810409CE7002004B010BDD8
:109B4000144682688DF80F4002F0010201920DF177
:109B50000F020092417C90F910007246FAF736FB32
:109B600004B010BD2DE9F041046884B00546B6226A
:109B70007E212046FFF7D0FF4FF0640806F034FE48
:109B800006460F4606F030FE831B61EB0701B3F576
:109B90007A7F71F10003F5D3B8F10108EED102210B
:109BA0002046FFF7FBFE636913B11A689B88538355
:109BB00006F01AFE06460F4606F016FE831B61EB02
:109BC0000702B3F57A7F72F10003F5D3636913B12D
:109BD0001A689B8813834FF00A0806F005FE0646B4
:109BE0000F4606F001FE831B61EB0701B3F57A7F98
:109BF00071F10003F5D3B8F10108EED142467C21A2
:109C00002046FFF789FF06F0EFFD06460F4606F0F7
:109C1000EBFD831B61EB0702B3F57A7F72F1000362
:109C2000F5D3002259212046FFF776FF06F0DCFD30
:109C300006460F4606F0D8FD831B61EB0702B3F51D
:109C40007A7F72F10003F5D394F91030A2688D4940
:109C500003EB83035E2092078DF80F0051F8230079
:109C600040F1E48001230DF10F020021019066F024
:109C700001F94FF4A473844A0198002166F0FAF8C0
:109C8000A3689B0740F1E5804FF00A0806F0ACFDA1
:109C900006460F4606F0A8FD831B61EB0701B3F5EE
:109CA0007A7F71F10003F5D3B8F10108EED10122FA
:109CB00059212046FFF730FF06F096FD06460F4675
:109CC00006F092FD831B61EB0702B3F57A7F72F118
:109CD0000003F5D38C2240212046FFF71DFF06F03C
:109CE00083FD06460F4606F07FFD831B61EB0702EE
:109CF000B3F57A7F72F10003F5D3022241212046A9
:109D0000FFF70AFF06F070FD06460F4606F06CFDF1
:109D1000831B61EB0702B3F57A7F72F10003F5D381
:109D2000EA6A5A4E95F82900B6FBF2F2092391B27D
:109D3000574AFFF787F84388B6FBF3F66E6302795C
:109D4000422142F0C0022046FFF7E6FE06F04CFD3D
:109D500005460E4606F048FD431B61EB0602B3F5CF
:109D60007A7F72F10003F5D3082243212046FFF7E2
:109D7000D3FE06F039FD05460E4606F035FD431BC1
:109D800061EB0602B3F57A7F72F10003F5D304228A
:109D900058212046FFF7C0FE06F026FD05460E4678
:109DA00006F022FD431B61EB0602B3F57A7F72F1E8
:109DB0000003F5D30A2253212046FFF7ADFE06F03B
:109DC00013FD05460E4606F00FFD431B61EB060230
:109DD000B3F57A7F72F10003F5D300227C2120468F
:109DE000FFF79AFE06F000FD05460E4606F0FCFC65
:109DF000431B61EB0602B3F57A7F72F10003F5D3E2
:109E000006227D212046FFF787FE06F0EDFC044682
:109E10000D4606F0E9FC031B61EB0502B3F57A7F02
:109E200072F10003F5D304B0BDE8F081636913B1AA
:109E30001A689B885383174B17491A68174B4E684B
:109E4000D200A3FB023292094B689B1B9A42FBD2C1
:109E500008E7104B10491A68104B48684FF4FA761F
:109E600006FB02F2A3FB023292094B681B1A9A42CC
:109E7000FBD26369002B3FF407AF1A689B881383FA
:109E800002E700BF60000020386C070840420F0066
:109E9000806D0708E8290020001000E0D34D621013
:109EA000F8B57822044600210068FFF735FE052743
:109EB00006F09AFC05460E4606F096FC431B61EB45
:109EC0000602B3F57A7F72F10003F5D3013FEFD1BB
:109ED000206820220121FFF71FFE052706F084FCE1
:109EE00005460E4606F080FC431B61EB0602B3F507
:109EF0007A7F72F10003F5D3013FEFD120683A4633
:109F00000221FFF709FE642606F06EFC04460D46AA
:109F100006F06AFC031B61EB0502B3F57A7F72F170
:109F20000003F5D3013EEFD10120F8BD70B5242226
:109F3000044641210068FFF7EFFD90B9052606F0C1
:109F400053FC04460D4606F04FFC031B61EB050273
:109F5000B3F57A7F72F10003F5D3013EEFD1012012
:109F600070BD206820223021FFF7D6FD0028E5D003
:109F7000206806223121FFF7CFFD0028DED02068BF
:109F800000223421FFF7C8FDD8E700BFF8B507224B
:109F900004460A210068FFF7BFFD052706F024FCF0
:109FA00005460E4606F020FC431B61EB0602B3F5A6
:109FB0007A7F72F10003F5D3013FEFD120682422AC
:109FC0004121FFF7A9FD052706F00EFC05460E46C8
:109FD00006F00AFC431B61EB0602B3F57A7F72F1CF
:109FE0000003F5D3013FEFD12068C0224221FFF7E3
:109FF00093FD052606F0F8FB04460D4606F0F4FB3B
:10A00000031B61EB0502B3F57A7F72F10003F5D310
:10A01000013EEFD10120F8BD10B5044600222121F8
:10A020000068FFF779FD2068FC222021FFF774FD0E
:10A03000206840222421FFF76FFD20680C22232195
:10A04000FFF76AFD206800222221FFF765FD01204D
:10A0500010BD00BFF8B50122074610210068FFF7C8
:10A060005BFD00B9F8BD142606F0BEFB04460D46A4
:10A0700006F0BAFB031B61EB0502B3F57A7F72F1C0
:10A080000003F5D3013EEFD13868A022BDE8F840C7
:10A09000112141E510B504682379012B84B010D05B
:10A0A000022B0BD1A368DB074FF0F0024CBFFF215E
:10A0B0007F21204604B0BDE81040DBE4002004B05E
:10A0C00010BDA268617C94F9100002F001020192B7
:10A0D0000DF10F020092F024FF228DF80F40FAF7E5
:10A0E00075F804B010BD00BF10B504682379CA43E9
:10A0F00041EA0211012B84B0CAB20ED0022B09D161
:10A10000A368DB074CBFD2215221204604B0BDE832
:10A110001040AFE4002004B010BD8DF80F20A268FD
:10A12000617C94F9100002F001020DF10F04CDE9F9
:10A130000042D222FAF74AF804B010BD10B5046804
:10A140002379012B84B010D0022B0BD1A368DB073D
:10A150004FF0B4024CBFFF217F21204604B0BDE880
:10A16000104087E4002004B010BDA268617C94F91F
:10A17000100002F0010201920DF10F020092B424CE
:10A18000FF228DF80F40FAF721F804B010BD00BF90
:10A1900010B504682379012B84B00FD0022B0AD1AB
:10A1A000A368DB070A4620464CBFA521252104B041
:10A1B000BDE810405EE4002004B010BDA26894F930
:10A1C00010008DF80F1002F00102617C0DF10F04F8
:10A1D000CDE90042A522F9F7F9FF04B010BD00BF98
:10A1E00010B504682379012B84B010D0022B0BD159
:10A1F000A368DB074FF096024CBFFF217F2120466A
:10A2000004B0BDE8104035E4002004B010BDA268E1
:10A21000617C94F9100002F0010201920DF10F022D
:10A2200000929624FF228DF80F40F9F7CFFF04B07B
:10A2300010BD00BF10B504682379012B84B00FD086
:10A24000022B0AD1A368DB070A4620464CBF8721B0
:10A25000072104B0BDE810400CE4002004B010BD9C
:10A26000A26894F910008DF80F1002F00102617CD1
:10A270000DF10F04CDE900428722F9F7A7FF04B0E2
:10A2800010BD00BF10B504682379C901012B84B04B
:10A29000CAB20BD0022B06D17821204604B0BDE80B
:10A2A0001040FFF7E7BB002004B010BD8DF80F2071
:10A2B000A268617C94F9100002F001020DF10F0414
:10A2C000CDE900427822F9F781FF04B010BD00BF4C
:10A2D00010B504682379012B84B011D0022B0CD166
:10A2E000A368DB074FF055024CBFA521252120466E
:10A2F00004B0BDE81040FFF7BDBB002004B010BDA6
:10A30000A268617C94F9100002F0010201920DF143
:10A310000F0200925524A5228DF80F40F9F756FF41
:10A3200004B010BD10B504682379012B84B00ED0A1
:10A33000022B09D1A368DB074FF031024CBFF42197
:10A3400074212046FFF796FB012004B010BDA268DF
:10A35000617C94F9100002F0010201920DF10F02EC
:10A3600000923124F4228DF80F40F9F72FFF0120DD
:10A3700004B010BD10B504682379012B84B00CD053
:10A38000022B07D101225821204604B0BDE810401D
:10A39000FFF770BB002004B010BDA26894F9100054
:10A3A000617C8DF80F3002F0010201920DF10F0275
:10A3B00000925822F9F70AFF04B010BD10B50468E6
:10A3C0002379012B84B00CD0022B07D10122482124
:10A3D000204604B0BDE81040FFF74CBB002004B09D
:10A3E00010BDA26894F91000617C8DF80F3002F066
:10A3F000010201920DF10F0200924822F9F7E6FEE8
:10A4000004B010BD10B504682379012B84B00CD0C2
:10A41000022B07D11A460821204604B0BDE810409F
:10A42000FFF728BB002004B010BDA268617C94F93E
:10A43000100002F0010201920DF10F0200920224BD
:10A4400008228DF80F40F9F7C1FE04B010BD00BF1F
:10A4500010B504682379012B84B00CD0022B07D1EE
:10A4600001220821204604B0BDE81040FFF702BBDE
:10A47000002004B010BDA26894F91000617C8DF832
:10A480000F3002F0010201920DF10F02009208223A
:10A49000F9F79CFE04B010BD30B505682B79012B8F
:10A4A00085B0044612D0022B0DD101220B21284683
:10A4B000FFF7E0FA38B120681D22092105B0BDE898
:10A4C0003040FFF729BB002005B030BDAA6895F9E0
:10A4D0001000697C8DF80F3002F0010201920DF13D
:10A4E0000F0200920B22F9F771FEE3E710B5154B4E
:10A4F000D3F8DC4184B024B12379012B10D0022B96
:10A5000002D0002004B010BDA16811F00101024684
:10A5100018BF8021204604B0BDE81040FFF7AABA5A
:10A52000A268617C8DF80F0002F0010294F910001E
:10A530000DF10F04CDE900428022F9F747FE04B087
:10A5400010BD00BFC06F0020F0B5054690F91000A7
:10A55000244C00EB800085B054F82000AC68A407C0
:10A5600010D5CDE90223019065F01CFDDDE9022341
:10A570000198002165F07EFCAB689B0718D501208F
:10A5800005B0F0BD6C6914B12668A4887483164CBC
:10A59000164E246877684FEAC40E154CA4FB0E4E85
:10A5A0004FEA9E1E7468A4EB070CE645FAD2D8E782
:10A5B0000D4B0E491A680E4B4FF4FA7000FB02F275
:10A5C000A3FB0232486892094B681B1A9A42FBD2DD
:10A5D0006B69002BD3D01A689B881383012005B0C8
:10A5E000F0BD00BF60000020E8290020001000E05E
:10A5F000D34D621030B50579012D83B08E460DD054
:10A60000022D08D18468E40758BF41F0800103B0EF
:10A61000BDE8304098E7002003B030BD14468268A2
:10A62000009402F00102417C90F910000192724600
:10A63000F9F7CCFD03B030BDF0B50546164695F9E7
:10A640001020244802EB820283B050F82200AA684E
:10A6500092070FD5CDE9000365F0A4FC019B00989B
:10A660000022314665F006FCAB689B0718D5012037
:10A6700003B0F0BD6A6912B1146892886283164A09
:10A680001468164A4FEAC40E154C5768A4FB0E4EC8
:10A690004FEA9E1E5468A4EB070CE645FAD2D9E7B0
:10A6A0000D4B0E491A680E4B4FF4FA7000FB02F284
:10A6B000A3FB0232486892094B681B1A9A42FBD2EC
:10A6C0006B69002BD3D01A689B881383012003B0D9
:10A6D000F0BD00BF60000020E8290020001000E06D
:10A6E000D34D621030B50579012D83B08E460DD063
:10A6F000022D08D18468E40758BF41F0800103B0FF
:10A70000BDE8304098E7002003B030BD14468268B1
:10A71000009402F00102417C90F91000019272460F
:10A72000F9F720FD03B030BD10B504460068037989
:10A7300082B0022B0CBF4321032106236A46FFF798
:10A74000D1FF68B1BDF80010BDF80220BDF804309B
:10A7500049BA52BA5BBAE1866287238702B010BD5C
:10A76000E086A06302B010BD70B50668F46982B0DF
:10A7700005466CB33379012B04F1030205D0022B9B
:10A780001AD00020A07002B070BDB368717C96F939
:10A790001000009203F0010301930C220D23F9F73E
:10A7A000E1FCA0700028EED06389AB83A389EB8322
:10A7B000E3892B8402B070BDB36813F0010F3046FB
:10A7C0004FF00D0314BF0C218C21FFF735FFE8E794
:10A7D00009211420FEF7E2FAF06104462E68C9E769
:10A7E00010B500680379012B84B00C4618D0022BF9
:10A7F00013D1836813F0010F14BF2221A221032378
:10A8000003AAFFF719FF30B1BDF90D3003EB830345
:10A810001B12E633238004B010BD002004B010BD2D
:10A820008368417C90F9100003F00103019303ABAE
:10A83000009322220323F9F795FC0028E4D1EAE7EC
:10A8400010B5044600680379012B84B01ED0022B9A
:10A8500019D1836813F0010F02AA4FF0060314BF49
:10A860001F219F21FFF7E8FE58B1BDF80810BDF881
:10A870000A20BDF80C3049BA52BA5BBAE181228293
:10A88000638204B010BD002004B010BD8368417C19
:10A8900090F9100003F00103019302AB00931F2213
:10A8A0000623F9F75FFCDFE710B50446006803797B
:10A8B000012B84B01ED0022B19D1836813F0010F35
:10A8C00002AA4FF0060314BF2521A521FFF7B4FE0D
:10A8D00058B1BDF80810BDF80A20BDF80C3049BACF
:10A8E00052BA5BBAA183E283238404B010BD002076
:10A8F00004B010BD8368417C90F9100003F001039F
:10A90000019302AB009325220623F9F72BFCDFE726
:10A9100010B500680379012B84B02ED0022B23D10F
:10A92000062302AAF721FFF787FEE8B19DF8092068
:10A930009DF808409DF80A109DF80C309DF80BC05A
:10A94000120142EA043242EA11121B019DF80D1075
:10A95000114C43EA0C3343EA11131049E265C1E993
:10A960007823E36304B010BD0C4A0B4BD2E9781294
:10A970000020D965DA6304B010BD8368417C90F98A
:10A98000100002AA03F00103CDE900230623F722F9
:10A99000F9F7E8FBC9E700BFC85E0020C06F0020E0
:10A9A00000B500680379012B85B01CD0022B0AD1B9
:10A9B000836813F0010F03AA4FF0030314BF0021B3
:10A9C0008021FFF739FE9DF80D309DF80C009DF8B1
:10A9D0000E100C4A1B0243EA00430B430120136094
:10A9E00005B05DF804FB8368417C90F9100003AA70
:10A9F00003F00103CDE9002303230022F9F7B2FBA2
:10AA0000E1E700BFC85E002000B500680379012BB4
:10AA100085B01CD0022B0AD1836813F0010F03AA62
:10AA20004FF0030314BF00218021FFF705FE9DF8BE
:10AA30000D309DF80C009DF80E100C4A1B0243EAE5
:10AA400000430B430120536105B05DF804FB8368AC
:10AA5000417C90F9100003AA03F00103CDE9002323
:10AA600003230022F9F77EFBE1E700BFC85E002068
:10AA700010B500680379012B84B029D0022B24D1B2
:10AA8000836813F0010F4FF0030303AA14BF1946A4
:10AA90008321FFF7D1FDB0B19DF80C309DF90C106A
:10AAA0009DF80D209DF80EC01B04002943EA0223E7
:10AAB000B8BF4FF07F410D4AA8BF002143EA0C0305
:10AAC0000B43C2F8E03404B010BD002004B010BD48
:10AAD0008268417C90F9100002F00102032303AC6C
:10AAE000CDE900421A46F9F73DFBD4E7C85E0020E5
:10AAF00000B500680379012B85B02BD0022B25D13E
:10AB0000836813F0010F03AA4FF0030314BF002161
:10AB10008021FFF791FDB0B19DF80C309DF90C102C
:10AB20009DF80D209DF80EC01B04002943EA022366
:10AB3000B8BF4FF07F410E4AA8BF002143EA0C0383
:10AB40000B43C2F8C43405B05DF804FB002005B027
:10AB50005DF804FB8368417C90F9100003AA03F0C0
:10AB60000103CDE9002303230022F9F7FBFAD2E722
:10AB7000C85E002010B5044600680379012B84B03C
:10AB80003DD0022B36D1836813F0010F02AA4FF09B
:10AB9000060314BF11219121FFF74EFD50B3BDF9FB
:10ABA000083006EE903ABDF90A30F8EEE66A07EE94
:10ABB000103ABDF90C30B7EE086A07EE903A66EE2F
:10ABC000866AB8EEC77AFDEEE66A27EE067AF8EEF8
:10ABD000E77A16EE903A67EE867ABDEEC77AFDEE1A
:10ABE000E77AE38617EE103A238717EE903A6387E9
:10ABF00004B010BD0020E086A06304B010BD8368DF
:10AC0000417C90F9100003F00103019302AB009323
:10AC100011220623F9F7A6FAC0E700BF10B50446D3
:10AC200000230068E386A3630279012A84B022D05E
:10AC3000022A1DD1836813F0010F02AA4FF0060308
:10AC400014BF03218321FFF7F7FC78B1BDF90A3067
:10AC5000BDF80810BDF80C205B4201EB410103EB8D
:10AC6000430302EB4202E1862387628704B010BDF2
:10AC7000184604B010BD8368417C90F9100003F0C1
:10AC80000103019302AB009303220623F9F76AFA4A
:10AC9000DBE700BF70B50446244894F9103003EB9D
:10ACA0008303154650F82300A3689A0782B00ED597
:10ACB000019065F077F9012301980022294665F09B
:10ACC000D9F8A3689B0717D5012002B070BD63694E
:10ACD00013B11A689B885383154B164A1B68566834
:10ACE0004FEAC30C144BA3FB0C3C4FEA9C1C53686B
:10ACF0009B1B9C45FBD2DBE70D4B0E491A680E4BA4
:10AD00004FF4FA7000FB02F2A3FB0232486892098A
:10AD10004B681B1A9A42FBD26369002BD4D01A6885
:10AD20009B881383012002B070BD00BF600000202B
:10AD3000E8290020001000E0D34D621010B503791F
:10AD4000012B82B08E460DD0022B08D18368DB0721
:10AD500058BF41F0800102B0BDE810409AE70020E2
:10AD600002B010BD14468268009402F00102417CDA
:10AD700090F9100001927246F9F7F4F902B010BD93
:10AD800070B504682379012B84B00D4615D0022BD1
:10AD900010D1A368E122DB074CBF11466121204698
:10ADA000FEF768FE30B12A46FF21204604B0BDE818
:10ADB0007040C3E7002004B070BDA26894F9100091
:10ADC000617C02F001020DF10F0601920096E12272
:10ADD0008DF80F20F9F7FAF9E4E700BF30B5046801
:10ADE0002379012B85B00D4616D0022B11D1A36813
:10ADF000DB074FF0C3024CBFE12161212046FEF783
:10AE000039FE30B12A46FF21204605B0BDE830406A
:10AE100094E7002005B030BDA26894F91000617C71
:10AE200002F0010201920DF10F020092C3228DF88F
:10AE30000F20E122F9F7CAF9E3E700BF70B5056812
:10AE40002B79012B84B004460E4619D0022B14D165
:10AE5000AB68DB074FF0F0024CBFE12161212846CF
:10AE6000FEF708FE48B1221DFF212846FFF766FFC6
:10AE700018B12379337004B070BD002004B070BDE8
:10AE8000AA6895F91000697C02F0010201920DF1A7
:10AE90000F020092F0228DF80F20E122F9F796F9C7
:10AEA000E0E700BF2DE9F0416B4A0468C16A6B4FCF
:10AEB000B7FBF1F182B006460F2389B290F8290062
:10AEC000FDF7C0FF00214388B7FBF3F70546776322
:10AED0002046FEF763FD0F224E212046FEF71CFEA2
:10AEE0004FF00F0805F080FC06460F4605F07CFC8D
:10AEF000831B61EB0701B3F57A7F71F10003F5D392
:10AF0000B8F10108EED16A794F2102F00F02204614
:10AF1000FEF702FE4FF00F0805F066FC06460F46EE
:10AF200005F062FC831B61EB0701B3F57A7F71F1D9
:10AF30000003F5D3B8F10108EED16A79502102F08F
:10AF40000F022046FEF7E8FD4FF00F0805F04CFC1D
:10AF500006460F4605F048FC831B61EB0701B3F57D
:10AF60007A7F71F10003F5D3B8F10108EED16A7967
:10AF700042EA02125221D2B22046FEF7CDFD0F273F
:10AF800005F032FC05460E4605F02EFC431B61EB36
:10AF90000602B3F57A7F72F10003F5D3013FEFD1DA
:10AFA000032214212046FEF7B7FD0F2705F01CFCF5
:10AFB00005460E4605F018FC431B61EB0602B3F58F
:10AFC0007A7F72F10003F5D3013FEFD13A46632156
:10AFD0002046FEF7A1FD642705F006FC05460E4657
:10AFE00005F002FC431B61EB0602B3F57A7F72F1B8
:10AFF0000003F5D3013FEFD1082265212046FEF77B
:10B000008BFD0DF1070264212046FFF797FE9DF8A6
:10B01000072022F0100242F06002642120468DF8E1
:10B020000720FEF779FD0F2705F0DEFB05460E46EB
:10B0300005F0DAFB431B61EB0602B3F57A7F72F190
:10B040000003F5D3013FEFD103212046FEF7A6FC14
:10B0500002B0BDE8F08100BFB86D070840420F00A4
:10B06000F0B583B015460DF107021C4606460F46A3
:10B07000FFF764FE9DF8072005EA0203A34201D111
:10B0800003B0F0BD22EA050222433946304603B040
:10B09000BDE8F040FEF740BD30B5092387B01A4641
:10B0A0000C210446FFF7DCFF282005F0CBFB01AAAA
:10B0B00008212046FFF742FE9DF904309DF8042048
:10B0C000002B01DA500603D40025284607B030BD16
:10B0D000122301AA10212046FFF704FB0546002891
:10B0E000F2D09DF805309DF804009DF807C01A09BC
:10B0F00042EA0011C209534A18BFA1F580511183D9
:10B100001B029DF8061003F4706343EA0100190561
:10B110009DF808309DF809104FEA031343EA0C33F9
:10B1200048BFA0F58050508343EA11101B03BDF8BF
:10B130000A304FEA01415BBA01F470219BB248BF6B
:10B14000A0F580100B430903BDF80C10D06148BF77
:10B15000A3F5801313624BBA99B21B04BDF80E30ED
:10B1600048BFA1F580315BBA1804918499B2BDF84B
:10B17000103048BFA1F580315BBAD18499B21B046D
:10B18000BDF8123048BFA1F580315BBA18041185B3
:10B1900099B2BDF8143048BFA1F580315BBA518532
:10B1A00099B21B0448BFA1F5803100239185204648
:10B1B00007220821FFF754FFA5220E212046FEF7A3
:10B1C000ABFC96220F212046FEF7A6FC022262214C
:10B1D0002046FEF7A1FC00220E212046FEF79CFC33
:10B1E00000220F212046FEF797FC022307220821A8
:10B1F0002046FFF735FF282005F024FB54231A468C
:10B2000020460621FFF72CFF0DF1030228212046DE
:10B21000FFF794FD9DF8033023F07F0343F05403C0
:10B220001A4620460721FFF71BFF0C231A4620462B
:10B230000921FFF715FF07231A4608212046FFF7CB
:10B240000FFF42E7C85E0020F0B5044683B00D460C
:10B250001746061D20680379012B18D0022B13D145
:10B260008368DB0732464FF0FF015CBF3246FF21A7
:10B27000FFF710FD30B115B12379DB07EAD40FB128
:10B2800023793B7003B0F0BD002003B0F0BD8268AD
:10B29000417C90F9100002F00102CDE90062FF222A
:10B2A000F8F760FFE6E700BF30B5044683B0051D40
:10B2B00020680379012B14D0022B0FD18368DB07A0
:10B2C0002A464FF0FF015CBF2A46FF21FFF7E2FC50
:10B2D00010B12379DB07EBD403B030BD002003B0FD
:10B2E00030BD8268417C90F9100002F00102CDE986
:10B2F0000052FF22F8F736FFEAE700BF30B50246FA
:10B30000044652F8040B0379012B83B00ED0022BB4
:10B3100009D1FF21FFF7BEFC18B12079C04300F02E
:10B32000010003B030BD002003B030BD8568417C12
:10B3300090F91000009205F001050195FF22F8F741
:10B3400011FFE9E730B5B42283B00446FF2100685D
:10B35000FEF7E2FB10B9002003B030BD206803798E
:10B36000012B04F1040514D0022BF4D18368DB0710
:10B370002A464FF0FF015CBF2A46FF21FFF78AFCF7
:10B380000028E8D02379DB07E6D520680379012B74
:10B39000EAD18268417C90F9100002F00102CDE907
:10B3A0000052FF22F8F7DEFEEAE700BF30B50A469A
:10B3B00083B00446A5210068FEF7AEFB10B900205B
:10B3C00003B030BD20680379012B04F1040514D0CB
:10B3D000022BF4D18368DB072A464FF0FF015CBFE4
:10B3E0002A46FF21FFF756FC0028E8D02379DB0727
:10B3F000E6D520680379012BEAD18268417C90F977
:10B40000100002F00102CDE90052FF22F8F7AAFE77
:10B41000EAE700BF70B582B0CDE900230446FFF72C
:10B4200091FF10B9002002B070BD20685522A521FF
:10B43000FEF772FB0028F5D0251D20682A46FF2163
:10B44000FFF77CFC0028EDD02379DB07F5D40DF164
:10B45000FF350DF1070615F8011F2046FFF7A6FF7F
:10B460000028DFD0B542F6D1DDE700BF002A37D093
:10B47000F0B5013A83B004464E1E51FA82F7051D1D
:10B4800016F8012F2068A521FEF746FB90B9002091
:10B4900003B0F0BD8268417C90F9100002F0010217
:10B4A000CDE90052FF22F8F75DFE0028EFD02379A6
:10B4B000DB0710D520680379012BEBD0022BE6D1F6
:10B4C0008368DB072A464FF0FF015CBF2A46FF2155
:10B4D000FFF7E0FBE9E7B742D2D1012003B0F0BDAE
:10B4E0000120704770B5962282B004460E4600686F
:10B4F000FF21FEF711FB10B9002002B070BD251D21
:10B5000020680379012B20D0022BF5D18368DB075B
:10B510002A464FF0FF015CBF2A46FF21FFF7BAFB26
:10B520000028E9D02379DB07EAD42468E122114618
:10B530002046FEF7F1FA0028DED03246FF212046F1
:10B5400002B0BDE87040FFF7F9BB8268417C90F91A
:10B55000100002F00102CDE90052FF22F8F702FECE
:10B56000DEE700BF002A4BD02DE9F041013A4F1C25
:10B5700082B004460E4657FA82F7051D20689622CF
:10B58000FF21FEF7C9FA98B9002002B0BDE8F081AA
:10B590008268417C90F9100002F00102CDE900526E
:10B5A000FF22F8F7DFFD0028EED02379DB0710D566
:10B5B00020680379012BEBD0022BE5D18368DB07F0
:10B5C0002A464FF0FF015CBF2A46FF21FFF762FBCE
:10B5D000E9E7D4F80080E12211464046FEF79CFAE4
:10B5E0000028D1D032464046FF21FFF7A7FB0028B4
:10B5F000CAD00136BE42C1D1012002B0BDE8F081FF
:10B600000120704770B505460B460446164655F8AE
:10B61000040B82B087211A46FEF77EFA2068037970
:10B62000012B18D0022B13D18368DB072A464FF079
:10B63000FF015CBF2A46FF21FFF72CFB30B12379C5
:10B64000DA07EBD416B1C3F34013337002B070BD08
:10B65000002002B070BD8268417C90F9100002F0B9
:10B660000102CDE90052FF22F8F77CFDE6E700BFBA
:10B6700070B5782182B00446164600680022FEF7B5
:10B680004BFA10B9002002B070BD251D2068037967
:10B69000012B14D0022BF5D18368DB072A464FF02B
:10B6A000FF015CBF2A46FF21FFF7F4FA0028E9D02A
:10B6B0002379DA07EAD45B09337002B070BD82687F
:10B6C000417C90F9100002F00102CDE90052FF2206
:10B6D000F8F748FDEAE700BF30B5CC2283B0044656
:10B6E000A5210068FEF718FA10B9002003B030BD9C
:10B6F00020680379012B04F1040514D0022BF4D146
:10B700008368DB072A464FF0FF015CBF2A46FF2112
:10B71000FFF7C0FA0028E8D02379DB07E6D52068D8
:10B720000379012BEAD18268417C90F9100002F084
:10B730000102CDE90052FF22F8F714FDEAE700BF4D
:10B7400030B5B42283B00446FF210068FEF7E4F967
:10B7500010B9002003B030BD251D20680379012BEE
:10B7600022D0022BF5D18368DB072A464FF0FF0178
:10B770005CBF2A46FF21FFF78DFA0028E9D0237924
:10B78000DA07EAD4CC212046FFF710FE0028E0D0EB
:10B7900002E02379DB07DDD520682A46FF21FFF789
:10B7A000CDFA0028F5D1D4E78268417C90F91000E9
:10B7B00002F00102CDE90052FF22F8F7D3FCDCE7EA
:10B7C0002DE9F04F89B00446CDE90623002004F1AD
:10B7D000040B0490029103905D462046049FFFF7FE
:10B7E000B1FD069BFE0003EBC70B20B90AE02379ED
:10B7F00013F0010A0DD020682A46FF21FFF79EFAB8
:10B800000028F4D1079B1A46049B137009B0BDE8C9
:10B81000F08F9B07F6D5F0212046FFF7C7FD0028E3
:10B82000F0D0069B083E334401270593D0463E46A0
:10B83000029B002B4AD0082E48D806F1FF3943FA64
:10B8400009F909F0010920684FEAC9127821FEF7C9
:10B8500063F90028D6D020680379012B47D0022B4A
:10B8600043D18368DB072A464FF0FF015CBF2A46BD
:10B87000FF21FFF70FFA0028C4D0237913F001024B
:10B88000E9D103F0600160294FEAD31C51D002993D
:10B8900019B1082E01D8E145B4D1BCF1000F3AD05E
:10B8A0001BF808303B430BF808307F00013617F0D7
:10B8B000FF07F6B2BCD108F101085FFA88F8B8F1C9
:10B8C000080F36D0029B0127002BB4D1049BD3B1C3
:10B8D000039BB34217D9059B13F808301F4214BFCE
:10B8E0004FF001094FF00009ADE700208AE78268B8
:10B8F000417C90F9100002F00102CDE90052FF22D4
:10B90000F8F730FCB7E7039BA3EB0609B9FA89F90E
:10B910004FEA591997E71BF8081021EA07010BF8BD
:10B920000810990941EA531313F0010F08BFB246FA
:10B93000BBE7402E06D8079B049A1B7893423FF63C
:10B940004CAF5FE79BF807C00BF1FF370BF1060B1D
:10B9500017F8011F082382EA010616F0010F4FEACB
:10B96000520218BF82F08C0203F1FF3318BFD2B22B
:10B9700013F0FF034FEA5101EDD1BB45E8D19445E7
:10B98000D9D1049B0133DBB20493BAF1000F3FF429
:10B9900039AFCDF80CA0CEE730B505682B79012B77
:10B9A00085B0044600F09280022B08D1AB68DB071B
:10B9B00002AA4CBF082188212846FFF76BF99DF8A1
:10B9C000083013F0100302D1184605B030BD2068CE
:10B9D000062302AA0021FEF785FE0028F5D09DF877
:10B9E00009209DF808109DF80A309FED3F6A120269
:10B9F00002EB01421344140248BF03F17F4307EEF8
:10BA0000903AF8EEE77A9DF80C109DF80B409DF8FF
:10BA10000D20364BC7EE866A090201EB04410A4449
:10BA2000090248BF02F17F4207EE902AB3F92C20A9
:10BA300007EE102AB3F92820F8EEE77A05EE102A6F
:10BA400087EE864AB3F92420B8EEC77AB8EEC55A15
:10BA5000D3ED087AA6EE875AF8EEE75A04EE902A5C
:10BA6000E6EE855AB3F92A20D3ED077A03EE902A41
:10BA7000F8EEE77AB3F92620E6EEA57A06EE102A6C
:10BA8000B3F91A20F8EEE44AF8EEE33A07EE102A8A
:10BA9000B8EEC66AB3F91820A6EEA36AE4EE247ADB
:10BAA00005EE902AB8EEC77A66EE846AF8EEE55A9B
:10BAB00027EE047AB6EE005AA5EE857AE6EE867A8F
:10BAC00083ED0D7AC3ED0C7A05B030BDAA68697CB0
:10BAD00095F9100002F00102019202AA00920822D8
:10BAE000F8F740FB6BE700BF00007848C85E002015
:10BAF00030B505682B7987B00022012B04468DF8FC
:10BB00000F2035D0022B12D1AB68DB070DF10F02ED
:10BB10004CBF2721A7212846FFF7BCF828B19DF884
:10BB20000F3013F0080305D1184607B030BD10469A
:10BB300007B030BD2068062304AA2821FEF7D2FDF5
:10BB400020B3BDF91030BDF91220002BB8BF03336C
:10BB50009B10E386BDF91430002AB8BF0332002BD6
:10BB6000B8BF033392109B102287638707B030BDA4
:10BB7000AA68697C95F9100002F0010201920DF1AA
:10BB80000F0200922722F8F7EDFAC7E7E086A063DC
:10BB900007B030BD30B5054600240068EC86AC63C4
:10BBA0000379012B87B02AD0022B0ED18368DB07E3
:10BBB0000DF10F024CBF21468021FFF76BF828B131
:10BBC0009DF80F4014F0080402D1204607B030BDA4
:10BBD0002868062304AA0121FEF784FD0028F5D079
:10BBE000BDF81430BDF81010BDF812205BBA49BA88
:10BBF00052BA5B42E9862A876B8707B030BD22467E
:10BC00008468417C90F9100004F0010401940DF166
:10BC10000F040094F8F7A6FAD1E700BF30B5044648
:10BC200000202568E086A0632B79012B87B027D000
:10BC3000022B10D1AB68DB070DF10F024CBF0621C0
:10BC400086212846FFF726F828B19DF80F3013F01B
:10BC5000040302D1184607B030BD2068062304AAA9
:10BC60000021FEF73FFD0028F5D0BDF81010BDF80B
:10BC70001220BDF81430E1862287638707B030BDFB
:10BC8000AA68697C95F9100002F0010201920DF199
:10BC90000F0200920622F8F765FAD5E710B503689F
:10BCA000DA6B82B0044612B1904740B123685B6BF7
:10BCB0001BB1214601A8984718B9FF23E38202B0BF
:10BCC00010BDBDF80630013B9BB2F7E7F0B585B07B
:10BCD000044618460D461646039364F063FA28445A
:10BCE0002768A073E673204600240094039B7C69B8
:10BCF00032462946A04705B0F0BD00BF38B504461E
:10BD00008B6801600D46984700230B4A226123751A
:10BD10002B6B13B1204698472075084B93F8E831F8
:10BD20001BB1237D23F0010323750023E38220460A
:10BD3000BDE83840B2E700BF0001FF00C06F00203F
:10BD40002DE9F041264ED6F8DC5184B09DB1B022E9
:10BD500080212846FDF7E0FE402280212846FDF79D
:10BD6000DBFE002280212846FDF7D6FE102280212E
:10BD70002846FDF7D1FE4FF480644FF000080DF126
:10BD80000F0795B12B79012B15D0022B0DD1AB6884
:10BD900013F001034FF000024FF04001284602BFAC
:10BDA0001A4640212846FDF765FE013CA4B29CB12D
:10BDB000D6F8DC51E5E7AA6895F91000697C8DF8A2
:10BDC0000F8002F00102013CCDE90072A4B24022D2
:10BDD000F8F7FCF9002CEBD104B0BDE8F08100BF0E
:10BDE000C06F00200B4B10B5D3F8DC418CB150383C
:10BDF000C2B280212046FDF78FFE0022802120461E
:10BE0000FDF78AFE20461022BDE810408021FDF794
:10BE100083BE10BDC06F0020F0B5204C204F2038ED
:10BE200000EB8000661DD7F8DC5185B00444064461
:10BE3000E5B12B792278012B1DD0022B0AD1AB68FA
:10BE400013F0010F4FF04001284604BF402128465F
:10BE5000FDF710FE0134B442EAD155B10022402171
:10BE6000284605B0BDE8F040FDF756BE0134B442A7
:10BE7000F0D105B0F0BD8DF80F20AA6895F910003B
:10BE8000697C02F0010201920DF10F020092402242
:10BE9000F8F79CF9D7F8DC51DCE700BF146E07080F
:10BEA000C06F00202DE9F041734ED6F8DC5184B00C
:10BEB000002D00F09680D42280212846FDF72CFE2C
:10BEC000802211462846FDF727FEA8228021284619
:10BED000FDF722FE3F2280212846FDF71DFED322DA
:10BEE00080212846FDF718FE002280212846FDF714
:10BEF00013FE402280212846FDF70EFE8D22802170
:10BF00002846FDF709FE142280212846FDF704FE8D
:10BF1000A12280212846FDF7FFFDC8228021284666
:10BF2000FDF7FAFDDA2280212846FDF7F5FD122201
:10BF300080212846FDF7F0FD812280212846FDF76B
:10BF4000EBFDCF2280212846FDF7E6FDD922802196
:10BF50002846FDF7E1FDF12280212846FDF7DCFDB2
:10BF6000DB2280212846FDF7D7FD4022802128468C
:10BF7000FDF7D2FDA42280212846FDF7CDFDA622A3
:10BF800080212846FDF7C8FDAF2280212846FDF715
:10BF9000C3FDA62280212846FDF7BEFDAE228021EA
:10BFA0002846FDF7B9FD202280212846FDF7B4FD83
:10BFB000002280212846FDF7AFFDB02280212846CF
:10BFC000FDF7AAFD402280212846FDF7A5FD0022AD
:10BFD00080212846FDF7A0FD102280212846FDF78C
:10BFE0009BFD4FF480644FF000080DF10F0755B32F
:10BFF0002B79012B2FD0022B0DD1AB6813F001034D
:10C000004FF000024FF04001284602BF1A4640217F
:10C010002846FDF72FFD013CA4B2002CE7D175B1F5
:10C02000812280212846FDF777FDC82280212846FD
:10C03000FDF772FDAF2280212846FDF76DFD01203E
:10C0400004B0BDE8F081013CA4B2002CE3D1012092
:10C0500004B0BDE8F081AA6895F91000697C8DF8FC
:10C060000F8002F00102CDE900724022F8F7AEF82D
:10C07000D6F8DC51CFE700BFC06F0020FAF74EBF03
:10C08000FAF74CBFFAF74ABFFAF748BFFAF746BFCC
:10C09000FAF744BF70B506461C48336803F13F43C6
:10C0A00003F57E039B0A82B0C05C0C46154661F026
:10C0B00069FDB2880092B2FA82F304F003028DF8AF
:10C0C0000420C4F3810230688DF80520C3F11F03FA
:10C0D000C4F3001264098DF80740C3F3CC0400EBED
:10C0E000840403F007038DF806209B00226A0F26C4
:10C0F0009D4006FA03F322EA03032362226A1543F2
:10C1000069462562F7F772F902B070BDD46A070874
:10C110002DE9F04FAE4CAF4DAC4283B050D21E462D
:10C1200002E00C34AC424BD294F805C08C45F8D1F7
:10C1300094F804C0844501D00028F2D194F807C0D7
:10C140009445EED12568002D3BD000236B60AB6099
:10C15000EB602B616B61AB61EB612C6022792A7122
:10C16000A779AF60217AE960012A33D0022A27D16A
:10C17000E07AFAF771FF94F90980A861A07A85F84E
:10C180001080FAF769FF6861F8B1934C08EB880AF0
:10C190004FEA880954F82A3004EB8A0AABB19AF8BE
:10C1A000123003B30E2200238671C271037209217B
:10C1B000FBF724F96B6923B11A689B88138300E0AD
:10C1C0000025284603B0BDE8F08F2846FDF7A2FB06
:10C1D0000025F6E7E07AFAF73FFF627AA37A6B74FC
:10C1E000A8612A74EDE79AF8080061F0CBFC9AF890
:10C1F00008104A09012301F01F01023A8B40032A6B
:10C2000008D8DFE802F0B6BCB00274494A6922EAF5
:10C2100003034B6109EB080304EB830308F1010BF3
:10C220005879FAF719FF5FFA8BFB824620B140F686
:10C230000A3380F808B0C38009EB080304EB8303DA
:10C24000D879FAF709FF034620B140F60A5280F880
:10C2500008B0C28009EB080204EB820201939079D6
:10C26000FAF7FAFE019B20B140F60A4280F808B0C6
:10C27000C28009EB080B04EB8B0B17F004079BF84B
:10C28000092000F08280BAF1000F0AD050464A21FE
:10C29000FFF700FF9BF80700FAF7DEFE9BF8092086
:10C2A000034643B118462A21FFF7F4FE09EB0803C1
:10C2B00004EB83035A7A019209EB080304EB83032E
:10C2C0009879FAF7C9FE18B1019A0A21FFF7E2FE40
:10C2D00009EB080B04EB8B0B9BF804A0BAF1000FE1
:10C2E00040F08A8009EB08033D4A54F8233093421A
:10C2F00000F0A6803B4A934200F0B8803A4A93424D
:10C3000000F0A980394A934200F08F80384A934266
:10C3100000F08080374A934200F0B3801A88002FE3
:10C3200002F441510CBF032200220A4342F4457239
:10C330001A809A8B22F400621204120C9A8307224C
:10C340001A821A8892B242F040021A80BAF1000FA3
:10C3500035D1C844686904EB88040123A37400281C
:10C360003FF425AF1EE71D490A6922EA03030B616A
:10C3700050E71A494A6A22EA03034B624AE717491F
:10C380000A6A22EA03030B6244E7BAF1000F0AD0FB
:10C3900050460A21FFF77EFE9BF80700FAF75CFE85
:10C3A0009BF809200346002B85D018460A21FFF789
:10C3B00071FE09EB080304EB83035A7A7BE75046CE
:10C3C000FAF74AFE0028C4D0036882881A83C0E7BF
:10C3D000246F0808987008086000002000380240A8
:10C3E0000030014000380040003C00400034014073
:10C3F00000500140005401405046FAF72DFE00283D
:10C400003FF470AF9BF809200921FFF743FE9BF82A
:10C4100004A067E702F56842516A41F48011516255
:10C42000516A21F48011516278E702F58232516A33
:10C4300041F400515162516A21F4005151626DE79B
:10C4400002F58432516A41F480515162516A21F4FB
:10C450008051516262E702F5FE32116A41F40041F7
:10C460001162116A21F40041116257E702F50032AE
:10C47000116A41F480411162116A21F48041116214
:10C480004CE702F56442516A41F400115162516A6D
:10C4900021F40011516241E72DE9F043002383B0FC
:10C4A0001A4634210120FFF733FEDFF87C9007465F
:10C4B000C9F8EC0160B34FF00508962604F094F932
:10C4C00004460D4604F090F9031B61EB0501B3F53A
:10C4D0007A7F71F10003F5D3013EEFD10DF1070230
:10C4E00031463846FEF72AFC044668B9B8F101081F
:10C4F000E3D199F8F031D9F8EC010C2B04BF0223F9
:10C50000C9F8F431FDF706FA204603B0BDE8F08320
:10C5100099F8F0310C2B01D00446F5E70123C9F856
:10C52000F4310446F0E700BFC06F0020F0B51023DF
:10C530008DB00546002228210220FFF7E9FD524C6C
:10C54000C4F8B800002800F091800221FDF726FA17
:10C5500002220021D4F8B800FDF7DEFA002384F8A7
:10C56000C03084F8BC5004F1C40304F284414FF09D
:10C57000202243F8042B8B42FBD1444E444F3568B4
:10C580003235D4F8B8000379012B71D0022B0FD1CA
:10C5900083683F4ADB074FF080015CBF3C4A802143
:10C5A000FEF778FB10B133689D42EAD8D4F8B800A2
:10C5B00010241123122113224FF0140E15271626D2
:10C5C00017258DF80C408DF80E30182419238DF89E
:10C5D00010108DF812201A211B224FF0010C8DF83B
:10C5E00014E08DF816708DF818608DF81A508DF8DB
:10C5F0001C408DF81E308DF820108DF822204FF051
:10C600001C0E1D271E261F254C24222303AA0021B1
:10C610008DF80DC08DF80FC08DF811C08DF813C0C6
:10C620008DF815C08DF817C08DF819C08DF81BC096
:10C630008DF81DC08DF81FC08DF821C08DF823C066
:10C640008DF824E08DF825C08DF826708DF827C070
:10C650008DF828608DF829C08DF82A508DF82BC0F0
:10C660008DF82CC08DF82D4063F054FC0DB0F0BD5A
:10C670008268417C90F9100002F00102CDE900725D
:10C680008022F7F76FFD8DE7C85E0020443500205B
:10C69000875F0020074B53F8203021B14BB11A6857
:10C6A0009B8853837047002BFCD01A689B881383A8
:10C6B000704770470C6B07082DE9F04F864CDFF888
:10C6C00020A294F8149294F8158294F8167283B00C
:10C6D000002604F5067501964FF0010EAB78E97857
:10C6E000C3F1FF039BB2002B48D10B460F468C468B
:10C6F0000A468846894601210191100240EA03401A
:10C70000172240EA0C0006EB020CACEB02030EFA17
:10C7100002F19BB2014204EB830314BF0221012109
:10C72000013AC3F89812531CEFD16C4B04351836FC
:10C73000AB42B6B2D2D14FF44073A4F8403F2023AD
:10C74000A4F8423F019B2BB184F8149284F815821F
:10C7500084F8167294F8443F6BB1D4F8480F50B186
:10C7600040F22A31F6F7F8FBD4F8480F03B0BDE8E1
:10C77000F04FF6F725BC03B0BDE8F08FB5F800C068
:10C78000C3F1FF03AAFB0CB001FB03F340091B122A
:10C790000A46052800F29B80DFE800F0886C5336DB
:10C7A0001C03AAFB0C077F09C7EB0717ACEB870735
:10C7B000BFB2C81AC7F13C0700FB07F7AAFB07077F
:10C7C0005FFA83F808EB57178946FFB20121BC4690
:10C7D000019192E7AAFB0C025209C2EB0212ACEBE8
:10C7E000820292B2A1EB030902FB09F9AAFB092913
:10C7F0005FFA83F808EB59198C465FFA89F90F46FE
:10C8000001214A46019178E7AAFB0C025209C2EBCA
:10C810000212ACEB82081FFA88F8CA1AC8F13C0869
:10C8200002FB08F8AAFB08285FFA83F909EB5818FD
:10C830008C465FFA88F80F4601211A46019143465B
:10C840005BE7AAFB0C025209C2EB0212ACEB8202BC
:10C8500092B2CF1A02FB07F7AAFB07275FFA83F908
:10C8600009EB57171A46FFB20B4688460121BC4612
:10C87000019142E7AAFB0C025209C2EB0212ACEB97
:10C8800082091FFA89F9CA1AC9F13C0902FB09F9A0
:10C89000AAFB0929DFB207EB59195FFA89F99C460F
:10C8A00088460B4601214A46019126E7A1EB030881
:10C8B0000CFB08F8DFB2AAFB080807EB58185FFA70
:10C8C00088F89C46012301938946434615E7434671
:10C8D0004A46BC4611E700BFC06F002058720020D6
:10C8E000898888882DE9F041284F00243B461D792E
:10C8F000212D03F1140304D001340F2CF7D1BDE82E
:10C90000F08104EB840007EB8000F6F709F9DFF80B
:10C9100088800646C8F8480F0028F0D02846FAF765
:10C920009BFBC8F84C0F58B1142202FB04744FF45F
:10C930000572C28000220272227A4A21FFF7AAFB06
:10C94000134A03213046F6F787F9D8F8480F00213B
:10C95000F6F7FEF90F49D8F8480F40F22A3260F096
:10C96000C3FD10B988F8440FC9E740F6A84209484A
:10C97000002169F0ACFFD8F8483F1B7C012288F801
:10C98000442F002BBBD1BDE8F04195E6F01000200C
:10C99000009F240058720020C06F0020084B93F8BD
:10C9A000BD204AB193F8BF3013F0400F14BF4FF4CD
:10C9B000F0704FF4C37070474FF4F070704700BFD1
:10C9C000C85E0020054B93F8BD0030B193F8BF302E
:10C9D00013F0400F0CBF0D2010207047C85E0020E0
:10C9E000104A70B5002302F570744FF40056A2F19E
:10C9F00046054FF0010E32F8020F03F01F01B0F5AB
:10CA0000005F4FEA531C0EFA01F103F1010305D058
:10CA100055F82C001680014345F82C10A242EAD1AB
:10CA200070BD00BF8A5F00204FF01E0C43EA022356
:10CA3000FF2A0CFB01011BB288BF43F00403B1F5D0
:10CA4000F07F07DA0C4A02EB41009BB2B0F8C4C099
:10CA50009C4500D170474FEA511C7C32A0F8C4308D
:10CA600001F01F0152F82C30012000FA01F10B43B4
:10CA700042F82C30704700BFC85E00204FF01E0CFB
:10CA80000CFB0101B1F5F07F01DB002070470B4882
:10CA900000EB4101B1F8C410080AC9B21080197046
:10CAA000490709D5118841F4807111801A7822F064
:10CAB000040201201A70704701207047C85E0020F0
:10CAC0002DE9F0471E2404FB010114787CB31D28D6
:10CAD0002DDC184E0FFA83FE06EB410CC1F1010567
:10CAE000483E012701E01D2B21DCB1F5F07F4EEA25
:10CAF000042405EB010311D2BCF800A001F01F08CB
:10CB0000A2454FEA511907FA08F807D0ACF80040DF
:10CB100056F8294044EA080446F8294012F8014F23
:10CB2000DBB20CF1020C03440131002CDBD1BDE877
:10CB3000F08700BF8C5F0020F0B5534CD4F8B8509C
:10CB400085B015B194F8BE300BB105B0F0BD01232E
:10CB500084F8BE302B79012B7BD0022B37D12846AD
:10CB60000DF10E028421FEF795F8D4F8B8502B7918
:10CB700094F8C020012B42F004027BD18DF80F20E5
:10CB8000AA6895F91000697C02F0010201920DF18A
:10CB90000F0200920422F7F719FB15E0022B0ED1C9
:10CBA000AB6813F0010F0DF10E024FF0840128461F
:10CBB00002BF0DF10E0284212846FEF76BF89DF8A6
:10CBC0000E3013F0040616D0D4F8B8502B79012B90
:10CBD000E4D1AA68697C95F9100002F00102019283
:10CBE0000DF10E0200928422F7F7BCFA9DF80E3088
:10CBF00013F00406E8D1254D254884F8C0303146AD
:10CC00003C2269F064FE05F570773146A5F1460EC9
:10CC1000012635F8023F1A0A22F0200203F004032D
:10CC200001F01F0013434FEA511C06FA00F001F116
:10CC3000010104D05EF82C3018434EF82C00BD42A0
:10CC4000E7D1FAF731F80028FBD184F8BE0005B02F
:10CC5000F0BDAA68697C95F9100002F0010201920A
:10CC60000DF10E0200928422F7F77CFAD4F8B85046
:10CC70002B797DE7022BAAD128460421FCF7FAFE86
:10CC8000D4F8B8502B79A2E7C85E00208A5F002054
:10CC9000445F002070B54A4DD5F8B84084B08CB3DD
:10CCA00095F8BC30012B40D0022B2DD1082294F9ED
:10CCB0001030444885F8BF2003EB8303042150F86B
:10CCC00023008DF80D2000238DF80C30A3688DF81B
:10CCD0000E109A078DF80F1040D5042303AA0021E7
:10CCE00063F0C8F8A3689B0721D537483C22FF2191
:10CCF00069F0EDFD95F8BD3023B9FFF71DFF012365
:10CD000085F8BD3004B070BD2379012B4AD0022BC9
:10CD100037D09DF80B3003F00503012B3ED0002BDC
:10CD200036D1D5F8B8400822C1E74822BFE7274BE3
:10CD300027491A68274B48684FF4FA7606FB02F237
:10CD4000A3FB023292094B681B1A9A42FBD2636919
:10CD5000002BCAD01A689B881383C6E7636913B196
:10CD60001A689B885383194B19491A68194B4E68E6
:10CD7000D200A3FB023292094B689B1B9A42FBD262
:10CD8000ABE70DF10B02A0212046FDF783FFC0E7C2
:10CD9000114A126840F2DC539A42B3D9D5F8B84030
:10CDA000482284E7A268617C94F9100002F0010235
:10CDB00001920DF10B020092A022F7F7D3F9A8E738
:10CDC000C85E002060000020445F0020E8290020A9
:10CDD000001000E0D34D62104435002070B5484C7F
:10CDE000D4F8B85084B095B194F8BF30180702D584
:10CDF00094F8BE306BB194F8BD3043B9FFF74AFFE9
:10CE000094F8BD30002B41D1002384F8BE3004B02B
:10CE100070BD94F8BD30012284F8BE20002BEDD007
:10CE20002B79012B35D0022BE8D10DF10E02802198
:10CE30002846FDF72FFF0028E0D094F8BF209DF88A
:10CE40000E309A42DAD194F8BC30002BD8D12D4B59
:10CE50002D4D1E68D5F86C35F31AB3F57A7FCFD90E
:10CE6000D4F8B8000379012B34D0022B04D10DF192
:10CE70000F02A021FDF70EFF9DF80F30590716D5C0
:10CE80000023C5F87035C5F86C65B9E7F9F70CFFF4
:10CE9000BAE7AA68697C95F9100002F001020192D4
:10CEA0000DF10E0200928022F7F75CF9C3E703F060
:10CEB0000503012B1CD0002BE5D194F8BF305B0695
:10CEC000E1D5D5F87035C3B1F31A642BDBD9FFF780
:10CED000E1FED8E78268417C90F9100002F001027F
:10CEE00001920DF10F020092A022F7F73BF9C3E780
:10CEF00094F8BF305A06E4D5C5E7C5F87065C2E7B7
:10CF0000C85E002044350020B091002000000000E1
:10CF1000437913F0010306D0D0E90731C268581AEB
:10CF2000531E184070471846704700BF437913F0EE
:10CF3000020307D0D0E9093200699B1A013820EAC0
:10CF400003007047184670474379024613F001000A
:10CF500018D010B4D168146AD369481E1B1B034053
:10CF60000CD053691B5D04F1010CD8B2BCFBF1F38A
:10CF700001FB13C15DF8044B1162704718465DF860
:10CF8000044B7047704700BF43799B070AD5436A3B
:10CF90008269D154436A02690133B3FBF2F102FBA7
:10CFA00011334362704700BF41717047D0E90920D7
:10CFB000101AB0FA80F04009704700BF014B1B689F
:10CFC0005B6818479C860020024B1B6808309B68F2
:10CFD000184700BF9C860020012070470120704741
:10CFE000012070470120704731B10C4BD3ED007A1E
:10CFF000F8EEE77AC1ED007A72B1094BDFED096A0C
:10D000001B68A3F5D543333B07EE903AF8EEE77A79
:10D0100087EEA67A82ED007A704700BF1097002055
:10D02000149700200000C84201207047012070477B
:10D03000704700BF044B03EBC00040F2FF739942FE
:10D04000A8BF19468180704798B50020184B194A2F
:10D050009B7982F86030032B1DD9191F022917D83C
:10D06000052B10B41AD0062B14BF4FF47A614FF47D
:10D070007A519FED0D7B00240F48104BD466B3FB13
:10D08000F1F382ED1C7B5DF8044B506693667047AC
:10D090000B4B536670470B4B536670474FF4FA5176
:10D0A000E7E700BFAFF300800000000000000000D1
:10D0B000D881002098B5002035D0000840420F00EC
:10D0C00031D0000879E50008034B03EB8000836F43
:10D0D0000BB19B681960704798B5002010B5D84C0B
:10D0E00004EB80039B6F0BB19B6819600F282ED84F
:10D0F000DFE810F02E0049006C009300B600D90064
:10D100000001230141015C017F01AA01CD01F00171
:10D1100017021000C900CB48A1F5DB511C3980FB78
:10D120000130C917C1EB600040F21472AD21FAF76B
:10D1300083FE94F8CD3000F0070203F01F0343EAAA
:10D140004213C0F3C70084F8CD3084F8CE0010BD80
:10D15000C900BC48A1F5DB511C3980FB0130C9175F
:10D16000C1EB600040F21472AD21FAF765FE94F84D
:10D17000BA3084F8B900C0F3022223F00703134346
:10D1800084F8BA3010BDC900AE48A1F5DB511C3996
:10D1900080FB0130C917C1EB600040F21472AD2171
:10D1A000FAF74AFE94F8BA2094F8BB3000F01F0159
:10D1B00002F00702C0F3451023F03F0342EAC10228
:10D1C000184384F8BA2084F8BB0010BDC9009D48FC
:10D1D000A1F5DB511C3980FB0130C917C1EB6000A0
:10D1E00040F21472AD21FAF727FE94F8BB2094F8B0
:10D1F000BD3000F0030102F03F0242EA811223F049
:10D200000103C0F380210B43C0F3870084F8BB20E7
:10D2100084F8BC0084F8BD3010BDC9008948A1F570
:10D22000DB511C3980FB0130C917C1EB600040F2B3
:10D230001472AD21FAF700FE94F8BD2094F8BE30C8
:10D2400000F07F0102F00102C0F3C31023F00F03CE
:10D2500042EA4102184384F8BD2084F8BE0010BDA4
:10D26000C9007848A1F5DB511C3980FB0130C91792
:10D27000C1EB600040F21472AD21FAF7DDFD94F8C5
:10D28000BE2094F8BF3000F00F0102F00F02C0F38F
:10D29000061023F07F0342EA0112184384F8BE20EF
:10D2A00084F8BF0010BDC9006648A1F5DB511C39E8
:10D2B00080FB0130C917C1EB600040F21472AD2150
:10D2C000FAF7BAFD94F8BF2094F8C13000F00101DC
:10D2D00002F07F0242EAC11223F00303C0F34121AE
:10D2E0000B43C0F3470084F8BF2084F8C00084F8E3
:10D2F000C13010BDC9005348A1F5DB511C3980FB7A
:10D300000130C917C1EB600040F21472AD21FAF789
:10D3100093FD94F8C12094F8C23000F03F0102F070
:10D320000302C0F3841023F01F0342EA8102184372
:10D3300084F8C12084F8C20010BDC9004148A1F59D
:10D34000DB511C3980FB0130C917C1EB600040F292
:10D350001472AD21FAF770FD94F8C23000F00702A4
:10D3600003F01F0343EA4213C0F3C70084F8C2303E
:10D3700084F8C30010BDC9003248A1F5DB511C3947
:10D3800080FB0130C917C1EB600040F21472AD217F
:10D39000FAF752FD94F8C53084F8C400C0F30222B5
:10D3A00023F00703134384F8C53010BDC900254896
:10D3B000A1F5DB511C3980FB0130C917C1EB6000BE
:10D3C00040F21472AD21FAF737FD94F8C52094F8B5
:10D3D000C63000F01F0102F00702C0F3451023F031
:10D3E0003F0342EAC102184384F8C52084F8C6000E
:10D3F00010BDC9001348A1F5DB511C3980FB013079
:10D40000C917C1EB600040F21472AD21FAF714FDA8
:10D4100094F8C62094F8C83000F0030102F03F02EF
:10D4200042EA811223F00103C0F380210B43C0F3D1
:10D43000870084F8C62084F8C70084F8C83010BD7F
:10D4400098B5002067666666C9004748A1F5DB51BC
:10D450001C3980FB0130C917C1EB600040F2147227
:10D46000AD21FAF7E9FC94F8C82094F8C93000F02F
:10D470007F0102F00102C0F3C31023F00F0342EA60
:10D480004102184384F8C82084F8C90010BDC900BF
:10D490003548A1F5DB511C3980FB0130C917C1EBC0
:10D4A000600040F21472AD21FAF7C6FC94F8C9206E
:10D4B00094F8CA3000F00F0102F00F02C0F306101A
:10D4C00023F07F0342EA0112184384F8C92084F84C
:10D4D000CA0010BDC9002448A1F5DB511C3980FBEE
:10D4E0000130C917C1EB600040F21472AD21FAF7A8
:10D4F000A3FC94F8CA2094F8CC3000F0010102F0AB
:10D500007F0242EAC11223F00303C0F341210B431F
:10D51000C0F3470084F8CA2084F8CB0084F8CC30EC
:10D5200010BDC9001048A1F5DB511C3980FB01304A
:10D53000C917C1EB600040F21472AD21FAF77CFC10
:10D5400094F8CC2094F8CD3000F03F0102F00302B3
:10D55000C0F3841023F01F0342EA8102184384F8C9
:10D56000CC2084F8CD0010BD67666666084AD2F804
:10D57000D4305BB140B19968B2F8D820054BB3FB09
:10D58000F2F35B100B6070479B681860704700BF38
:10D5900098B5002040420F00F0B54D4E96F8DA30B5
:10D5A00083B03BB196F8DB50012D04465ED0022DCE
:10D5B0003ED00DB103B0F0BD012280210068454F7F
:10D5C000FCF7AAFA01223870FF212068FCF7A4FAC0
:10D5D0002A46387029462068FCF79EFA96F8DC2027
:10D5E000387091212068FCF797FA2946387001229B
:10D5F0002068FCF791FA2A463870FF212068FCF772
:10D600008BFA2A46387080212068FCF785FA294673
:10D610000346012220683B70FCF77EFA2E4A3870E0
:10D620001268C6F8E020012386F8DB3003B0F0BDB5
:10D630000068284F01AA1321FDF780FB9DF80430F4
:10D6400038705B0725D1D6F8E430002BB2D0224ADF
:10D65000D6F8E010126892B2521A9342AAD24FF052
:10D66000FF3200237A6086F8DB30A3E701AA006866
:10D67000184F0021FDF762FB9DF804303870DA077F
:10D68000E1D4154A02231268C6F8E02086F8DB30A0
:10D6900090E720682B4601AA1E21FDF723F8BDF86C
:10D6A000043002460B2120683A7001225CBAFCF774
:10D6B00033FA0A4B3870A4B2A3FB0434E408012205
:10D6C00000237C6086F8E82086F8DB3072E700BF34
:10D6D00098B500208C14002044350020CDCCCCCC53
:10D6E0000C4A13787BB10C4B93F8DA1059B193F8CC
:10D6F000E81059B150680022FA2883F8E820A8BF42
:10D700004FF0FF3070476FF0010070476FF002007C
:10D71000704700BF8C14002098B500202DE9F0411F
:10D72000114C04F1EC0884F8ED1017460025022393
:10D730004246FF21064684F8EC50FCF75BFF80B1BF
:10D74000424630460223FF21FCF7CCFF48B194F853
:10D75000EC2094F8ED3003EB022328463B80BDE833
:10D76000F0816FF00C00FAE798B500200B4B93F8AE
:10D77000EC2182B193F8ED2152B109498868002269
:10D78000B0F5967F83F8ED21A8BF4FF0FF307047CA
:10D790006FF0020070476FF00100704798B50020ED
:10D7A0008C140020014B1B685B6818479086002092
:10D7B000014B1B689B68184790860020014B1B6833
:10D7C000DB68184790860020014BD868704700BF7F
:10D7D0008C140020044B93F8EE3113B1034B1869FD
:10D7E00070476FF00100704798B500208C1400203E
:10D7F000437A5A1C0344D2B242729972037A93421A
:10D8000000D97047002AFCD010B5044604F10A0183
:10D81000D0E9003098470023637210BD08B5284B4B
:10D82000284ED3F8F051B0682CF0A0FA28462CF01E
:10D830009DFAB06841798B073BD500210846FEF779
:10D8400029FF00210120FEF725FF1F4CB068036867
:10D850005B689847C8B92B6828465B6898470028DA
:10D86000F4D0D4F89C202B68B4F8A010DB68518366
:10D87000284698470146B068026813689847D4F86C
:10D880009C30B4F8A0201A83E0E7B068D4F8A82050
:10D890000368B4F8AC10DB68518398472B680146E5
:10D8A0001B6828469847D4F8A830B4F8AC201A83EF
:10D8B000D1E7036841F002019B699847BDE700BFCB
:10D8C00098B5002028830020F02A0020F0B541F010
:10D8D000010285B000212A4F2A4D2B4E0446FCF749
:10D8E0001BF93B68C6F8E030287016E0A368DB0738
:10D8F0000DF10F024FF0130120465EBF0DF10F0234
:10D9000093212046FDF7C6F99DF80F30287013F0DB
:10D9100007030ED1D6F8E4204ABB2379012B18D097
:10D92000022BE3D09DF80F30002013F0070328707E
:10D93000F0D001220B212046FCF7EEF8002203462E
:10D94000114620462B70FCF7E7F82870012005B03F
:10D95000F0BDA268617C94F9100002F0010201920E
:10D960000DF10F0200921322F6F7FCFBCCE73968A9
:10D97000D6F8E00089B2091A8A42CED21846E6E704
:10D98000443500208C14002098B500202DE9F04F7C
:10D99000794B9D79C7B005B1FEE7774AD779012366
:10D9A000937107F0F7071368D77103931B79012B65
:10D9B00004460E4600F09E80022B40F099800398AA
:10D9C000836813F0010118BF29463A46FCF752F864
:10D9D000694B1B68039305ADFF2C4FF009036C7076
:10D9E00088BFA4082B708CBF04F0C0084FF000085B
:10D9F000022300204FF00A0B0DF1150A4FF00B091E
:10DA000012E0BEF5827F05F803B016F800C00AF8F0
:10DA1000032015D80130362805F8049001F10601DD
:10DA200005F807C0734612D09C1C48EA0002B4F502
:10DA3000827F03F1040E1946D2B203F10307E0D945
:10DA400001306FF0004E36284C497346ECD1B1F5E9
:10DA5000827F00F28D8008210DF1150205F80E106D
:10DA6000A021D1540233039C454994F9102002EBC4
:10DA7000820251F82200A268920766D52A46002148
:10DA800062F0F8F9039B9B689B0746D53A4B3D4DE6
:10DA900018680379012B0DF1130418D0022B08D15B
:10DAA0002246A021FDF7F6F818B1237813F02003E1
:10DAB00019D0D5F8A830B5F8AC2059690A4214BF7E
:10DAC0005A831A832C4B18680379012BE6D182689C
:10DAD000417C90F9100002F00102CDE90042A02241
:10DAE000F6F740FBE0E7244A937147B0BDE8F08FBA
:10DAF00005AD71E7039881682A4601F001050146EA
:10DB000090F91000497C019505AD2F700095F6F74E
:10DB10005DFB194B1B6803935EE71B4B1B491A689F
:10DB20001B4B48684FF4FA7404FB02F2A3FB023269
:10DB300092094B681B1A9A42FBD2039B5B69002B2C
:10DB4000A4D01A689B881383A0E7626912B1116898
:10DB500092884A830C4A0D4C11680D4A6668C900C8
:10DB6000A2FB012189096268921B9142FBD285E7E1
:10DB70006FF0004377E700BF805F00200100008066
:10DB800060000020F02A0020E8290020001000E0BA
:10DB9000D34D621038B583681C686379DB0748D5BC
:10DBA000A37994F85C2203F001010D461ABB94F8A6
:10DBB0005F32012B3ED0002B40D194F85E3294F8B6
:10DBC0005DC263450DD2B4F866224FF0010E0EFA25
:10DBD00003F001330243D8B2604592B2F7D3A4F800
:10DBE0006622012384F85F32E06B85EA0301BDE819
:10DBF00038405FF0CDBDE06B43681A68D36AC3F369
:10DC00004E03536294F86D32012B07D094F86132C1
:10DC100023B1B4F868320133A4F8683285F0010109
:10DC20005FF0B6FD00224FF08073A4F86622C4F8BE
:10DC30005C3238BD94F85D3284F85E32002384F89B
:10DC40005F32E06BBDE838405FF0A2BD30B5032025
:10DC500083B00D461446FBF727FE01909DB107EEF9
:10DC6000900A9FED0B7AF8EE677AF0EE006A67EEA5
:10DC7000877AB8EE047AA7EEA67ADFED067A67EE29
:10DC8000277AC5ED007A0CB1034B236003B030BD99
:10DC90006740533A00007A443313904300B500685C
:10DCA0000379012B85B00DD0022B07D1012303AAE4
:10DCB000FF21FCF7C1FC05B05DF804FB002005B0B6
:10DCC0005DF804FB8268417C90F9100002F00102CB
:10DCD000019203AA0092FF22F6F744FA05B05DF81C
:10DCE00004FB00BF30B5044600680379012B85B002
:10DCF00029D0022B1ED1826812F0010F18BF5121CA
:10DD000003AA08BFD121FCF797FC98B1BDF80C30ED
:10DD1000194A5BBA9BB2D360D368B3F5C87F0EDCF7
:10DD20001649174AD1F8F43115683233AB4218D38B
:10DD300005B030BD104B6FF00102DA60F0E74FF034
:10DD4000FF33D360ECE78368417C90F9100003F067
:10DD50000103019303AB009351220223F6F702FA69
:10DD6000D3E701F5FC72C1F8F4512068002351217A
:10DD7000FCF740FC05B030BD8C14002098B50020A5
:10DD80004435002000B500680379012B85B008D028
:10DD9000022B2FD0204B002283F8EE2105B05DF836
:10DDA00004FB8368417C90F9100003F0010303AA8F
:10DDB000CDE9002302230022F6F7D4F9164B83F8AD
:10DDC000EE010028EAD0BDF80C305BBA9BB2B3F587
:10DDD000FA6F1AD21149124AA1FB0313DB0807EEAE
:10DDE000903AF8EEE77AFDEEE77AC2ED047A05B0F4
:10DDF0005DF804FB826812F0010F18BF002103AA2E
:10DE000008BF8021FCF718FCD8E7054B4FF0FF3224
:10DE10001A6105B05DF804FB98B50020CDCCCCCCE0
:10DE20008C14002010B500680379012B84B00C46D7
:10DE30001DD0022B18D1826812F0010F14BF0021EF
:10DE4000802103AAFCF7F8FB60B15CB19DF80D30AE
:10DE50009DF90C20DB0903EB830302EB820203EB49
:10DE60004203238004B010BD002004B010BD8368BD
:10DE7000417C90F9100003F00103019303AB009380
:10DE800000220223F6F76EF90028DED1EAE700BF90
:10DE900070B50668F56982B00446002D50D00023A5
:10DEA0002B7004230DEB03023046FF21FCF71AFC14
:10DEB00010B9002002B070BD206804236A46FF211B
:10DEC000FCF710FC0028F4D09DF804108A09023AEF
:10DED000012AEED99DF805309DF800409DF80120FB
:10DEE00003EB012302EB0422C3F30D03C2F30D0283
:10DEF000991A0029B8BF4942FF29DADC9DF802408F
:10DF00009DF803109DF8066001EB04214C119DF86B
:10DF1000071001EB0621C4EB5116002EB8BF764264
:10DF2000FF2E4FEA6111C4DC134421445B104910F9
:10DF3000C5F805300123C5F801102B7002B070BD83
:10DF400009211420FAF72AFFF06105462668A6E7A2
:10DF500070B50568E8690C461646A0B3D0F80130E4
:10DF6000CCB1D0F805209FED1B7ADFED1B5ADFED19
:10DF70001B6A07EE902AF8EE677AB7EE006A77EE32
:10DF8000C77A77EEA77A87EEA57A77EE467A67EEBC
:10DF9000E67AC4ED007AAEB107EE903A9FED107AC2
:10DFA000DFED106A9FED106AF8EEE77A67EE877A88
:10DFB00087EEA67ADFED0D6A77EE467A77EEA67ADF
:10DFC000C6ED007A70BD09211420FAF7E7FEE8617A
:10DFD000C4E700BF9AC9CC449AC94C460E76D745CF
:10DFE0000000484300E0FF44000048423393884368
:10DFF000F8B52DED048B4B4B1B7E022B0E461746BE
:10E0000018D09FED490A7EB1DFED487ADFED486A0E
:10E010009FED487A20EE000A20EE270AC0EE267A0D
:10E0200077EE877AC6ED007A0FB1434B3B60BDECCB
:10E03000048BF8BD414C94F8083243B1404B1B6847
:10E040009A071ED4D4F8043293ED350ADBE73C4B33
:10E050001B689B07F6D53B4BB3F9222001EE102A33
:10E06000B3F92020B3F91E3000EE902A00EE103AEA
:10E07000B8EEC11AF8EEE00AB8EEC00AFAF7C8FC2A
:10E08000C1E7D4ED7E8A94ED7F9A2F4DF0EE680AB9
:10E09000B0EE490AF9F7EAFDB5EEC00AF1EE10FA62
:10E0A00048BFDFED2A7AF0EE490AB0EE408A48BF59
:10E0B00030EE278AB0EE680AFAF7A2FCDFED246A98
:10E0C0009FED247AD5F8E80328EE268AF0EE408A00
:10E0D000C8EE077AFCEEE77A17EE903A9BB21B1A6D
:10E0E00007EE903AF8EEE77A87EEA60A20EE070AE6
:10E0F000F9F7E0FBD5EDFF7A287CD4ED800AE0EE5D
:10E10000687A05F5747305F56E75002818BF1D460D
:10E11000B0EE670AD5ED057A70EEA70AFAF770FC43
:10E1200071E700BF3084002000000000CDCC9C3F90
:10E1300000409C4682E6C5473313904398B50020C3
:10E1400008000010D089002004A50020DB0FC94082
:10E150000000C84235FA8E3C2DE9F04F87B0994651
:10E160009DF84430BDF840B0019307468A4690467A
:10E17000F4F7D6FC0446002800F09480594E96F837
:10E1800009520A2D00F29E805C2303FB05630022E6
:10E19000C3F80C2283F810223A791309691C013B59
:10E1A000C9B2032B86F80912029102F00F0C42D873
:10E1B0004D4A039332F8130040FA0CF2D3073AD5D4
:10E1C000012202FA0CF2013A104062F045FE474A81
:10E1D000039B0299D35C464A184400EB400002EBD3
:10E1E00080034FF0020C1972019983F806A083F89E
:10E1F00007C000FA0CFA002958D15AF802103D481D
:10E20000019301F13F4101F57E01890A405C5FF015
:10E21000B9FC019B364A998804914FF0011152F8DC
:10E220000A00059104A9F5F7E1F8314A019B5AF873
:10E2300002209B8853835C2707FB056742464946BB
:10E240002046C7F80C42F4F707FD5946D7F80C02F0
:10E25000F4F77EFDD7F80C3259680B68B3F8442008
:10E260006FEA42426FEA524292B2A3F844201A88FF
:10E2700092B242F001021A804A79032A29D8DFE8D3
:10E2800002F01B1D1F02403305EB45005C22C5EB6D
:10E29000C000194C02FB05650022C5F8143204EBDE
:10E2A00080041A60204607B0BDE8F08F3A7A6146D4
:10E2B0001846FDF7EFFEBEE73433E5E73833E3E712
:10E2C0003C33E1E70D4A00210420FAF775FC0024F5
:10E2D000E8E75C22002302FB0565C5F814321B60E9
:10E2E000FFDE00BF98B500201C6B0708246B0708F1
:10E2F000F02A0020D46A0708A4B700201C020808EE
:10E3000030B503682F4C2DED028BA34283B0F0EEA5
:10E31000408AB0EE608A13D004F58064A3420FD027
:10E3200004F57054A3420BD004F58064A34207D0D7
:10E3300004F58064A34203D0234B1C68640801E009
:10E34000214B1C680192B4FBF1F202F57F420023DD
:10E35000FF32120C0093B4FBF2F4B4FBF1F5224649
:10E36000ABB20221FFF7F8FED0B1B5EE408AF1EE74
:10E3700010FA19D0DFED150A07EE904A68EE200A70
:10E38000F8EE677A60EEA70A9FED117AC0ED040AF5
:10E3900027EE607A0123A8EEA77A037180ED037A55
:10E3A00003B0BDEC028B30BD07EE905ADFED070ADB
:10E3B000B8EE677A07EE904A67EE200AF8EE677AC1
:10E3C000E2E700BF00000140EC0E00206F12833A2C
:10E3D00000007A442DE9F04F85B09A469DF8383018
:10E3E000009381468B469046F4F79AFB044600283A
:10E3F00000F08980584E96F809720A2F7ED85C2367
:10E4000003FB07630022C3F80C2283F8102299F85B
:10E41000042013097D1C013BEDB2032B86F8095241
:10E4200002F00F0139D84D4A019332F8130040FA37
:10E4300001F2D30731D501228A40013A104062F03F
:10E440000BFD474A019BD35C464A184400EB400051
:10E4500002EB800340F20321D98000991D728500F0
:10E46000002944D1A9584048009301F13F4101F5EA
:10E470007E01890A405C5FF085FB009B394A9988E0
:10E4800002914FF001115059039102A9F4F7AEFF28
:10E49000344A009BAA589B8853835C2505FB07657B
:10E4A000324AC5F80C42B2FBF8F1204689B2F4F7C3
:10E4B000D3FB5146D5F80C02F4F74AFCD5F80C32E0
:10E4C00059680B68B3F844206FEA42426FEA52423F
:10E4D00092B2A3F844201A8892B242F001021A8044
:10E4E0004A79032A2FD8DFE802F0282A2C1299F85B
:10E4F000082018460221FDF7CDFDCEE71C4A002179
:10E500000420FAF759FB002005B0BDE8F08F403336
:10E510005C2000FB07600021C0F81432154A196026
:10E5200007EB470306EB8B06C7EBC30702EB870736
:10E530000120B76705B0BDE8F08F3433E8E7383322
:10E54000E6E73C33E4E75C22002302FB0766C6F8FB
:10E5500014321B60FFDE00BF98B500201C6B07085B
:10E56000246B0708F02A0020D46A070840420F00F5
:10E570001C020808A4B7002010B50B4B82B053F85A
:10E58000304001916CB107EE901A94ED047A94ED4D
:10E59000030AF8EEE77AA7EE870A65F067F8A36842
:10E5A000186002B010BD00BF98B500202DE9F043FF
:10E5B000364E96F8603083B00D46062B61D8DFE802
:10E5C00003F0284F394A04040400052B4DD030498C
:10E5D000304C062B08BF21464FF000080192CDF8C1
:10E5E00000800A4614230221FFF7B6FD07460028E3
:10E5F00045D08146122259F8140B49465EF074FF4B
:10E600000446A0BB012446F83570204603B0BDE89F
:10E61000F083DFED210A4FF4C871B0EE600AFFF716
:10E620006FFE041E18BF012446F83500204603B0D3
:10E63000BDE8F083DFED190A9FED190A4FF4FA6186
:10E64000FFF75EFE041E18BF012446F83500204681
:10E6500003B0BDE8F083134BDFED130A9988DCE7C4
:10E66000DFED120A4FF47A71D7E71149B4E741465A
:10E670004846482268F02BF901233B71C3E7044662
:10E68000C1E7002446F83540BFE700BF98B5002039
:10E69000C0C62D00001BB7006F12833AACC5A73768
:10E6A000ACC5A736D8810020000000006F120339E6
:10E6B000808D5B0010B50B4C94F80836012B05D00B
:10E6C000022B09D0084BC4F80C3610BD60F016FBC5
:10E6D000064BC4F80C3610BD60F010FB044BC4F8B8
:10E6E0000C3610BD98B50020C9D0000865D90208C5
:10E6F000DDD0000810B5174C84F8ED10017984F8CE
:10E70000EE2001294FF0000282B084F8EC2012D0F4
:10E7100002290CD1032304F1EC02FF21FBF714FFC3
:10E72000002814BF00206FF00C0002B010BD6FF085
:10E730000C0002B010BD8268417C90F91000EC34EE
:10E7400002F00102CDE900420323FF22F5F73EFD6E
:10E75000E6E700BF98B5002000680379012B0BD0D5
:10E76000022B08D183680F4A13F0010316D000234F
:10E770005121FBF7E9BE704700B58368094A417C27
:10E7800090F9100083B003F00103CDE900230023CA
:10E790005122F5F71BFD03B05DF804FBD121FBF717
:10E7A000D3BE00BF90B7002030B5184D95F8EC31BE
:10E7B00083B00BB903B030BD04460DF1050100680C
:10E7C00060F0B8FC9DF8053073B901212068104A4B
:10E7D00085F8EE104FF406440323FF21A5F8EC4022
:10E7E000FBF708FF03B030BD0DF10602962120684B
:10E7F000FEF794FF074ABDF806300749A2FB032342
:10E80000DB0801228B6085F8ED21DEE798B500205A
:10E8100084B60020CDCCCCCC8C1400202DE9F04166
:10E82000DFF8608004460F4616460025204620216A
:10E8300068F064F80446E0B103461C4613F8010B87
:10E840002028FAD02046FAF733FF40F634024FF47E
:10E850006171F9F7F1FAA0F5617088FB0023C01728
:10E86000C0EBE300302804D84DB178703378013321
:10E8700033700DB90125D9E72046BDE8F081387025
:10E88000F4E700BF1F85EB512DE9F043954E346846
:10E8900085B0002C66D096F80690B9F1000F00D034
:10E8A000FEE796F807C001230CF0F70C86F807C0C6
:10E8B000B3712379012B05460F4600F0CE80022B61
:10E8C00000F08D80B0F5807F0DF10F0800F0EB8037
:10E8D000012B00F0D780022B06D1204650220821C0
:10E8E000FBF7C8F8346823797F4D012B19D0022B30
:10E8F0000AD142462046A021FCF7CCF920B19DF870
:10E900000F4014F020044BD0D5F8A830B5F8AC2057
:10E91000596934680A4214BF5A831A832379012B38
:10E92000E5D1A268617C94F9100002F00102CDE902
:10E930000082A022F5F716FCE0E7B9F1000F0FD135
:10E94000F479356804F0F704F4712B79012B00F0A9
:10E95000B580022B04D1224649462846FBF78AF8A7
:10E960000023B37105B0BDE8F083022B15D16246D8
:10E970000A212846FBF77EF830680379012B07EB64
:10E98000040226D18568417C90F9100005F001054C
:10E99000CDE90025C022F5F7E5FB0134362CCCD0BB
:10E9A00035682B79012B5FFA84FCDED1AA6895F9D2
:10E9B0001000697C8DF80FC002F00102CDE90082E1
:10E9C0000A22F5F703FC30680379012B07EB0402F8
:10E9D000D8D0022BE1D1C021FCF75CF9DDE7494634
:10E9E00020466246FBF746F83468237981460DF1EC
:10E9F0000F08012BEAB227D1A16894F9100001F0A9
:10EA0000010C617C8DF80F20CDF804C0CDF800809A
:10EA10000922F5F7DBFB34682379B5F5807F7FF4B5
:10EA200057AF012B3FD1A26894F91000617C02F02E
:10EA30000102CDE9008240228DF80F200A22F5F76D
:10EA4000C5FB3468237943E7022B45D120460921D1
:10EA5000FBF710F834682379DFE7A16894F9100018
:10EA600001F0010E0DF10F08617CCDF804E04A467B
:10EA7000CDF800808DF80FC0F5F7A8FB346881460B
:10EA80002379B6E7A26894F91000617C02F00102D4
:10EA9000CDE9008250228DF80F200822F5F796FB71
:10EAA0003468237920E7022B7FF41EAF20464022F2
:10EAB0000A21FAF7DFFF3468237909E7A96895F995
:10EAC000100001F001074A46697C8DF80F40CDE93E
:10EAD0000087F5F77BFB43E7B5F5807F7FF4FBAE5E
:10EAE0009FE700BF805F0020F02A0020024B1B68D8
:10EAF0000BB1FEF74BBF7047805F002010B58379E4
:10EB0000C26B13F0010F0446406B20D013F0200FAE
:10EB1000526814BF0221422120B1127AFDF7BAFADD
:10EB2000E36B5A68012384F86032A4F85C325079B0
:10EB30000B4C1168205C0A8C83409BB292B222EA93
:10EB400003020A840A8C92B213430B8410BD13F0A3
:10EB5000200F526814BF022122210028DDD1E1E7F5
:10EB60008075070838B583681C686379990745D4B0
:10EB7000D90700D438BD94F85C32002BFAD194F850
:10EB80005D320133DBB2092B84F85D3200F0AC80DA
:10EB90000A2BEFD194F85F52002D00F0C480B4F836
:10EBA0006602820500F0010302D4002B40F0C4800D
:10EBB000B4F86A320133A4F86A3201239D42A4F802
:10EBC0005C32D7D1A179E06B002384F85F3201F089
:10EBD00001015EF0DDFDE36B76485B685A791968E8
:10EBE000835C0A8C05FA03F39BB292B222EA030219
:10EBF0000A840A8C92B213430B8438BD94F86112D4
:10EC0000002967D1D4E90902904200F09E80501C8F
:10EC1000A569A062AA5C25695200A84234BF0546D6
:10EC20000D4694F86002A56242F400720A254FF086
:10EC3000010CA4F8642284F8625284F861C20028AE
:10EC400050D0A07905071CD410F0400590D00921C0
:10EC50004FEA520CC00702F0010248BF82F00102E5
:10EC6000A4F864C2002A57D1A26B12B1106892882E
:10EC7000428384F86212002D3FF47AAF00292DD030
:10EC800076E7E36B4B485D686B792A68C35C606B21
:10EC90000CFA03FC138C9BB223EA0C0CA2F820C0E4
:10ECA000138C9BB2138410B12A7AFDF7F3F9236C0D
:10ECB000A06B002284F86022002B64D020B15B6836
:10ECC00001211A7AFDF7E6F9A37913F0400F637971
:10ECD0003FF44EAF94F9621200294CD1002284F81F
:10ECE000612245E7A079AFE794F85F32002B7FF40B
:10ECF00041AF94F85E32082B3FF63CAFB4F8662281
:10ED0000012000FA03F101330A43D9B2082992B273
:10ED1000F7D9A4F8662238BDA26B002AA9D01068E2
:10ED200092880283A5E7B4F8663243F001009B05A0
:10ED3000A4F866023FF53CAFE36A40083BB3216BA1
:10ED4000C0B2984794F85F5237E794F860120029F0
:10ED50007FF40EAFA27912077FF50AAF236CA06B88
:10ED600023B318B15B681A7AFDF794F92046FFF7D0
:10ED7000C5FE6379FCE6A079B4F86422013949B292
:10ED800000F0400564E70121F8F738FB9CE7E369F0
:10ED90006269C0B2D054E369E26894F85F5201330B
:10EDA000B3FBF2F102FB1133E36106E71946F8F712
:10EDB00025FBDBE78075070838B54368344A1B68D4
:10EDC000934204462BD002F58062934227D002F58D
:10EDD0007052934223D002F5806293421FD002F515
:10EDE000806293421BD02B4B1A6852081346B3FB28
:10EDF000F1FCBCF5803F15D21FFA8CF12046F3F7E9
:10EE00002BFF23681A6853790BBB937973B9636836
:10EE10001A6813889BB243F00103138038BD1D4B61
:10EE20001A68E3E7012BE4D95B08E0E75AB2002A4D
:10EE30001FDB19480121851803F01F03520901FA4D
:10EE400003F3302185F8001340F82230DFE759B290
:10EE5000002915DB104D012005EB010C03F01F0309
:10EE6000490900FA03F330208CF8000345F82130FB
:10EE7000CBE70A4A03F00F031A4430231376C6E7A0
:10EE8000064903F00F03194430230B76BDE700BF9A
:10EE900000000140EC0E002000E100E0FCEC00E08E
:10EEA0000346C06B996087E7002ABCBF80185242B6
:10EEB000002B30B53BDB5D180028B7BF121A841851
:10EEC00014460020A4F11D0C0029BCBF2B460021D4
:10EED000BCF1000FC8BFA2EB0C04A5F10F02C8BF24
:10EEE0002418002AC4BF9B1A5D1884421EDBC1F19E
:10EEF000010C114AC1EB0113AC4400EB4303CCEB12
:10EF00000C1C01344FEA4C0C02EB43024FF0200E74
:10EF10008D42A8BF002304DB22F813E01E339C457A
:10EF2000FAD10130A04202F10202F1D130BD5C18E9
:10EF30000D465B422146BFE78C5F00201B4B1C48FF
:10EF4000196C1C4A10B441F0805101241964046208
:10EF50005321FF24CA205462506251625B6FDB0070
:10EF600085B013D40023144902930291029A1348E6
:10EF700004320292029A136003930391039B03935A
:10EF8000039B186005B05DF8044B70470A4B0022E4
:10EF900001920193019B0193019A084B12689A42D6
:10EFA000E0D105B05DF8044B704700BF0038024067
:10EFB00000000E42002800405028004076614E6953
:10EFC0002DE9F04F002383B0C0E900339B4605468E
:10EFD00000911FF019FA9C4E9C4FDFF88C82DFF8ED
:10EFE0008CA29B4C0190D946B279022A00F0B780DE
:10EFF000012A00F0C580974800228446014691F915
:10F000000430012B01F10C0140D00132082AF6D165
:10F010009049002291F90430022B01F10C0142D0F9
:10F020000132082AF6D18B49002291F90430032BD2
:10F0300001F10C0144D00132082AF6D185490022A1
:10F0400091F90430042B01F10C0146D00132082A59
:10F05000F6D1002290F90430052B00F10C0000F0ED
:10F06000A0800132082AF5D17B4A1068410640F1A0
:10F07000AE80774900220B79122B01F1140100F0C8
:10F08000F78001320F2AF6D10022F6E002EB4202AD
:10F090005CF82220002A41D16E4991F90430022BFC
:10F0A00001F10C01BCD102EB42025CF82220002AE3
:10F0B0003FD1684991F90430032B01F10C01BAD119
:10F0C00002EB42025CF82220002A3DD1614991F90D
:10F0D0000430042B01F10C01B8D102EB42025CF8C0
:10F0E0002220002AB6D05D4A217992F83DE092F8BC
:10F0F0003C208E4501D09142ABD1594A5B4601215B
:10F100000420F9F759FD0BF1010BBBF10F0F04F1CE
:10F1100014047FF469AF03B0BDE8F08F227997F84B
:10F120003D1097F83CE09142E7D072457FF470AF14
:10F13000E3E7227998F83D1098F83CE09142DCD062
:10F1400072457FF470AFD8E722799AF83D109AF8AB
:10F150003CE09142D1D072457FF470AFCDE7E268D8
:10F16000500704D522F0040242F00802E260910642
:10F170007FF541AF22F0200242F04002E2603AE720
:10F18000E268130704D522F0080242F00402E260AC
:10F1900050067FF530AF22F0400242F02002E260DC
:10F1A00029E702EB42025CF82220002A3FF45CAF20
:10F1B0002C4A217992F83D0092F83C2088429CD05C
:10F1C00091429AD0244A106841063FF552AFC203DB
:10F1D00076D42279A2F1340101298ED902F0EF020E
:10F1E000202A8AD072786AB1032A0BD0E2685006CE
:10F1F0001DD4910687D52A68911C01322A6045F8F2
:10F20000214080E7E26853070AD5019B4B4515D999
:10F2100022F0080209F10109E2605FFA89F9EAE7E0
:10F22000009B002B3FF46FAF12077FF56CAF6A684D
:10F2300005EB820101326A604C6364E7009B002B9E
:10F24000D9D01307F3D4D6E7088A00207003002032
:10F25000F01000205C89002004000010540A0020F7
:10F2600058020808A00C0020BC0500200808002057
:10F27000224B02EB820203EB820220494FF0000C8A
:10F280000B79122B01F114010BD00CF1010CBCF124
:10F290000F0FF5D1002A9AD011682268914296D1B9
:10F2A0002BE742B31268216891423FF426AF142243
:10F2B000124B02FB0CFC53F80C208A4287D11CE74E
:10F2C0000E490B79212B4FF0000201F1140108D0F7
:10F2D00001320F2A3FF47DAF0B79212B01F114018C
:10F2E000F6D1142101FB02F2044B21689A58914295
:10F2F0007FF46FAF01E72168D9E700BFF01000206D
:10F30000F0B583B005461FF07FF80C2806462BDCCD
:10F31000FDF79CFE214A224B927903EB42031B79B5
:10F32000002B32D02B68B3422BDB002E27DD1D4F84
:10F330000435002402E00134A64220D03A6855F892
:10F34000040FE1B2C2F30072FFF730F90028F2D1E6
:10F35000154D164A05260146234604202E7003B09B
:10F36000BDE8F040F9F728BC0F49114A0C230120F1
:10F3700000930870334600210420F9F71DFC03B008
:10F38000F0BD09490B4A0320F2E70B4A0221042091
:10F3900003B0BDE8F040F9F70FBC00BFD8810020F2
:10F3A0008075070804000010E4810020F8020808B6
:10F3B00070020808BC0208089C0208082DE9F04108
:10F3C000334B1E7882B00546A6B9324B1B787BB111
:10F3D000314FFFF76FF997F8081611F0FD0424D0AC
:10F3E0002E4A0221042002B0BDE8F041F9F7E4BB47
:10F3F0002B4AF6E7284F274B97F8106697F8112607
:10F400001B780136B61A002BF2D0102EE1DD25490B
:10F41000254A10230220009308703346002104205F
:10F42000F9F7CAFB02B0BDE8F0816B68B34225DB97
:10F43000002EF7DDDFF87C80303502E00134B44285
:10F44000F0D0D8F8003055F8040FB7F80226C3F30F
:10F45000007CE1B2B7F80036CDF800C0FEF7BAFF85
:10F460000028EBD10F4D114A052601462346042002
:10F470002E7002B0BDE8F041F9F79EBB094D009334
:10F4800004200B4A287033462146F9F795FBC9E75B
:10F49000548100205681002098B50020C803080838
:10F4A00020030808E48100203C030808A0030808A2
:10F4B0006803080804000010014B00221A75704709
:10F4C0008C140020014B01221A7570478C14002007
:10F4D000034A044B92F8602003EB420358797047CB
:10F4E00098B50020807507080F49104B91F86020EF
:10F4F00003EB42035B7903B9704710B50C4B1C78E2
:10F5000084B1002301EBC00E4FF0010C51F8332001
:10F510002AB112791AB1984208BF8EF806C0013399
:10F520009C42F3D110BD00BF98B50020807507083C
:10F530001810001010B5154CD4F82426D4F828362D
:10F54000D4F81C1682B002FB03F38B428DF807003F
:10F550001AD0D4F81836D4F820060DF10701184453
:10F5600066F07CFFD4F81836D4F82426D4F81C169C
:10F570001344D4F82826B3FBF1F0013201FB103319
:10F58000C4F81836C4F8282602B010BD98B500207B
:10F590000B4B10B4002203F22C6408200121C3F8A5
:10F5A0002046C3F81C065DF8044BC3F82416C3F8C4
:10F5B0001426C3F81826C3F82826C3F8382670473F
:10F5C00098B500200F4B93F86030062B17D8DFE872
:10F5D00003F00416070A0D1013004FF4C8707047AB
:10F5E0004FF4FA607047084B988870474FF47A6080
:10F5F00070474FF4FA5070474FF47A5070474FF409
:10F600007A70704798B50020D8810020034B53F8DA
:10F61000300010B103685B681879704798B5002016
:10F62000034BD3F80C2612B10F2800D810477047AF
:10F6300098B5002010B51420F7F70EFD90B10446E0
:10F64000012140F21F23C3800172F7F7D7FE216822
:10F65000114BA0884883002283F84026C3F83C461B
:10F6600083F841262520F7F7F7FC044690B140F2D5
:10F670001F220223C28003720121F7F7BFFE216817
:10F68000054BA0884883002283F84826C3F84446E7
:10F6900083F8492610BD00BF98B5002010B5037946
:10F6A000012B84B00C4621D0022B1DD18368DB07CF
:10F6B0000DF10F024CBF01218121FBF7EBFA9DF800
:10F6C0000F30114A1070C3F3C002C3F3001CC3F320
:10F6D0008001A270C3F38012DB0984F800C061705E
:10F6E000E270237104B010BD0020E8E782680DF1DC
:10F6F0000F0102F00102CDE900121A46417C90F997
:10F700001000F4F72FFDDAE78C1400202DE9F04308
:10F7100083B014460F4601AA50210546FBF70EFBA5
:10F720009DF804303C4EDFF8F490307001335B00FC
:10F73000DBB201AA238046212846FBF7FFFA237893
:10F74000DFF8DC80307009FB03F303F5FA73A8FBE4
:10F7500003239DF8042099090132DB0902FB0133E0
:10F76000A280A8FB03239B0901AAE3605121022385
:10F770002846FAF7B7FF2378BDF80410307009FB6C
:10F7800003F349BA03F5FA73A8FB0323CAB2C1F322
:10F7900007218A40013292B29909DB0902FB013349
:10F7A000E280A8FB03239B09238201AA702128463B
:10F7B000FBF7C4FA9DF80430307001335B00DBB214
:10F7C00001AA6380712102232846FAF78BFFBDF856
:10F7D0000420F978307052BAD3B2C2F307229340B2
:10F7E00001339AB2228119B1E388D31A9AB22281E5
:10F7F000A1780A4B0A4803FB01F101F5FA71A0FB5D
:10F8000001139909DB0902FB0133A0FB03239B09C8
:10F81000638203B0BDE8F0838C140020002F3A000F
:10F82000D34D62102DE9F043A84FA94CDFF8A48214
:10F830008FB006464FF000094FF4FA7309AA8921E8
:10F840000068C7F8E43087F8DA90FBF777FA9DF89C
:10F850002420207042F0010289213068FAF75CF917
:10F860004A46207088213068FAF756F90122207044
:10F8700080213068FAF750F901222070FF213068AA
:10F88000FAF74AF94A46207049463068FAF744F9CF
:10F8900009AA207091213068FBF750FA9DF82430B6
:10F8A000207001224946306887F8DC30FAF734F9D5
:10F8B0004A462070FF213068FAF72EF94A46207038
:10F8C00080213068FAF728F909AA20706021306891
:10F8D000FBF734FA9DF82420207042F012026021D8
:10F8E0003068FAF719F920250223207009AA44216B
:10F8F00030688DF825508DF82490FAF77BFEFF22B2
:10F90000207001213068FAF707F93568207001226C
:10F9100080212846FAF700F901222070FF212846AD
:10F92000FAF7FAF84A46207049462846FAF7F4F8FA
:10F9300006222070FF212846FAF7EEF809AA207067
:10F9400083212846FBF7FAF99DF82420207042F025
:10F95000040283212846FAF7DFF807222070FF21EE
:10F960002846FAF7D9F80122207081212846FAF7B3
:10F97000D3F80122207080212846FAF7CDF86B22B7
:10F98000207094212846FAF7C7F84A462070832150
:10F990002846FAF7C1F8D8F800302070C7F8E030F0
:10F9A00014E0AB68DB0709AA4FF0830128465EBF6D
:10F9B00009AA83212846FBF76DF99DF824302070B1
:10F9C00083B9D7F8E430002B40F00F832B79012B5B
:10F9D00000F0FE82022BE4D09DF82430002020703D
:10F9E000002BEED0012283212846FAF795F809AAC8
:10F9F000207092212846FBF7A1F900222070812176
:10FA000028469DF82490FAF787F806222070FF21F7
:10FA10002846FAF781F809AA207083212846FBF7C7
:10FA20008DF99DF82420207002F0FB0283212846E6
:10FA3000FAF772F801222070FF212846FAF76CF8D5
:10FA40000122207000212846FAF766F80022207073
:10FA5000FF212846FAF760F800222070802128460E
:10FA6000FAF75AF80623207007AAB0213068FAF78F
:10FA700039FE01222070FF213068FAF74DF800228C
:10FA800020704F213068FAF747F82C2220704E2161
:10FA90003068FAF741F800222070FF213068FAF749
:10FAA0003BF8B4222070B6213068FAF735F84FEAF7
:10FAB000D918B8F1000F4FF00005207018BF4FF0B3
:10FAC0000C0809F07F0EAC46012017E098B5002025
:10FAD0008C14002044350020F44503F0070317D0B0
:10FAE00011F81C2C42FA03F3DB070CF1010105F1BC
:10FAF000010548BF5FFA81FC302D12D0EBB20EAA8F
:10FB000002EBD301984503F0070200FA02F2E3D9B1
:10FB100011F81C3C013523EA0202302D01F81C2C9F
:10FB2000ECD1062307AAB0213068FAF763FD012261
:10FB30002070FF213068F9F7EFFF00221146207096
:10FB40003068F9F7E9FF00222070FF213068F9F7EB
:10FB5000E3FF0022207009213068F9F7DDFF002261
:10FB6000207010213068F9F7D7FF00222070112192
:10FB70003068F9F7D1FF0122207024213068F9F7AD
:10FB8000CBFFFF22207025213068F9F7C5FF002246
:10FB9000207075213068F9F7BFFF01222070FF2126
:10FBA0003068F9F7B9FF2C2220704E213068F9F740
:10FBB000B3FF0022207048213068F9F7ADFF2946D5
:10FBC000207020223068F9F7A7FF00222070FF2163
:10FBD0003068F9F7A1FF2946207009223068F9F74B
:10FBE0009BFF0022207054213068F9F795FF042212
:10FBF000207031213068F9F78FFF03222070322105
:10FC00003068F9F789FF8322207040213068F9F7C6
:10FC100083FF2522207046213068F9F77DFF0022FE
:10FC2000207060213068F9F777FF002220702721CB
:10FC30003068F9F771FF0622207050213068F9F71B
:10FC40006BFF0022207051213068F9F765FF962282
:10FC5000207052213068F9F75FFF0822207056218A
:10FC60003068F9F759FF2A46207057213068F9F7B4
:10FC700053FF0022207061213068F9F74DFF002208
:10FC8000207062213068F9F747FF0022207064215C
:10FC90003068F9F741FF0022207065213068F9F7DC
:10FCA0003BFFA022207066213068F9F735FF012262
:10FCB0002070FF213068F9F72FFF322220702221B7
:10FCC0003068F9F729FF1422207047213068F9F7CE
:10FCD00023FFFF22207049213068F9F71DFF002221
:10FCE00020704A213068F9F717FF00222070FF21A9
:10FCF0003068F9F711FF0A2220707A213068F9F78D
:10FD00000BFF002220707B213068F9F705FF2122CC
:10FD1000207078213068F9F7FFFE01222070FF2162
:10FD20003068F9F7F9FE3422207023213068F9F7A2
:10FD3000F3FE0022207042213068F9F7EDFEFF2229
:10FD4000207044213068F9F7E7FE26222070452113
:10FD50003068F9F7E1FE0522207046213068F9F796
:10FD6000DBFE4022114620703068F9F7D5FE0622EE
:10FD700020700E213068F9F7CFFE1A222070202162
:10FD80003068F9F7C9FE4022207043213068F9F746
:10FD9000C3FE00222070FF213068F9F7BDFE032268
:10FDA000207034213068F9F7B7FE442220703521E5
:10FDB0003068F9F7B1FE01222070FF213068F9F7B1
:10FDC000ABFE0422207031213068F9F7A5FE09222C
:10FDD00020704B213068F9F79FFE052220704C21DE
:10FDE0003068F9F799FE042220704D213068F9F748
:10FDF00093FE00222070FF213068F9F78DFE00226B
:10FE0000207044213068F9F787FE202220704521B8
:10FE10003068F9F781FE0822207047213068F9F731
:10FE20007BFE2822207048213068F9F775FE0022F9
:10FE3000207067213068F9F76FFE0422207070216E
:10FE40003068F9F769FE0122207071213068F9F7F6
:10FE500063FEFE22207072213068F9F75DFE0022F9
:10FE6000207076213068F9F757FE00222070772144
:10FE70003068F9F751FE01222070FF213068F9F750
:10FE80004BFE012220700D213068F9F745FE00225B
:10FE90002070FF213068F9F73FFE01222070802199
:10FEA0003068F9F739FEF822207001213068F9F73F
:10FEB00033FE01222070FF213068F9F72DFE012268
:10FEC00020708E213068F9F727FE01222070002172
:10FED0003068F9F721FE00222070FF213068F9F721
:10FEE0001BFE0022207080213068F9F715FE0422E5
:10FEF00020700A213068F9F70FFE3568207009AAD2
:10FF000084212846FAF71AFF9DF82420207002F079
:10FF1000EF0284212846F9F7FFFD012220700B2112
:10FF20003068F9F7F9FD05A9207030680390FFF7F4
:10FF3000B5FB039809AA05A9FFF7E8FB9DF8143063
:10FF4000002B65D00C9B03F684539DF81620002AE5
:10FF500055D00C9A02F2B22203EB42039DF817200F
:10FF600022B1BDF8342002F5257213449DF8182003
:10FF700022B1BDF8362002F2262213440121306856
:10FF8000C7F85C36E822F9F7C7FDD7F85C16207091
:10FF900044F61F639942306802D95FF005F9306872
:10FFA00001221146F9F7B8FD402120703068FDF7B5
:10FFB0008DFC50B1012130680222F9F7ADFD00211E
:10FFC00020703068FDF782FC28BB0FB0BDE8F083DD
:10FFD000AA68697C95F9100002F00102019209AA51
:10FFE00000928322F4F7BEF8E7E4D8F80020D7F8AF
:10FFF000E01092B2521A9342BFF4E8ACE5E79DF8E4
:020000040801F1
:100000001520002AAAD00C9A02F525721344A5E700
:1000100040F6363399E7E82201213068F9F77CFD94
:10002000002502234FF0200C09AA207044213068DB
:100030008DF825C08DF82450FAF7DCFAD6F8008048
:10004000207005A94046FFF729FB09AA05A94046EB
:10005000FFF75CFB502257214046F9F75DFD08226F
:10006000207056214046F9F757FD08222070502194
:100070004046F9F751FDBDF8342020704FF47A71F5
:1000800048F20E6301FB02337C4A934240F2F28055
:100090007B4AA2FB03231B0C5A1E32F0FF0309D03C
:1000A0002B465208013322F0FF019BB20029F8D100
:1000B0001B029BB21343C3F30722DBB28DF810205F
:1000C0008DF8113004AA022351214046FAF792FA22
:1000D0000C9A20704FF47A7148F20E6301FB0233E0
:1000E000684A934200F2C480654AA2FB0332120CB4
:1000F000013AD2B246214046F9F70EFDD7F85C1618
:10010000207044F61F63994202D940465FF04CF8D4
:1001100004AA01214046FAF711FE022220700121B3
:1001200040469DF81050F9F7F7FC0021207040463A
:10013000FDF7CCFB2A4601214046F9F7EDFC356876
:10014000207005A92846FFF7A9FA09AA05A928469B
:10015000FFF7DCFA482211462846F9F7DDFC0822B1
:10016000207047212846F9F7D7FC0322207032215E
:100170002846F9F7D1FC0722207030212846F9F7EC
:10018000CBFC01222070FF212846F9F7C5FC202274
:10019000207030212846F9F7BFFC00222070FF2193
:1001A0002846F9F7B9FC0622207070212846F9F795
:1001B000B3FCBDF83610344A207046F644034FF4C1
:1001C0007A7000FB0133A2FB03239DF817201B0B61
:1001D0001AB1BDF82A2013449BB2002B46D05A1EF8
:1001E00032F0FF0309D000235208013322F0FF014F
:1001F0009BB20029F8D11B029BB21343C3F3072221
:10020000DBB28DF810208DF811307121022304AA81
:100210002846FAF7EFF9D7F85C16207044F61F630A
:10022000994202D928465EF0BFFF04AA0121284660
:10023000FAF784FD02222070012128469DF8106003
:10024000F9F76AFC002120702846FDF73FFB324693
:1002500001212846F9F760FC642201232070C7F8C9
:10026000E42087F8DA300FB0BDE8F0831A46C8E71B
:10027000FF223FE72B462A4620E700BF1B0C010068
:10028000950370F41B280D014963A41310B5174C96
:1002900084F8ED10017952BAA4F8EE2001294FF04C
:1002A000000282B084F8EC2012D002290CD1042381
:1002B00004F1EC02FF21FAF747F9002814BF0020EF
:1002C0006FF00C0002B010BD6FF00C0002B010BD5A
:1002D0008268417C90F91000EC3402F00102CDE913
:1002E00000420423FF22F3F771FFE6E798B50020F0
:1002F0002DE9F04FA24FA34D066800213C4685B082
:10030000834685F8EC115A37C4F12D0905F1EC0A42
:10031000884615E0022A0FD1B26812F0010F4FF0A3
:10032000030352464FF0FF01304601BF03235246FC
:10033000FF213046FAF708F9BC421AD014F8011F21
:10034000327985F8EE1009EB0403012A85F8EC8078
:1003500085F8ED30DED1B368717C96F9100003F0BA
:100360000103CDE900A3FF220323F3F72FFFBC42D3
:10037000E4D14FF40743A5F8EC30402385F8EE3084
:1003800052460323FF213046FAF734F900238DF853
:100390000E300DF10E0130465EF0CCFE9DF80E30B1
:1003A000002BF6D04FF40640A5F8EC000120764A69
:1003B00085F8EE000323FF213046FAF71BF94FF4CE
:1003C0000740714AA5F8EC0000240323FF213046C2
:1003D00085F8EE40FAF70EF94FF40060A5F8EC004E
:1003E0000920694A85F8EE000323FF213046FAF719
:1003F00001F94FF43063A5F8EC30634A85F8EE401C
:1004000030460323FF21FAF7F5F800287FD0DBF808
:1004100000600DF10E025E213046FDF77FF9BDF858
:100420000E30B3F5D77F00F0A38079D8512B75D06B
:1004300040F29480AD2B00F09B80D62B40F08A8058
:10044000212408BB0A224B213046FEF753F90F2224
:1004500060213046FEF74EF90D2263213046FEF74B
:1004600049F9B82269213046FEF744F940F60D7289
:1004700078213046FFF70AFF40F60E627A213046B7
:10048000FFF704FF002875D0DBF8000021215EF0A3
:10049000A1FDDBF800400DF10E02DE212046FDF744
:1004A0003DF9BDF80E309FED397AC3F30903ADF87D
:1004B0000E3003EB8303DB0007EE903AF8EEE77AA9
:1004C000204667EE877A0623FCEEE77A4FF4D8449D
:1004D00017EE902A110E85F8EE10110C52BA85F81D
:1004E000EF10A5F8F020FF215246A5F8EC40FAF7EE
:1004F00081F84FF407414023DBF80000A5F8EC1029
:1005000085F8EE3052460323FF21FAF773F885F899
:10051000EC0105B0BDE8F08F1E2BB5D1142490E797
:1005200040F2E132934221D00AD940F28F42934205
:1005300003D040F291529342A6D14FF4FA7480E76F
:1005400040F2D922934211D040F2E122934209D1E4
:10055000642476E7602B3FF473AF95E71D2BDBD166
:100560000F246EE7B3F5E67FF2D08DE7C82468E785
:10057000322466E7214630465EF02CFD84E700BF5A
:100580009475070898B5002084B600209A99893F91
:1005900070B503791F4E49BA012B82B00446A6F804
:1005A000EC1015461BD0022B0AD106F1EC02FF21FC
:1005B000F9F7CAFF20B12379012B1ED0022B03D0FB
:1005C0006FF00C0002B070BD01232A46FF212046C7
:1005D000FAF732F80028F3D0002002B070BD83682B
:1005E000417CEC3603F00103CDE90063FF220223D6
:1005F00090F91000F3F7EAFDDCE7A268617C94F95A
:10060000100002F00102CDE90052FF22F3F7AAFD2B
:10061000E0E700BF98B5002003682DE9F041DF69ED
:100620001FB13B46BDE8F0411847002A164611DDD0
:1006300004460D460E4400E023689B682046984718
:100640000028F9D0236815F8011B1B68204698473D
:10065000AE42F1D1BDE8F081DEE700BF0F4B1B6871
:10066000DB0606D50E4B93F8603613F0040F18BF67
:1006700000200C4B9B7A7BB90B4A0C4B12781B6801
:100680003AB12BB11A689B8808B113837047538322
:10069000704780F00100F4E7FCF768BF000000102D
:1006A00098B50020B4820020B0820020AC820020E7
:1006B000BFF34F8F0549064BCA6802F4E06213434B
:1006C000CB60BFF34F8F00BFFDE700BF00ED00E040
:1006D0000400FA0508B572B600224FF0FF3193000E
:1006E00003F1604303F561430132082AC3F8801027
:1006F000C3F88011F3D1FFF7DBFF00BF012108B57C
:100700000846F3F7C7FEFFF7E5FF00BF00B583B06B
:100710000D49002200920091009B04330093009B3E
:100720001B68012B02D003B05DF804FB019201911C
:10073000019B064904330193019B1A600B6883F304
:1007400008884B689847FEE7502800400000FF1FCC
:1007500010B4EFF31183102282F31288094C0A4877
:1007600022684FF0E021013222608A69C0F87026C9
:100770000022C0F874260A69DBB283F311885DF8A1
:10078000044B70474435002098B5002030B4EFF397
:100790001182102383F312884FF0E023D2B29969BB
:1007A000186910F4803F0D481EBF0121C0F874166F
:1007B00099690B4B1D68D0F8743682F3118809488B
:1007C00004684FF47A7202FB04F02B44401A0021B3
:1007D000B0FBF4F030BCE3FB0201704798B5002099
:1007E00044350020E8290020124B5B68C3F308035E
:1007F000FBB9EFF31183E3B930B40F4A0F4C4FF05C
:10080000E02C1168DCF8180013688B42F9D1D4F899
:1008100070168142F5D30A4A15684FF47A7404FBC6
:1008200005F20021101AB0FBF5F0E3FB040130BC27
:100830007047ABE700ED00E04435002098B500209C
:10084000E829002090B170B5461EFFF7CDFF0446A1
:100850000D46FFF7C9FF031B61EB0502B3F57A7F75
:1008600072F10003F5D3013EEFD270BD704700BFB7
:1008700070B5006801220921F9F74EF96426FFF7E7
:10088000B3FF04460D46FFF7AFFF031B61EB050204
:10089000B3F57A7F72F10003F5D3013EEFD170BD5D
:1008A0002DE9804883B0431C0193DFF83C810A2383
:1008B0000093D8F89C10D8F8A830B8F8A000B8F881
:1008C000AC20DDF804B048834FF0320A1A834FF0B1
:1008D00005094C69204214BF4883088359690A42BC
:1008E00014BF5A831A830120FFF7B8FE56465746B5
:1008F000FFF77AFF04460D46FFF776FF001B61EB1A
:100900000501B0F57A7F71F10003F5D3013FEFD116
:10091000D8F89C30B8F8A02059690A4214BF5A830D
:100920001A83D8F8A830B8F8AC2059690A4214BF25
:100930005A831A830020FFF791FEFFF755FF044604
:100940000D46FFF751FF001B61EB0501B0F57A7F03
:1009500071F10003F5D3013EEFD1B9F1000F0BD0D7
:10096000B9F1010910D0B8F8A000D8F89C10B8F877
:10097000AC20D8F8A830ACE70BF1FF3BBBF1000F7F
:1009800019D04FF00009EEE74FF4FA76FFF72CFF8D
:1009900004460D46FFF728FF001B61EB0501B0F58B
:1009A0007A7F71F10003F5D3013EEFD14FF0FA0ADF
:1009B000BBF1000FE5D14FF47A76FFF715FF04463F
:1009C0000D46FFF711FF031B61EB0501B3F57A7FBD
:1009D00071F10003F5D3013EEFD1009B013B009381
:1009E0007FF467AFFFF78AFEF02A00200178F9B1A3
:1009F000F8B5104F0546002602E015F8011FB1B109
:100A0000D7F87846637A5A1C2344D2B2627299723C
:100A1000237A9342F1D8002AEFD004F10A01D4E9F5
:100A200000309847667215F8011F0029E8D1F8BD1B
:100A3000704700BF98B5002030B583B00F4C0190CF
:100A40000F480091FFF7D2FFDDE900320D49D4F8DD
:100A500078065CF029FFD4F878566A7A32B12B68B0
:100A6000686805F10A01984700236B7294F87C3698
:100A700013B1012384F87D3603B030BD98B5002052
:100A800004040808F1D700080FB470B582B006A9B5
:100A900051F8040B0191FFF7CFFF0E48FFF7A6FFB7
:100AA0000D4BB3F87E6636B902B0BDE8704004B0B5
:100AB0007047013EF8D0FFF797FE04460D46FFF75A
:100AC00093FE031B61EB0502B3F57A7F72F100031D
:100AD000F5D3EEE76004080898B5002000283DD063
:100AE0000378002B3AD02DE9F04F87B0584905AA7A
:100AF00065F093FE0446002800F09F804FF0000B45
:100B0000DFF87C91DFF87C81DFF87CA15D465F46F1
:100B10004FF0FF360BE0BBF1000F26D04C4905AA81
:100B2000002065F07AFE0BF1010B044610B3BBF117
:100B3000010F15D0BBF1020FEDD14946204665F0FB
:100B40004CFF00286BD045F001054146204665F07A
:100B500044FF00285CD045F00205DFE73D4893E7FD
:100B60002046F8F7A5FD0746D8E72046F8F7A0FD90
:100B70000646D3E770B2384900230C4694F90020AA
:100B8000824224D00133082B04F10C04F6D1002F4B
:100B90004CD0002D08BF03250023EDB2CDE9015351
:100BA00000971A46194628F0A9FE044600284AD0A4
:100BB0002A483A463146F7F7C9FF31462848F7F741
:100BC000C5FF284B2146D3F8F00159F0F1FA03EBA9
:100BD000430301EB83035C68002CD8D022483146E4
:100BE000F7F7B4FF5DB16179A94208D01F482A46E2
:100BF000F7F7ACFF2368E9B29B6920469847E36AA0
:100C0000002BDAD01A48F7F7A1FF0023E362D4E7FC
:100C10002046514665F0E1FE00289CD17EE715494B
:100C2000204665F0DAFE00288DD18EE71248314665
:100C3000F7F78CFF07B0BDE8F08F4FF0FF30254687
:100C40002746064697E731460C48F7F77FFFF1E75E
:100C50001C50080804050808787F00206404080870
:100C6000D404080898B50020840408089C040808E7
:100C7000BC0408082C2708081C04080844040808B9
:100C8000100408081404080818040808002868D08C
:100C90002DE9F04F90F800C085B00446BCF1000F7C
:100CA0002AD000F100475A4E8646023F014663466D
:100CB000722207E0984526D1B94212D011F8013FBF
:100CC00016F8012FA3F14105192DA2F1410098BF9B
:100CD0002033192802F12008ECD99A4213D1002AB6
:100CE000EAD14C4C0023C4F8F03D84F8F73DA4F859
:100CF000F83D05B0BDE8F08F0021012005B0BDE84A
:100D0000F04F59F0AFBA444E214663466C2207E0DB
:100D100098452AD1B94212D011F8013F16F8012F97
:100D2000A3F14105192DA2F1410098BF20331928E4
:100D300002F12008ECD99A4217D1002AEAD1374BA8
:100D40001B685B07D5D4334C94F9F63D002BD0D10A
:100D500094F9F13D002BC5DC05B0BDE8F04F50F033
:100D6000E9B80021012059F07DBA2D48732307E02E
:100D700065455BD1774513D01EF801CF10F8013FD0
:100D8000ACF141011929A3F1410298BF0CF1200CEB
:100D9000192A03F12005EBD9634547D1002BE9D18E
:100DA0001C4B002293F9F70D83F8F02D1C461646D4
:100DB00093F8A2140129A1F1030509D0052D07D943
:100DC0000EB184F8F70D174805B0BDE8F04F5BE6AB
:100DD00093F8A314A52903F1140303D00132782A50
:100DE000E6D1EDE7012803D0013840B20126F5E74E
:100DF0000D4984F8F00D0023013284F8F12D81F8BB
:100E0000803684F8F73D05B0BDE8F04F4EF0B4BE33
:100E10001005080804A500201805080800000010A7
:100E20000C1F08080405080898B50020DFF880A208
:100E30002046F8F73DFC9AF9807607FA80F5772D81
:100E4000064600F2D1802046202165F057FD8046FD
:100E5000002800F01C810346984613F8012B202A35
:100E6000FAD04046F8F724FC01245FFA80F94046A6
:100E7000202165F043FD8046002800F00D810346E7
:100E8000984613F8012B202AFAD04046F8F710FCB8
:100E900001340090E4B24046202165F02FFD8046E9
:100EA000002800F0F7800346984613F8012B202A0B
:100EB000FAD04046F8F7FCFB01340190E4B240461A
:100EC000202165F01BFD8046002800F0BF8003460E
:100ED000984613F8012B202AFAD04046F8F7E8FB91
:100EE00001340290E4B24046202165F007FD8046BF
:100EF000002800F0A9800346984613F8012B202A09
:100F0000FAD04046F8F7D4FB01340FFA80FBE4B284
:100F10004046202165F0F2FC0246002800F0B58032
:100F200003461A4613F8011B2029FAD010460392F3
:100F3000F8F7BEFB0134039A0FFA80F8E4B21046CA
:100F4000202165F0DBFC002856D003461A46013309
:100F500011782029FAD010460392F8F7A9FB039ADA
:100F600003461BB210462021039365F0C7FC039B88
:100F7000002800F0938002461046013201782029B3
:100F8000FAD00393F8F794FB04F0FD04042C039BC0
:100F900008BFC2B27FF417AFB9F1010F04D9A9F1AC
:100FA000030105293FF60FAF22B1A52A2FD0482A09
:100FB0007FF409AF3DB33B4905EB850501EB8501A6
:100FC00081F8A2940098C1F890040198C1F89404A3
:100FD0000298C1F89804A1F89CB4A1F89E84A1F8E5
:100FE000A03481F8A32484E62F49304877230022D7
:100FF00005B0BDE8F04F47E55FFA88F2034680464A
:10100000062CC9D0DFE6274981F8F75DD8E7FDB99E
:10101000244C0099C4F890140199C4F894140299CE
:10102000A4F8A03484F8A294C4F89814A4F89CB44A
:10103000A4F89E8484F8A324012301373E448AF84F
:10104000806684F8F73D54E6834661E702904AE7FC
:10105000144C009805EB850504EB8501A1F8A0343C
:1010600094F8F73DC1F890040198C1F89404013355
:10107000029881F8A294C1F89804A1F89CB4A1F850
:101080009E8481F8A3245BB2D7E7804657E70446E5
:101090008146ECE6019012E70090FCE60134E4B2F0
:1010A0000246ADE704A50020200508082C05080825
:1010B00098B500202DE9F04782B0404901AA65F0BB
:1010C000ACFB002875D04FF0000A4FF0FF343B4DC9
:1010D000D1465646D0462746BAF1040F09D8DFE874
:1010E0000AF0453F390E03000378482B47D0562BB2
:1010F00042D03348FFF7C8FC02B0BDE8F087F8F7EC
:10110000D7FA3F280646F4D8002001AA294665F000
:1011100084FB0AF1010A0028DED1BAF1040F3BD0AA
:1011200030DDBAF1050FE4D1264AF900B30103F42A
:101130007C6308F03F0843EA0803B9F1000F01D0CF
:1011400043F40053394404EB011402EB4404A4F8C3
:101150008436D1E7F8F7ACFA3F288046D4D9C8E7FF
:10116000F8F7A6FA8F280446CED9C2E7F8F7A0FA16
:1011700003280746C8D9BCE74FF00109C4E74FF080
:101180000009C1E7BAF1020FB3DC0F4923463A4622
:10119000012059F0EDF8AFE70A4A07EBC70304EB6B
:1011A000031302EB4303F900B3F88496C9F3403903
:1011B000BCE74FF0FF373C46E7E700BF1C5008088C
:1011C0000405080898B500201CBC002080B519480B
:1011D000194DFFF70BFC1948FFF708FCD5F87846C6
:1011E000627A32B12146606851F80A3B9847002381
:1011F0006372D5F8F0713B6838465B699847B0B9BF
:101200000A26FFF7F1FA04460D46FFF7EDFA031B35
:1012100061EB0502B3F57A7F72F10003F5D3013E6D
:10122000EFD13B6838465B6998470028E8D0012039
:101230000CF0E8F84C05080898B500206805080887
:1012400030B42F4C94F8043B012B86B002D006B08A
:1012500030BC704794F8093B0A2B04D0294806B0EB
:1012600030BCFFF7C3BB41218DF801102649002394
:101270001520497D8DF80200CDE90333EB20CDE93F
:101280000133A6228DF803008DF80410B22003214B
:101290008DF805008DF814308DF800208DF80610BB
:1012A000EC460DF1120541F2210083EA02230822E7
:1012B00013F4004F80EA43010ABF5B008BB29BB27C
:1012C000013AF5D1654502D01CF8012FEDE7C3F3D3
:1012D00007228DF814308DF81320EC461523C4F83E
:1012E000743BBCE80F00094D0FC59CE8030045F8AE
:1012F000040B0748297006B030BCFFF777BB00BF6E
:1013000098B50020740508088C140020BCC000208B
:1013100084050808F8B52F482F4FFFF767FB2F48C3
:10132000FFF764FBB7F87E66002E43D1D7F8784606
:10133000627A32B12146606851F80A3B984700232F
:101340006372002587F8785BC7F8B85B87F8BC5BE9
:101350001DF0F4F82248FFF749FBD7F87846627A87
:101360002AB12146606851F80A3B98476572D7F860
:10137000F0713B6838465B699847B0B90A26FFF7B9
:1013800033FA04460D46FFF72FFA031B61EB050203
:10139000B3F57A7F72F10003F5D3013EEFD13B68DC
:1013A00038465B6998470028E8D000200CF02AF8FE
:1013B000013EBBD0FFF718FA04460D46FFF714FABA
:1013C000031B61EB0502B3F57A7F72F10003F5D3DD
:1013D000EEE700BFA005080898B5002060040808E3
:1013E00068050808F8B530490522044665F09CFAFE
:1013F00018BB2E4E96F87C3623B9012286F87C263F
:1014000086F87D362A48FFF7F1FA2A48FFF7EEFA08
:10141000B6F87E6616B9F8BD013EFCD0FFF7E4F9D8
:1014200004460D46FFF7E0F9031B61EB0502B3F537
:101430007A7F72F10003F5D3EEE71F4903222046BD
:1014400065F072FA50BB194E96F87C3613B196F8D7
:101450007D36FBB91948FFF7C9FA1648FFF7C6FAF7
:10146000B6F87E763FB9002386F87C3686F87D365E
:10147000F8BD013FF7D0FFF7B7F904460D46FFF777
:10148000B3F9031B61EB0502B3F57A7F72F1000338
:10149000F5D3EEE70A48FFF7F7FAE4E7BDE8F840CE
:1014A0000848FFF7F1BA00BFCC05080898B500203E
:1014B000D405080860040808002008082406080865
:1014C000EC05080838060808F8B5244C94F87C3672
:1014D0001BB194F87D36002B34D12148FFF786FAF2
:1014E00005F0AEF81F48FFF781FAD4F878566A7A0B
:1014F00002BBD4F8F0713B6838465B699847B0B9D5
:101500000A24FFF771F905460E46FFF76DF9401BF7
:1015100061EB0601B0F57A7F71F10003F5D3013C70
:10152000EFD13B6838465B6998470028E8D0002037
:101530000BF068FF2B68686805F10A0198470023E3
:101540006B72D6E70848FFF79FFA0848FFF79CFA46
:10155000002384F87C3684F87D36F8BD98B50020E9
:101560006806080868050808EC0508084806080821
:1015700070B50C48FFF73AFA0B4BB3F87E6616B914
:1015800070BD013EFCD0FFF72FF904460D46FFF772
:101590002BF9031B61EB0502B3F57A7F72F10003AF
:1015A000F5D3EEE76004080898B5002070B504464E
:1015B0000F48FFF71BFA2046FFF718FA0D48FFF710
:1015C00015FA0D4BB3F87E6616B970BD013EFCD01E
:1015D000FFF70AF904460D46FFF706F9031B61EB16
:1015E0000502B3F57A7F72F10003F5D3EEE700BF91
:1015F000700608086004080898B50020800601D528
:10160000002933D10CB470B5194C1A49D4F87806B6
:1016100082B007AB069A01935CF046F9D4F878568D
:101620006A7A32B12B68686805F10A01984700238D
:101630006B721148FFF7DAF9B4F87E663EB9012003
:1016400002B0BDE8704002B07047013EF7D0FFF72E
:10165000CBF804460D46FFF7C7F8031B61EB050204
:10166000B3F57A7F72F10003F5D3EEE700207047FF
:1016700098B50020F1D7000860040808F0B50446CA
:1016800083B070B302785AB300F10040434D214655
:101690000238722307E0974237D1884214D011F8FC
:1016A000012F15F8013FA2F1410EBEF1190FA3F170
:1016B000410C98BF2032BCF1190F03F12007EAD981
:1016C000934222D1002BE8D1354B364AC3F8C02BC8
:1016D000C3F8C42BC3F8C82BC3F8CC2B03B0F0BDA0
:1016E0001446314D314E35F8241005EB8403324653
:1016F0005888CDE900100120234600210444FFF75B
:101700007DFF042CEFD103B0F0BD2046F7F7D0FFEA
:10171000032805462FD82046202165F0EFF804461F
:10172000002839D003461C4613F8012B202AFAD092
:101730002046F7F7BDFF012706462021204665F029
:10174000DDF8034688B1184601330278202AFAD022
:10175000F7F7AEFF4FB1A6F2EE2240F2DC539A4209
:1017600003D8A0F2EE229A420ED9114803B0BDE888
:10177000F040FFF789B90F490F480323002203B057
:10178000BDE8F040FFF780B9054B03EB8505A5F8F0
:10179000C06BA5F8C20BA1E70746CEE71005080805
:1017A00098B50020E803D00758C100207806080843
:1017B000040508088C0608082C0508082DE9F043E4
:1017C00087B040B3037807462BB300F10040564E74
:1017D00039460238722207E09C4532D1814212D04C
:1017E00011F8013F16F8012FA3F14105192DA2F1BF
:1017F000410498BF2033192C02F1200CECD99A42F5
:101800001FD1002AEAD149486022002107B0BDE873
:10181000F04365F05CB8454D454F0024D5E901061D
:1018200015F80C1B0091CDE90106012023463A462C
:1018300004440021FFF7E2FE082CEFD107B0BDE819
:10184000F0833846F7F734FFC3B2072B054647D875
:101850002021384665F052F80446002856D0034649
:101860001C4613F8012B202AFAD02046F7F720FF58
:10187000071E18BF012701262046202165F03EF8EB
:10188000044600284ED003461C4613F8012B202A9C
:10189000FAD02046F7F70CFF01368046F6B2204614
:1018A000202165F02BF8034698B39946013399F847
:1018B0000020202AF9D04846F7F7FAFE0136044600
:1018C00020214846F6B265F019F808B10136F6B2A3
:1018D000032E0ED0174807B0BDE8F043FFF7D4B889
:1018E000154916480723002207B0BDE8F043FFF76B
:1018F000CBB8134B6DB205EB450503EB850383F8BD
:10190000D07BC3F8D48BC3F8D84B97E7064607467D
:10191000B2E72021059064F0F1FF059B1C460028EA
:10192000D4D1D7E78046BAE71005080868C100207F
:101930009406080804050808AC0608082C050808E1
:1019400098B500202DE9F04184B010B10378044629
:10195000CBB9384C384F002594F8A20094F8A36016
:10196000B4F8A0100091CDE9010601202B463A46BB
:1019700005440021FFF742FE102D04F10404EBD1D1
:1019800004B0BDE8F081F7F793FE0F2805462CDC84
:101990002046202164F0B2FF044628B103461C46CD
:1019A00001332278202AFAD0244B254F28350126EE
:1019B00003EB85082046F7F77BFE37F8021B8842C9
:1019C000034606F1FF3219DC012A4FF02C012046B4
:1019D00026D0022A1CD0A8F8303C64F08FFF441CAB
:1019E00060B1032ECCD00136E4E7164916480F2328
:1019F000002204B0BDE8F041FFF746B80D4B134894
:101A0000002243F8252004B0BDE8F041FFF73CB8C0
:101A10000A4A02EB850585F8333C04B0BDE8F08145
:101A200088F8323C64F06AFF0028E7D0441C013695
:101A3000C0E700BFC8C10020BC06080898B5002058
:101A4000F0750708D00608082C05080804050808E2
:101A50002DE9F04188B0002841D003780446002BDE
:101A60003DD000252D2B5CD0A3F13002092A58D996
:101A7000202B50D163780134002BF3D1052D4AD1AE
:101A8000BDF914309AB20F2A45D8BDF91610A1F548
:101A9000FA7292B2B2F5FA6F3DD8BDF91800A0F50E
:101AA000FA7292B2B2F5FA6F35D8BDF91A40A14276
:101AB00031DCA0422FDB81422DDCBDF91C5005F149
:101AC0007D0292B2FA2A26D8204A22F8331002EB7D
:101AD000C30358809C809D7108B0BDE8F0811B4C09
:101AE000DFF870800025B4F9020094F90670B4F9AB
:101AF000046034F9081BCDE9001001202B46CDE924
:101B00000267054442460021FFF778FD102DEAD117
:101B100008B0BDE8F0810E4808B0BDE8F041FEF71E
:101B2000B3BF042DF7DC2046F7F7C2FD08AB03EB8B
:101B30004503013523F80C0C14F8013FA3F13002E2
:101B4000092AF9D9002B8DD198E700BFB480002075
:101B500004050808D8060808F0B58BB007465EF003
:101B600021FB10F0FF0432D03C4E07F1050C394642
:101B7000722205E098423FD1614512D016F8012F3C
:101B800011F8013BA3F14105192DA2F1410498BFC1
:101B90002033192C02F12000ECD99A422CD1002AD2
:101BA000EAD12F482F4A904238BF40F2FF3103D389
:101BB00020E0143090421DD20388C3F30B038B4204
:101BC000F7D129490BB0BDE8F040F7F73FBE264DED
:101BD000264FA968D5E90006CDE901060120234674
:101BE000009104443A460021FFF708FD082C05F156
:101BF0000C05EED10BB0F0BD1D4905AA384664F0C6
:101C00000CFE78B11A4E06AD0024F7F751FD05AA77
